:020000040000FA
:06000000DEEF92F0120099
:020006001200E6
:0600080004EF6AF0120093
:02000E000301EC
:0100100002ED
:020011000100EC
:020013000000EB
:060018004CEF00F01200A5
:02001E000A00D6
:1000200074270100CC050000210000006D270100AD
:10003000F60700000700000061270100F000000043
:100040000C0000002C270100C8060000350000004D
:10005000E7260100500B0000450000007B26010050
:10006000000A00006C000000EB25010060000000A9
:100070009000000013000000FE0A000002000000D3
:10008000E4250100EF070000070000001100000058
:08009000FE0400000200000064
:08009800D8CFE4FFE0CFE4FF44
:1000A000E46EDACFE4FFE2CFDAFFE9CFE4FFEACF94
:1000B000E4FFD9CFE4FFDACFE4FFFCC0E4FFFDC0EA
:1000C000E4FFFEC0E4FFFFC0E4FFF6CFE4FFF7CF9C
:1000D000E4FFF8CFE4FFF5CFE4FFF3CFE4FFF4CF84
:1000E000E4FFFACFE4FFFBCFE4FFE6523CEC8DF0F7
:1000F00010EC8CF0E552E5CFFBFFE5CFFAFFE5CF42
:10010000F4FFE5CFF3FFE5CFF5FFE5CFF8FFE5CF4F
:10011000F7FFE5CFF6FFE5CFFFF0E5CFFEF0E5CF47
:10012000FDF0E5CFFCF0E5CFDAFFE5CFD9FFE5CF75
:10013000EAFFE5CFE9FFE5CFDAFFE550E5CFE0FFE5
:10014000E5CFD8FF10000901009B1200EBEC0FF087
:1001500083E90050011003E0F5EC0FF010E1E66ACE
:10016000F8EC0FF08AEC10F0A2EC85F044E90B01FA
:10017000D60ED16F060ED1CBF3FFF46E04D000EB98
:10018000F3FF01EBF4FFD0EF10F0DCEC11F041E8ED
:100190000B01CFBF03D00B01300ED06FD950010F30
:1001A000E66EDACFE6FF0BEC8DF042E9000901E1E3
:1001B00018D10AEC11F001E0C3D0C85103E07F0E62
:1001C000C85D21E10A0E015CE9E00D0E015C03E16E
:1001D0000A0E016E18D0080E015C07E1EA51000812
:1001E000DDE2EA07A5EC11F0D9D7010403E0030E24
:1001F000015C09E1EA6B4B0EE66EC70EE66E000E7F
:10020000F0EC0FF0CBD70D0E015CC8E091EC11F0D3
:1002100083EC10F004E1D25102E10601EA073A0E44
:10022000015C2AE1060E0601EA5D26E30EEC11F000
:1002300023E1490E015D20E1500E025D1DE1440EF7
:10024000035D1AE109010051100B16E10B01CFBF4C
:1002500003D00B01310ED06F0601EA05D7EC0FF089
:10026000EF6A050EE66E080EE66E1AEC11F03C0E13
:10027000ED6FEA6BFD0E62D00A0E015C8FE10B019F
:10028000CFBF03D00B01320ED06F0601EA07A5ECF9
:1002900011F0040EEA5D01E27BD00EEC11F001E0FA
:1002A00077D0430E015D74E14D0E025D71E1540E95
:1002B000035D6EE109010051100B6AE1070E016E4A
:1002C0000150D7EC0FF0EF50220806E00601EA518A
:1002D000015C02E2012AF4D70150D7EC0FF0EF6A7B
:1002E000140EE66EE66A070EE66E080EE66E8AECFF
:1002F00010F03AEC86F046E90601E96BEA51016E2E
:100300000150D7EC0FF0EF502C0804E0015002E050
:100310000106F6D701500B01D26B000FD16F080E0A
:10032000D223D12B000ED223D1CBE6FFD2CBE6FFD6
:100330001AEC11F00A0EED6FEA6BFE0EEB6F2ED782
:10034000FE0EEB5D29E10B01CFBF03D00B01330E95
:10035000D06F0D0E015C03E00A0E015C08E106019E
:10036000EA51EA2BD7EC0FF0200EEF6E03D0060116
:1003700091EC11F083EC10F004E1D25102E106019E
:10038000EA070601EC07EC5101E008D7A5EC11F0F3
:10039000CCEC05F0060122D00B01CFBF03D00B013E
:1003A000340ED06F0D0E015C0AE0060191EC11F0E5
:1003B00083EC10F004E1D25102E10601EA070601E4
:1003C000EC070A0E015C07E1EA07A5EC11F0CCECA2
:1003D00005F00601EA6BEC5101E0E0D6EA6BEB694F
:1003E000DDD60601A5EC11F0D4EF10F0DCEC11F035
:1003F00042E8090100B305D000A3FED7050E36EC94
:1004000011F0016A0901C451026E0A0E015C0AE290
:10041000D1EC3DF002500901C45D02E0016AF3D75E
:10042000012AF1D73BEF11F0DCEC11F044E8880E23
:10043000036E130E046E800EE66EE66A7E0E00EC0E
:1004400010F0016E800EE66EE66A7F0E00EC10F092
:10045000026E3E0E015C05E1200E025C02E1010E1F
:1004600022D0450E015C05E1520E025C02E1000E55
:100470001AD0010EE66EBEEC92F041E90306000EC2
:10048000045A03EBD1FB04EBD2FB0B01D151D21187
:10049000D2E10601D4510108000ED55503E2D4077C
:1004A000000ED55B000E45E9E7CFD9FF1200EBEC5B
:1004B0000FF084E941E80801CF51D0110FE0DFECE3
:1004C00011F001E17ED03FEC11F001E37AD0DFECD6
:1004D00011F0E9EC11F0A2EC10F0F1D77F0E06015B
:1004E000C85D61E1046ADFEC11F00A080BE10D0E52
:1004F000045C08E0090100B1FDD70D0EE0EC0FF03F
:1005000020E1FBD70D0E045C1CE1DFEC11F00A08C2
:1005100018E0090100B1FDD70A0EE0EC0FF0FCE095
:100520000B0151510EE0090100B1FDD7230EE0ECA3
:100530000FF0FCE0090100B1FDD7200EE0EC0FF058
:10054000FCE0DFEC11F03DE0090100B1FDD7CFEC9C
:100550000FF021EC11F0FBE00B01515112E0DFEC48
:1005600011F00A080EE1090100B1FDD7230EE0ECFD
:100570000FF0FCE0090100B1FDD7200EE0EC0FF018
:10058000FCE0D9CFE9FFDACFEAFFEFCFF6FFEE2AA2
:10059000EFCFF7FF000EEE22EFCFF8FFEE220800BC
:1005A000F550046EA0D7DFEC11F00BE0090100B1AB
:1005B000FDD7CFEC0FF021EC11F0FBE0A2EC10F036
:1005C000F2D7D4EF10F0EBEC0FF083E941E808012B
:1005D000CF51D0110FE0F5EC0FF001E171D03FECFD
:1005E00011F06EE2F5EC0FF0E9EC11F0002A000ECC
:1005F0000122F1D77F0E0601C85D55E1036AF5ECD3
:100600000FF00A080BE10D0E035C08E0090100B1D0
:10061000FDD70D0EE0EC0FF020E1FBD70D0E035CD3
:100620001CE1F5EC0FF00A0818E0090100B1FDD754
:100630000A0EE0EC0FF0FCE00B0151510EE0090155
:1006400000B1FDD7230EE0EC0FF0FCE0090100B192
:10065000FDD7200EE0EC0FF0FCE0F5EC0FF030E001
:10066000090100B1FDD775EC10F0FDE00B0151510F
:1006700012E0F5EC0FF00A080EE1090100B1FDD718
:10068000230EE0EC0FF0FCE0090100B1FDD7200ED5
:10069000E0EC0FF0FCE0FDEC11F0002A000E01226E
:1006A000EF50036EACD7F5EC0FF00AE0090100B192
:1006B000FDD775EC10F0FDE0002A000E0122F3D703
:1006C000D4EF10F0EBEC0FF082E90801CF51D0111C
:1006D00008E03FEC11F00FE262EC10F000EBEFFFEE
:1006E0000AD0090100B1FDD700EBE6FFE1EC8CF088
:1006F00041E90009F9E0D0EF10F0EBEC0FF087E9E9
:10070000045005101FE00601F751041802E1F851EA
:10071000051814E0080E0B01CC1510E104EBF1F6FE
:1007200005EBF2F600EBF3F601EBF4F602EBF5F66F
:1007300003EBF6F604EBF7F605EBF8F606013C0ED4
:10074000F96F05D0D8EC10F0F76BF86BF96BD0EFC0
:1007500010F0EBEC0FF083E942E8030EE66ED7EC05
:1007600011F0036EF450046E470EE66EC70EE66E8F
:10077000000E34EC10F00AE000EBD2FBD16BD1514B
:100780000601FA130B01D2510601FB13440EE66E6B
:10079000C70EE66E000E34EC10F005E006010050C6
:1007A000FA130150FB133BEF11F0EBEC0FF083E970
:1007B00046E897EC11F000EBE6FF01EBE6FFEFEC0B
:1007C00011F05BE0DDEC0FF0C5EC10F056E0E2EC70
:1007D00011F053E0E2EC11F050E005EBE9FF06EB1D
:1007E000EAFFEF504F0849E10528E96E000E0620A8
:1007F000EA6EEF502D0841E124EC11F0020E0B01DE
:100800000524D16F000E0620D26FD1CBE6FFE66E35
:10081000EFEC11F032E024EC11F082EC11F0056EF7
:10082000F450066E94EC10F0D7EC11F0076EF45013
:10083000086E055006100BE107EBE9FF08EBEAFF35
:10084000EF501BE03F0EE66EC70EE66E11D005EBD3
:10085000E6FF06EBE6FF07EBE6FF08EBE6FF6CECD6
:1008600085F044E9000909E005EBE6FF06EBE6FF49
:1008700094EC10F02DEC8BF043E947E9E7CFD9FF7A
:100880001200EBEC0FF082E942E800EBC8F606013B
:10089000C851240A01E172D1070A01E164D1010AB9
:1008A00001E15BD1030A01E12BD1010A01E112D17F
:1008B000600A01E1F1D0030A01E1D1D0010A01E1AE
:1008C000A7D0030A01E191D0530A01E17ED0030AC7
:1008D00071E0010A5CE0160A4CE0030A3FE0010AFD
:1008E00036E0070A26E0010A22E0030A14E07E0A45
:1008F0000FE07F0A01E04ED13C0ED46FD56B51EC76
:1009000010F00601010ECD6F0A0ECE6FCF6B42D1F3
:1009100074EC72F03FD10A0EBAEC0FF00601030E30
:10092000CD6F140ECE6FCF6B23EC12F033D1CD6BA5
:1009300031D151EC10F00BEC3EF00BEC3EF0060127
:10094000020ECD6FCBEC10F00601CC6B23D1050E5F
:10095000CD6F030ECBEC10F00A0EB1D0060ECD6FAA
:10096000020ECE6FCF6BC96B0BEC3EF00BEC3EF082
:1009700011D1E66A5FEC11F065EC11F00B01CFBF0D
:1009800003D00B01F00ED06FCFEC3DF003D1090E78
:10099000BAEC0FF0E0EC10F0EEA106D0430EE66EDC
:1009A000200EE66E010ED6D05A0EE66E200EE66ED2
:1009B000010ED0D0080EBAEC0FF0E0EC10F0660E8D
:1009C000E66E200EE66E010EC5D0070EBAEC0FF0F3
:1009D0000601030ECD6F230ECE6FCF6BC96B810E58
:1009E000E66E200EE66E010EB5D0050E07EC12F095
:1009F000ABEC10F006E2070E2BEC10F00601400EF7
:100A000005D0080E2BEC10F00601020ECD6F14D0AD
:100A1000050E07EC12F0260EE66EC70EE66E000E0F
:100A2000F0EC0FF0090E2BEC10F0ABEC10F002E242
:100A3000430E01D0020ECD6FCAC6CEF6CBC6CFF69E
:100A40000A0ED880CE57000ECF57050ECF03F3CF36
:100A5000CFF6CE03F3CFCEF6F450CF279BD0050EC2
:100A6000BAEC0FF044EC10F00601020ECD6F3C0E14
:100A7000CE6FCF6B070EC96F2CEC12F0020E6AEC32
:100A800010F00E0EE66EC70EE66E000EF0EC0FF0E4
:100A90000601400EC86F7ED0050EBAEC0FF044EC94
:100AA00010F057EC10F013E0A1EC90F000090FE00B
:100AB0000601020ECD6F3C0ECBEC10F0020E6AEC7C
:100AC00010F0330EE66EC70EE66E000E43D0060140
:100AD000200EC86F020EBAEC0FF00B01516B06012D
:100AE000CD6BC96B0001C80507E0050EC85D04E0C9
:100AF000780E0601D26F02D00601D26BD36B4AD0BA
:100B0000060EBAEC0FF0020E6AEC10F00601030EAE
:100B1000CD6F780ECE6FCF6B2CEC12F00D0E57EC24
:100B200010F006E1DE0EE66E200EE66E010E12D02B
:100B3000000EE66EC70EE66E000EF0EC0FF002EB54
:100B4000E6FF03EBE6FF53EC11F0F60EE66EC60E81
:100B5000E66E000EF0EC0FF01DD00A0ECE6FCF6BDC
:100B6000400ECD6F17D0060EBAEC0FF00601240E22
:100B7000CD6F2C0ECE6F010ECF6F0CD0CC51CC2B85
:100B80000B01D16F140ED15D02E2020E01D0030EF3
:100B900044EC11F03BEF11F0DCEC11F05DE80601E4
:100BA000ED6B3C0ED46FD56B0B01CFBF03D00B01A7
:100BB000350ED06FFE0E0601EB5D20E10001C80589
:100BC00007E0050EC85D04E044EC10F065EC11F0A0
:100BD0000B01CFBF03D00B01360ED06F73EC11F0B9
:100BE0008AEC10F0FEEC50F044E90B01CFBF06EFA9
:100BF0000BF00B01350ED06F06EF0BF0FF0EEB5D27
:100C000015E00B01CFBF03D00B01370ED06F73EC93
:100C100011F0CFEC18F042E90B01CFBF03D00B016C
:100C2000350ED06F49EC11F006EF0BF0C8517F0A7A
:100C300002E101EF0BF05F0A01E144D2600A01E139
:100C40006ED1630A01E151D1020A01E106D1330AF2
:100C500001E1DAD0030A6EE0010A2CE0110A16E085
:100C6000010A02E006EF0BF0050EEA5D02E206EF74
:100C70000BF09EEC10F0F00EE66EC60EE66E000E67
:100C8000AFEC0FF002E006EF0BF038D0020EEA5D99
:100C900002E206EF0BF012EC11F002E006EF0BF0AF
:100CA0004B0E015D02E006EF0BF065EC11F0100E4B
:100CB000EEEF0AF0040EEA5D24E30EEC11F021E100
:100CC000430E015D1EE1530E025D1BE14D0E035DFF
:100CD00018E173EC11F0DCEC85F042E9F3CFE9FFA9
:100CE000F4CFEAFFE906000EEA5A000EE926080EE4
:100CF000EA22EF50310802E106EF0BF07F0EEEEF33
:100D00000AF00601C95102E006EF0BF0020EEA5D9F
:100D100002E206EF0BF012EC11F002E006EF0BF02E
:100D20004B0E015D02E006EF0BF065EC11F0110EC9
:100D3000EEEF0AF0100EEA5D17E3380E0801005DD1
:100D400013E1390E015D10E1180EE66EE66A73ECF0
:100D500011F0A60EE66E0B0EE66E3AEC86F046E952
:100D60000B01BD6B06EF0BF0080E0601EA5D16E302
:100D70000EEC11F013E1430E015D10E1500E025D27
:100D80000DE1420E035D0AE1460E045D07E13A0EF5
:100D9000055D04E173EC11F008DDB9D1080E060120
:100DA000EA5D19E30EEC11F016E1430E015D13E16B
:100DB000500E025D10E1490E035D0DE1520E075D1C
:100DC00002E106EF0BF0040E2BEC10F00601010E11
:100DD000C96F06EF0BF00601C95102E006EF0BF0F8
:100DE000020EEA5D02E206EF0BF012EC11F002E0F7
:100DF00006EF0BF04B0E015D02E006EF0BF065EC29
:100E000011F0120EEEEF0AF0060EEA5D15E30EEC9D
:100E100011F012E1490E015D0FE1500E025D0CE18F
:100E2000520E035D09E1390E065D06E0220EE66E04
:100E3000210EE66E010E89D1020E0601EA5D01E285
:100E4000E5D312EC11F001E0E1D34B0E015D01E0BE
:100E5000DDD365EC11F0210EC1D3020EEA5D0BE388
:100E600012EC11F008E14B0E015D05E149EC11F0C7
:100E7000CC6B220EB3D3050E0601EA5D07E3450EE7
:100E80000801005D03E1520E015D03E057EC11F033
:100E900002E1230EA3D3060EE66EE66ADE0EE66ED0
:100EA000C60EE66E000EAFEC0FF001E0AFD397EC8C
:100EB00011F0000EE66E080E20EC10F001E1A6D352
:100EC000DDEC0FF0CCEC11F001E1A0D3080EE66EE2
:100ED000E66A1BEC10F0CE0EE66E000EE66E3AEC03
:100EE00086F046E90001D66B91D3A9EC11F001E040
:100EF0008DD32C0E0801085D03E1070E091502D001
:100F0000070E07150001C86FE80404E0050EC85D70
:100F100001E07CD349EC11F0CC6B400E5FD3020EA4
:100F2000EA5D07E3450E0801005D03E1520E015D35
:100F300003E057EC11F00FE1020E0601C95D01E17B
:100F400024D3030EC95D01E120D3050EC95D01E084
:100F50005DD3030E43D3020E0601EA5D06E312ECF5
:100F600011F003E14B0E015D0CE0530E0801005D32
:100F700003E1480E015D05E0050E0601C95D01E0D3
:100F80008DD00601EA6B1E0ECE6FCF6B0001C96BD0
:100F9000020E6AEC10F00601C92BC951090A01E1E1
:100FA0007BD0010A63E00F0A5BE0010A3BE0030A21
:100FB00033E0010A2BE0070A20E0010A0CE0030AF3
:100FC00001E024D3C40EE66EC60EE66E000EF0EC11
:100FD0000FF0050E0ED0B70EE66EC60EE66E000ED2
:100FE000F0EC0FF0050E78EC11F0060E78EC11F035
:100FF000070EE66EF8EC0FF02BD0040E07EC12F0A3
:10100000A90EE66EC60EE66E000E9FD09B0EE66E33
:10101000C60EE66E000E99D0910EE66EC60EE66E16
:10102000000E93D0160EE66EE8EC10F06FEC10F0A8
:1010300006E18D0EE66EC60EE66E000E86D0800EC0
:10104000E66EC60EE66E000EF0EC0FF01BEC10F034
:1010500053EC11F0C10EE66EC60EE66E000E75D0B2
:101060000E0EE66EC70EE66E000E6FD0030E07EC96
:1010700012F06C0EE66EC60EE66E000EF0EC0FF08F
:10108000040EE66EF8EC0FF053EC11F0620EE66E13
:10109000C60EE66E000E59D0200EA0D2070EEA5DF5
:1010A0000BE3080EE66EE66A590EE66EC60EE66EB5
:1010B000000EAFEC0FF004E087EC11F001E0A6D2D7
:1010C000020E8CD2A9EC11F024E12C0E0801085D6F
:1010D00003E1070E091502D0070E07150001C86FBE
:1010E000E80403E0050EC85D05E10601D26BD36B91
:1010F000E66A0AD00601D251D31101E087D2780EF8
:10110000D26FD36B010EE66EE66AD9EC8BF042E942
:101110007DD29EEC10F0470EE66EC60EE66E000E17
:10112000AFEC0FF015E10001C80507E0050EC85D42
:1011300004E044EC10F065EC11F0010E6AEC10F0E4
:10114000F20EE66E200EE66E010EF0EC0FF05ED2AF
:101150009EEC10F0410EE66EC60EE66E000EAFEC91
:101160000FF001E09CD0080E0601EE15000801E327
:101170004DD2070EE66E080EE66E52EC42F016EC0B
:1011800010F0036ED251046ED351056ED451066E29
:1011900003500001881908E10450891905E1055040
:1011A0008A1902E106508B1901E130D20350885DA3
:1011B0000450895905508A5906508B5938E2D95044
:1011C000030FE96EDACFEAFF8851EE5C0B01D16FB5
:1011D00000018951EE580B01D26F00018A51EE587F
:1011E0000B01D36F00018B51EE580B01D46FD1511D
:1011F000076ED251086ED351096ED4510A6E0001A8
:101200008C518D118E118F1108E007508C270850DA
:101210008D2309508E230A508F2300010750882701
:101220000850892309508A230A508B23EFD1D950C3
:10123000030FE96EDACFEAFFEE50885D0B01D16F44
:10124000EE50000189590B01D26FEE5000018A590E
:101250000B01D36FEE5000018B590B01D46FD151AC
:101260000B6ED2510C6ED3510D6ED4510E6E000127
:101270008C518D118E118F1108E00B508C5F0C502A
:101280008D5B0D508E5B0E508F5B00010B50885FA5
:101290000C50895B0D508A5B0E508B5BB7D1020EF0
:1012A000E66EE66A3E0EE66EC60EE66E000EAFEC29
:1012B0000FF001E07AD04EEC11F001E376D09EEC15
:1012C00011F0020EE66E080E20EC10F0B6EC0FF0F6
:1012D00004E0F2EC11F0EDEC10F0B6EC0FF003E0EE
:1012E0006FEC10F0176EB6EC0FF004E0F2EC11F0BA
:1012F000F5EC10F0B6EC0FF003E06FEC10F0186EA8
:10130000B6EC0FF003E06FEC10F0196EB6EC0FF0D6
:10131000B6EC0FF0B6EC0FF005E0F7EC11F01A6E3A
:10132000F4501B6E0150021001E170D1010E19142E
:101330000001C26FC25136E0530E175C0CE10FEB97
:10134000D1FB10EBD2FB11EBD3FB12EBD4FB2BEC5C
:1013500011F0EDEC10F0570E185C0CE113EBD1FB23
:1013600014EBD2FB15EBD3FB16EBD4FB2BEC11F0FB
:10137000F5EC10F00FEB9AFB10EB9BFB11EB9CFBD9
:1013800012EB9DFB13EB9EFB14EB9FFB15EBA0FBFD
:1013900016EBA1FB1AEBA4FB1BEBA5FB0001780EDF
:1013A000C56F34D10001C56B31D1030EE66EE66A1C
:1013B000380EE66EC60EE66E000EAFEC0FF01DE1C5
:1013C0004EEC11F01AE29EEC11F0030EE66E080EE0
:1013D00020EC10F005E0F7EC11F01C6EF4501D6EDF
:1013E0000150021001E112D10001C25101E10ED100
:1013F0001CEBA2FB1DEBA3FB09D116EC11F02D0E8B
:10140000E66EC60EE66E000EAFEC0FF004E10001D2
:10141000C95126E119D0070EE66EE66A250EE66E82
:10142000C60EE66E000EAFEC0FF042E1110EE66E56
:10143000E66A130EE66EC60EE66E000EAFEC0FF017
:1014400013E10001C9510CE1010EE66EE66ED9EC24
:101450008BF042E932EC12F0E9EC12F04EEC12F0B3
:101460000001010EC96FD2D0150EE66EE66AFD0EC0
:10147000E66EC50EE66E000EAFEC0FF001E1C6D0D1
:10148000110EE66EE66AEB0EE66EC50EE66E000E17
:10149000AFEC0FF06BE00001C96B020E07EC12F02D
:1014A0000001C80570E0050EC85D01E0AFD06BD04B
:1014B0009EEC10F0E50EE66EC50EE66E000EAFEC8B
:1014C0000FF011E12C0E0801085D08E1070E06156A
:1014D0000A0D070E07150B01F32402D0070E06159F
:1014E0000001CB6F93D0070EE66EE66ADD0EE66E66
:1014F000C50EE66E000EAFEC0FF00BE00B0EE66EC5
:10150000E66AD10EE66EC50EE66E000EAFEC0FF089
:1015100003E10B0151697AD0060EE66EE66ACA0E47
:10152000E66EC50EE66E000EAFEC0FF01FE00C0E7F
:10153000E66EE66ABD0EE66EC50EE66E000EAFEC18
:101540000FF014E00B01515115E0090EE66EE66A4A
:10155000B30EE66EC50EE66E000EAFEC0FF006E0C1
:10156000B1EC11F003E057EC11F004E12CEC12F0B7
:10157000420E34D087EC11F006E0B1EC11F003E03C
:1015800057EC11F004E12CEC12F0410E27D0040EC0
:10159000E66EE66AA90EE66EC50EE66E000EAFECCC
:1015A0000FF00BE0060EE66EE66AA20EE66EC50EC2
:1015B000E66E000EAFEC0FF003E12CEC12F00DD054
:1015C000110EE66EE66A900EE66EC50EE66E000E31
:1015D000AFEC0FF006E10BEC3EF0010E44EC11F025
:1015E00015D0060EE66EE66A890EE66EC50EE66E4C
:1015F000000EAFEC0FF00AE132EC11F0F7EC1BF04B
:1016000004D032EC11F02EEC75F043E95EE9E7CF3F
:10161000D9FF1200DCEC11F046E87F0E0601C85D30
:101620000BE0200EC85D01E03BD10001C80504E0DD
:10163000050EC85D01E034D10B01515101E030D1FC
:101640000AEC11F001E02CD1EA5101E029D10901A5
:10165000415101E025D10901C45101E021D10B0123
:101660009151921103E00B01500549E00601F1513F
:101670000008000EF2551BE20B01500518E10601AF
:10168000F1510008000EF2550FE2F3C6E6FFF4C672
:10169000E6FFF5C6E6FFF6C6E6FFF1C6E6FFF2C6D0
:1016A000E6FF74EC1FF046E9D8EC10F0F9D0FF0E1D
:1016B000C5EC0FF001E39BD00B01500501E097D082
:1016C000200EC5EC0FF004E20601FA9B040E33D0A5
:1016D000040EC5EC0FF016E20601FA95FC5101E08C
:1016E000DFD0060E0B01916F926B0B01D950020FE8
:1016F000936FDACF94FBE96EDACFEAFFEF6A7BEC07
:101700001BF0CED0080EC5EC0FF006E20601FA97EA
:10171000EEA3C6D0020E0FD0100EC5EC0FF004E2FF
:101720000601FA99030E07D0400EC5EC0FF008E24F
:101730000601FA9D050EE66E63EC1FF041E9B0D09C
:10174000010EC5EC0FF02DE27C0E0601FA17FB6BC3
:10175000020E016E01EBE6FF8BEC13F08FEC10F044
:1017600033EC16F08FEC10F0E4EC14F041E9016E6C
:10177000010EFDEC10F0020EFDEC10F001EBE6FFA7
:1017800053EC15F08FEC10F0D1EC15F08FEC10F05D
:10179000FDEC16F041E9016E020E015C01E180D022
:1017A00023D0020EC5EC0FF012E20601FA93020EEE
:1017B000016E01EBE6FF33EC16F08FEC10F08BECD2
:1017C00013F041E9016E020E015C6AE00DD0800E5B
:1017D000DCDB0DE20601FA9FFB6B020EE66EE4EC29
:1017E00014F041E902085CE04EEC12F059D02EEC06
:1017F00010F07C0EE2EC0FF053E2000EE66EE66AAB
:10180000A6EC00F042E92EEC10F0200EDBDB04E247
:101810000601FB9B040E3ED02EEC10F0040ED2DB32
:101820001DE20601FB95FC513BE1840EE66EC50E00
:10183000E66E000EE66ED950020FE66EDACFE6FFD6
:1018400019EC43F045E9D950020FE66EDACFE6FF16
:101850008AEC10F0FEEC50F044E922D02EEC10F0AF
:10186000080EB0DB06E20601FB97EEA319D0020ECC
:1018700011D02EEC10F0100EA5DB04E20601FB994E
:10188000030E08D02EEC10F0400E9CDB09E206019E
:10189000FB9D050EE66E8AEC10F052EC4AF043E92F
:1018A00047E9E7CFD9FF12000B01CFBF03D00B01EF
:1018B000380ED06F0601F951000805E2F907F95119
:1018C00002E1F76BF86BC8517F0A01E1FAD05F0AB9
:1018D00001E171D0220A6DE0210A54E0020A49E0D8
:1018E000330A3CE0030A30E0010A24E0110A01E077
:1018F00012000A0ECE1908E1CF5106E10BEC3EF0C2
:10190000320E6AEC10F007D0050ECE5D000ECF59F6
:1019100002E2020EA0DB0601EEA106D0020EE66E88
:10192000200EE66E010E23D0100EE66E200EE66E3F
:10193000010E1DD06EEC11F001E0C5D05A0EE66E1E
:10194000200EE66E010E13D06EEC11F001E0BBD05C
:10195000660EE66E200EE66E010E09D06EEC11F0FA
:1019600001E0B1D0810EE66E200EE66E010EF0EFC2
:101970000FF0140ECE5D000ECF5901E3A4D0060E79
:101980002BEF10F016EC11F00AEC12F001E09BD0F6
:10199000F6EC01F0180EE66E210EE66E010E20DB6D
:1019A000090141510008FCE3020EE66EDFEC3DF058
:1019B00033D0E66A2FD0FF0EEB5D0AE0ED0504E1BF
:1019C000ED6BEA6BEB690FD0ED51010801E2ED0719
:1019D000D2510008000ED35508E2D207000ED35BA7
:1019E000D251D31102E1210E14D00B01515116E056
:1019F000512B3C0EE76E511902E7513502D051517F
:101A0000E75C0CE20601D251D31102E1420E01D093
:101A1000400EE66E41EC04F041E912000001715104
:101A2000800B04E011DB01E1D2510DE03C0EB9EC7A
:101A300011F0E5CFD4FBE7CFD3FB0B01370ED31961
:101A40001FE1D4511DE10B0151511AE1E3DB18E113
:101A5000EA5116E10901415113E10901C45110E1B4
:101A60004EEC11F00DE21E0EE66E200EE66E010E3B
:101A7000B7DA090141510008FCE30F0E36EC11F012
:101A80000001C80503E0050EC85D15E100017751AE
:101A9000000811E20B01C6050EE10001CA51000861
:101AA0000AE2010E0601EE1504E0CEDA04E1D2519D
:101AB00002E1800EF0DA000175A905D00001CD6BBE
:101AC000120087EC72F012000B01CFBF03D00B01A4
:101AD000390ED06F0601C851200A01E012003C0EF9
:101AE00010EC12F01FE00B0151510AE193DB08E109
:101AF000EA5106E10901415103E10901C45106E03F
:101B0000020E0601D05F000ED15B1200F70EE66EEA
:101B1000200EE66E010E64DA090141510008FCE373
:101B2000020EA4DB12000B01CFBF03D00B013A0E53
:101B3000D06F0001CC510DE117DBC3EC11F0D9DA05
:101B400045EC5EF041E9E7500001CC6F0001CD6B40
:101B50002AD0020EE66EE66A07DBFCC0D7FBFDC0AA
:101B6000D8FBFEC0D9FBFFC0DAFBC3DA7EEC5EF027
:101B7000E552E5CFD6FBE7CFD5FB0001CC510B01F9
:101B8000D525D36F000ED621D46FD32B000ED423CE
:101B9000D3CBE6FFD4CBE6FF4AEC5FF0E55202EC94
:101BA00012F0D1CBCCF0000175B918D00F0E0001A6
:101BB000CD5D09E2000171AF03D00001CD6B0ED005
:101BC0000001CD2B0BD00F0ECD5D08E1000171514E
:101BD000800B04E1CCC0CDF000010E930001CD518B
:101BE0000F081DE2000171AF03D000010E9317D062
:101BF000020E00010E1507E10001CC51730803E34A
:101C000000010E830AD0020E00010E1508E07D0EC1
:101C10000001CC5D04E300010E93080E3CDA0601DE
:101C2000C851200A01E012000B0150511DE0ABEC3D
:101C30007CF0000819E20B0151510AE1EBDA08E1EE
:101C4000EA5106E10901415103E10901C45106E0ED
:101C5000040E0601D05F000ED15B06D032EC12F00C
:101C6000AEEC7CF04EEF12F00001CA51000802E227
:101C7000010E11DA010E0601C919C96F12000B011C
:101C8000CFBF03D00B013B0ED06F120095DB43E8B2
:101C9000000166050DE0020E665D0AE00F0E665D4E
:101CA00007E0800E00017115000802E3000E01D06C
:101CB000010E036E0B01CFBF03D00B013C0ED06FA2
:101CC0000601C851200A4BE10001EF510001785D87
:101CD00038E2800E0001711534E10601F0511CE17B
:101CE0000B0150511AE00B01515117E193DA15E144
:101CF000EA5113E10901415110E10901C4510DE11B
:101D00000601EEA505D0010EE66E63EC1FF041E979
:101D10000601480EF06F01D0F0070601EF510FE108
:101D2000E66A56DA0601EEA506D0010EE66E83D904
:101D300052EC4AF043E90601480EEF6F06D0EF0778
:101D400004D00601060EEF6FF06F0B01505107E053
:101D50000001CA5104E1035002E0010E9CD944E99C
:101D6000E7CFD9FF120028DB41E8000166050DE04E
:101D7000020E665D0AE00F0E665D07E0800E000150
:101D80007115000802E3000E01D0010E016E0B0177
:101D9000CFBF03D00B013D0ED06F0601C851200A02
:101DA0000AE10B01505107E00001CA5104E1015062
:101DB00002E1010E70D9F8D10B01CFBF03D00B01A6
:101DC0003E0ED06F0601FC51000801E2FC07D02B4B
:101DD000000ED123CD51000811E2CEC6D1FBCFC6F3
:101DE000D2FBCE07000ECF5B0B01D151D21106E121
:101DF000CDC6E6FF41EC04F041E901D055DD1E0EF1
:101E00000FDB01E161DE3C0E0BDB01E18CDE2C0E11
:101E1000E66E010EE66E5CDA01E131DF580EE66E29
:101E2000020EE66E55DA01E131DF100EE66E0E0E9F
:101E3000E66E4EDA06E197DF100E0601D05F0E0E59
:101E4000D15B7F0E0601C85D15E0D407000ED55B9F
:101E5000D451D5110FE13C0ED46FD56B0B01CFBF20
:101E600003D00B01F10ED06F010E0EDA0B0E06013E
:101E7000CE6FCF6B12001200C5EC8CF00001C86B66
:101E8000E66A41EC04F041E91200A5D884E900506B
:101E9000050A55E0010A4DE0070A45E0010A1AE08B
:101EA000030A58E100017851E66EE66A5B0EE66EC1
:101EB000C50EE66E000EE66E000EE66E070EE66ECE
:101EC0006DEC43F047E9B0DA540EE66EC50EE66EEF
:101ED000000E3AD000010EA307D04ED9340EE66EA4
:101EE000C50EE66E000E06D047D9230EE66EC50E6F
:101EF000E66E000EE66E9FD888D9010EE66EE66AA1
:101F0000CDC0E6FFE66AE66AE66A1B0EE66EC50E1F
:101F1000E66E000EE66E8FD878D9180EE66EC50E06
:101F2000E66E000E11D0F40EE66EC40EE66E000EE4
:101F30000BD0D90EE66EC40EE66E000E05D0BC0EB8
:101F4000E66EC40EE66E000EE66E75D819EC43F030
:101F500045E96ADA01EBF3FF02EBF4FF21D1E66E0B
:101F6000C2D9B4EC84F047E900091200E7D9CAD914
:101F7000CCEF11F04CDA65EF11F095EC5FF0E55223
:101F800041DA0B01D151D21112000601FA150B01F1
:101F9000D16FD26BD1510008000ED255120000EB68
:101FA000F6FF01EBF7FF02EBF8FF08001200EA6A08
:101FB000000FE96E080EEA221200B9D982EF11F083
:101FC000E66EF0D10601FB150B01D26FD15100086E
:101FD000000ED2551200D9CFE6FFE1CFD9FF120093
:101FE000E66E57EC02F043E9120007DAEF501200F8
:101FF00018EC8BF041E9F3CFE6FFF4CFE6FF1200D7
:102000000901C5250B01D16FD26BD237E66ED2CB59
:10201000E6FF4DEC5FF0E552E5CFEAFFE7CFE9FFE1
:10202000440EE926090EEA22EF50120042E9ABD92C
:102030000B01D151120001EBE6FF02EBE6FF1200AB
:10204000E66EF7D9CCEF11F0030E93D9DBD90B0173
:10205000010ED1191200E66E1EEF12F0000E0601FD
:10206000FA150B01D16F1200E66E03EBE6FF04EBED
:10207000E6FF68EC86F045E9F3CFD1FBF4CFD2FB65
:102080000B01F350F41012000601D26BD36B000168
:10209000050EC86F1200E66EE66AA9EC03F042E98D
:1020A0001200E6680CD9E668C9D900EF8CF0E66E3C
:1020B0007ED9026EF450036E02EBE9FF03EBEAFFF8
:1020C000EF501200CFC8E9FFD0C8EAFFCF2B000EB7
:1020D000D0231200E66EF7EC3DF041E9120001EB6F
:1020E000E9FF02EBEAFFEF50120087D9EFCFE6FFDE
:1020F00059D1FCC0E6FFFDC0E6FFFEC0E6FFFFC011
:10210000E6FFE7EF61F0EA510B01D16FD26BC80E29
:10211000D1191200D60EE66E060EE66E120041E9E7
:10212000016E01EBE6FF120003EBE6FF04EBE6FFB6
:1021300009EC7FF042E9F3CFE6FF1200050EE66EF0
:10214000E66A1200D9CFE9FFDACFEAFFEE2A000EE5
:10215000EE22EE2212000601CA07000ECB5BCA5126
:102160000008000ECB551200E66AE66A200EE66E05
:10217000410EE66ED2EF90F0010EE66EE66ACCC03C
:10218000E6FFE66AE66AE66A1200036EF450046E41
:10219000035004101200CE6FCF6BC96B2CEF12F0FE
:1021A00041E9E7CFD9FF120042E9E7CFD9FF12009A
:1021B0000601F16BF26BF36BF46BF56BF66B1200CF
:1021C0000601030ECD6F5F0ECE6FCF6BC96B120091
:1021D000EED8016EF450026E12000F6ED251106EE6
:1021E000D351116ED451126E1200136ED251146E6F
:1021F000D351156ED451166E1200E66E01EBE6FF58
:1022000032EC17F042E9016E12007AEC44F04BE92F
:1022100014EF12F0FF0E0601EB5D12002B0E080109
:10222000005D12004F0E0801005D12000A0EE66EFE
:10223000E66A120009EC7FF042E9F3CFECF6060102
:102240001200F5CFE6FFAED0400EE66EC70EE66E8A
:10225000000EE66E12000B01D11FD21FD31FD41F38
:10226000D1511200EAC6E6FF73EF11F0E66EDFEC23
:102270003DF041E9120043E9E7CFD9FF1200BD0E5E
:10228000CF5D080ED0591200E66E41EC04F041E932
:1022900012000A0E0601CA6FCB6B1200010E060176
:1022A000EE1500081200E3EC02F042E91200BEDF76
:1022B000E50EE66EC60EE66E000EAFEF0FF0010EF5
:1022C000E66ED9EC8BF042E91200E66A1EEF12F0DE
:1022D000D0C6E6FFD1C6E6FFBDEF0FF0030EE66EF7
:1022E000E66A0AEF12F0000EE66E080EE66E1200C5
:1022F000E66E7EDED8DFB30EE66EC60EE66E000E2C
:10230000F0EF0FF0000EE66EE66A19EF12F00B0E1A
:10231000E66EE66A4D0EE66EC60EE66E000EAFEF96
:102320000FF0EA51EA2B43DE01EBEFFF1200420E01
:10233000E66EC70EE66E000EE66E12003C0EE66E0E
:10234000C60EE66E000EE66E1200EA5130DEEF6A4F
:102350001200F4DED80EE66EC60EE66E000EAFEF8B
:102360000FF0ECDEAD0EE66EC50EE66E000EAFEFC2
:102370000FF0E66EE66AD0C6E6FFD1C6E6FF95EC42
:102380005FF0E5521200FCC0D1FBFDC0D2FBFEC0E5
:10239000D3FBFFC0D4FB1200016EF450026E01505B
:1023A00002101200E1EC8CF041E90009120018EC77
:1023B0008BF041E9F35012000EDE81E91200EFDDEF
:1023C000F5501200FADD056EF450066E0550061049
:1023D0001200E66E77DEE552E750EF6E120029D864
:1023E000C5EF10F028DEC8EC41F016EF10F023DE48
:1023F00009EC7FF042E9F350120000EBE9FF01EB3A
:10240000EAFF1200E5CFD2FBE7CFD1FB1200E66E68
:102410005FEF11F0CEC6E6FFCFC6E6FFBDEF0FF0CF
:10242000E66EE66A68EF11F0F350016EF450026E4A
:10243000120003EC91F045E9F3501200E66AD9EC82
:062440008BF042E91200DE
:0A2446000B01916B926B0801CF6B44
:10245000D06B0001CA6B12000B01506B516B000175
:10246000CA6B12007F0E0601C85D0AE10B01010E66
:10247000516F390EE66ECA0EE66E000E32EF20F096
:10248000F6EC01F02D0EE66ECA0EE66E000E32EC92
:1024900020F014EC02F00B01516F12007F0E0601C8
:1024A000C85D08E10B01516B280EE66ECA0EE66EA0
:1024B000000E13D00B01515107E00B01260ED16F16
:1024C000CA0ED26F000E06D00B01240ED16FCA0EB9
:1024D000D26F000ED36FBCEC1FF032EF20F0C6ECD1
:1024E0001FF081E943E80B0151516FE07F0E0601B7
:1024F000C85D06E19DEC1FF0E3EC02F042E963D019
:102500000B0180054DE1450E0701055D49E0410ED7
:10251000055D46E0610E055D43E0670E055D40E048
:10252000500E055D3DE00551036E060EE66E070E8A
:10253000E66EC5EC20F0A2EC85F044E9F1EC21F068
:10254000016A026AD890025004E6000E015C040E93
:10255000025808E2D5EC21F02AEC22F0012A000E04
:102560000222F0D7C5EC20F069EC21F01EEC22F03D
:10257000C5EC20F02AEC22F01C0EE66ECA0EE66EC8
:10258000000EA1EC21F003EB07F7080EE66E070E34
:10259000E66E72EC20F0C5EC20F08EEC82F046E99D
:1025A0009DEC1FF069EC21F01EEC22F09DEC1FF079
:1025B00093EC20F0E9EC20F072EC20F09DEC1FF0A1
:1025C000FDEC82F044E941EC22F044E9E7CFD9FF89
:1025D0001200C6EC1FF081E945E8E66A010EE66EDE
:1025E000D650E66EE66A6EEC21F0056EE750046E9A
:1025F000D7500426000E0522016A080E015C0CE289
:102600000150EA6A060FE96E000EEA22EF50042636
:10261000000E0522012AF1D7DAEC21F098EC81F0C6
:1026200042E9016A160E015C11E2C5EC21F0D5BF4A
:10263000D66961EC20F00150EA6A520FE96E0B0E88
:10264000EA22E552E750EF6E012AECD70B01686BE6
:10265000090EE66E49EC20F0EAEC22F08AEC21F05B
:10266000CEEC1FF08AEC21F0160EE66EE66A17EC4F
:1026700021F06AEC8FF04AE9110EE66ECA0EE66EA2
:10268000000E32EC20F017EC21F0E3EC02F042E90E
:1026900048EC22F04EEC20F0FDEC82F044E948ECEE
:1026A00022F0080EE66E49EC20F01CEC21F041EC23
:1026B00022F046E9E7CFD9FF1200C6EC1FF084E90B
:1026C00042E86FEC22F019EC42F044E9B5EC22F05C
:1026D0000250020A10E0030A03E0010A19E108D0DF
:1026E000B6EC20F00450EE1802E10550ED1810E0B1
:1026F0000DEC22F00DD0B6EC20F00450EE1802E103
:102700000550ED1805E0AEDE0DEC22F0010E026E74
:10271000025037EF20F03BEC22F044E8020EE66E68
:1027200049EC20F073EC21F0080EE66ECA0EE66E5E
:10273000000E99EC21F022EC20F060C0E6FF61C0B1
:10274000E6FF90EC1FF000016251A4EC21F00001C3
:1027500066510F0A20E0020A18E0090A10E0060A92
:1027600008E0030A1EE1FC0EE66EC90EE66E000EDE
:102770001DD0F40EE66EC90EE66E000E17D0EE0EFA
:10278000E66EC90EE66E000E11D0E50EE66EC90EBD
:10279000E66E000E0BD0DC0EE66EC90EE66E000E85
:1027A00005D0D30EE66EC90EE66E000E73EC22F075
:1027B00000016851040A18E0070A10E0020A08E064
:1027C000010A18E1C90EE66EC90EE66E000E14D0BD
:1027D000C00EE66EC90EE66E000E0ED0B90EE66EA5
:1027E000C90EE66E000E08D0AC0EE66EC90EE66E9F
:1027F000000E02D0AFEC22F073EC22F0B3EC1FF02D
:102800004D0807E179C0E6FF7AC0E6FF76EC22F0DA
:102810000AD079C0E6FF7AC0E6FFCBEC22F076EC76
:1028200022F0CBEC22F090EC1FF000016351A4ECFD
:1028300021F064C0E6FF65C0E6FF90EC1FF00001E8
:102840006951A4EC21F06AC0E6FF6BC0E6FF90EC92
:102850001FF000016751A4EC21F000016651A4ECC7
:1028600021F000016851A4EC21F0BFC0D1FB0B01A5
:10287000D26BD1BFD269DFEC21F0C0C0E6FFC1C08E
:10288000E6FF90EC1FF0C7C0D1FB0B01D26BD1BFAC
:10289000D269DFEC21F04FEC22F0D3EC1FF0DAC06C
:1028A000E6FFDBC0E6FF90EC1FF00001DD350FE234
:1028B0000001DF35DF510001DD1908E60001DE51BE
:1028C0000001DC5D0001DF510001DD5902E3000E73
:1028D00001D0010E000905E0DCC0D1FBDDC0D2FB58
:1028E00004D0DEC0D1FBDFC0D2FBDFEC21F0B3ECC3
:1028F0001FF04D0803E121EC21F002D0D1EC22F0D1
:10290000DFEC21F00001E251A4EC21F0E5C0D1FBA5
:102910000B01D26BD1BFD269DFEC21F0E8C0E6FF3A
:10292000E9C0E6FF90EC1FF0EAC0E6FFEBC0E6FF6F
:1029300090EC1FF0EDC0E6FFEEC0E6FF90EC1FF05C
:10294000DCC0E6FFDDC0E6FF90EC1FF0DEC0E6FF76
:10295000DFC0E6FF90EC1FF0B3EC1FF04D0807E17D
:10296000E3C0D1FBE4C0D2FB99EC22F006D0E3C077
:10297000E6FFE4C0E6FFB7EC21F0DFEC21F06CC02D
:10298000D1FB0B01D26BD1BFD269DFEC21F0BBECE4
:1029900020F06DC0E6FF6EC0E6FFD3EC1FF0BBEC8D
:1029A00020F06FC0E6FF70C0E6FFD3EC1FF000011F
:1029B000D951A4EC21F0810EE66E0B0E1BEC20F039
:1029C00045E9E7CFD9FF12003BEC22F042E8EDECFD
:1029D00020F0A50EE66EC90EE66E000EF5EC22F0B4
:1029E00027EC21F015EC22F0FCEC22F027EC21F092
:1029F000A2CBE6FFA3CBE6FF93EC1FF0A4CBE6FF50
:102A0000A5CBE6FF93EC1FF00001C251A8EC21F02A
:102A1000C5C0D1FB0B01D26BD1BFD26905EC22F04E
:102A200000017751A8EC21F04D0E00010F5D03E18C
:102A30002CEC21F002D0D7EC22F005EC22F07DC086
:102A4000E6FFFCEC22F01EEC44F046E98FEC21F0AE
:102A5000BBEC20F07EC0D1FB7FC0D2FB99EC22F012
:102A6000D2AF02D0D369D4698DEC22F0DEEC1FF036
:102A700080C0E6FF81C0E6FF82C0E6FF83C0E6FFBC
:102A8000B6EC1FF084C0E6FF85C0E6FF86C0E6FF17
:102A900087C0E6FFB6EC1FF0830EE66E0B0E1BEC54
:102AA00020F037EF20F03BEC22F047E89E0EE66E78
:102AB000C90EE66E000EF5EC22F032EC21F0026A4F
:102AC000040E025C57E27FEC20F0D23547E2D15190
:102AD0000008000ED25542E2560EE66E0E0EE66E6D
:102AE0008D0EE66E3E0EE66E0250EA6AB50FE96E96
:102AF000000EEA22EFCFE6FFE0EC5DF072EC60F052
:102B0000C1EC5EF0E552E5CFD4FBE5CFD3FBE5CFDA
:102B1000D2FBE7CFD1FB0B01D151056ED251066E2E
:102B2000D351076ED451086EBBEC20F009EC20F0B5
:102B3000C0EC21F035EC21F07AEC44F04BE9E2EC0A
:102B400021F07FEC20F0280ED15F000ED25BBCECB0
:102B50001FF0A2EC1FF0AFEC22F005D0990EE66E4C
:102B6000C90EE66E000EE66EBBEC21F032EC21F0F1
:102B7000022AA6D7C6C0D1FB0B01D26BD1BFD26946
:102B8000BCEC1FF035EC21F0F8EC22F0E2EC21F087
:102B9000850EE66E0B0E1BEC20F048E9E7CFD9FF5F
:102BA00012003BEC22F043E8010E046E020E046EAC
:102BB000CFEC20F0920EE66EC90EE66E000EA5EC8C
:102BC00022F08FEC21F00F0EF66E000EF76E000E65
:102BD00012EC20F0100EF66E000EF76E000E12ECE6
:102BE00020F077EC20F0DDEC22F000011051111103
:102BF000121104E04FEC21F0CBEC1FF0045057EC25
:102C000022F0E66EA1EC22F0860EE66EC90EE66EAC
:102C1000000EE66E7CEC22F08AEC21F059EC43F0D9
:102C200048E98FEC21F0930EE66E000EDAEC1FF00F
:102C30000001CB51A8EC21F00B01CD51A8EC21F003
:102C4000950EE66E0B0EDAEC1FF0CE0EE66E000E61
:102C5000DAEC1FF0870EE66E0B0E1BEC20F044E959
:102C6000E7CFD9FF12003BEC22F046E800018C517F
:102C70008D118E118F1105E1046A056A066A076AD3
:102C800020D08C0EE96E000EEA6EEE500001885DD9
:102C90000B01D16FEE50000189590B01D26FEE503C
:102CA00000018A590B01D36FEE5000018B590B01C3
:102CB000D46FD151046ED251056ED351066ED451EA
:102CC000076E00017151E66EE66A7F0EE66EC90E70
:102CD000E66E000EA5EC22F08FEC21F0000172519F
:102CE000A8EC21F000017651A8EC21F0A5C0E6FF88
:102CF000A6C0E6FF93EC1FF0A7C0E6FFA8C0E6FF62
:102D000093EC1FF0A9C0E6FFAAC0E6FF93EC1FF00A
:102D10004D0E00010F5D03E12CEC21F002D0D7EC49
:102D200022F005EC22F04D0E00010F5D09E1BBC061
:102D3000D1FBBCC0D2FBBDC0D3FBBEC0D4FB0AD00C
:102D4000BBC0E6FFBCC0E6FFBDC0E6FFBEC0E6FFFD
:102D5000A7EC1FF08DEC22F0B6EC1FF000017751CC
:102D6000A8EC21F004EBE6FF09EC20F007EBE6FF0E
:102D7000B6EC1FF091C0E6FF92C0E6FF93EC1FF0A7
:102D800000017351A8EC21F0C4C0D1FB0B01D26B40
:102D9000D1BFD26905EC22F0C3C0D1FB0B01D26BCD
:102DA000D1BFD26905EC22F0BBEC20F0CCC0E6FF2D
:102DB000E66AE66AE66ADEEC1FF000017451A8ECF0
:102DC00021F0BBEC20F0CDC0E6FFE66AE66AE66AD9
:102DD000DEEC1FF000017551A8EC21F0ABC0E6FF5E
:102DE000ACC0E6FF93EC1FF0890EE66E0B0E1BECF9
:102DF00020F047E9E7CFD9FF12003BEC22F042E890
:102E0000780EE66EC90EE66E000EA1EC21F08FEC96
:102E100021F0000113511411151115E013C0F6FF34
:102E200014C0F7FF15C0F8FF0800F5500CE013C000
:102E3000E6FF14C0E6FF15C0E6FFCBEC1FF087EC01
:102E400021F0CBEC1FF0680EE66EC90EE66E000EA8
:102E5000E66ECBEC1FF08F0EE66E0B0E1BEC20F037
:102E600037EF20F090EC22F00A0E0024E66E6FECB3
:102E70008AF041E90701C85152E0C80EE66E070E1C
:102E8000E66E610EE66EC90EE66E000EF5EC22F0FF
:102E90006BEC22F0E2EC21F073EC21F0A2EC1FF0DD
:102EA00000017751E66EE66AA2EC1FF0A2CBE6FFC6
:102EB000A3CBE6FFA2EC1FF0A4CBE6FFA5CBE6FF79
:102EC000A2EC1FF00001C251E66EE66AA2EC1FF010
:102ED000C5C0D1FB0B01D26BD1BFD269BCEC1FF0D6
:102EE000A2EC1FF0EDEC20F03BEC20F015EC22F012
:102EF0003BEC20F0000405E10B018B0ED16F0B0EB3
:102F000004D00B018D0ED16F0B0ED26FD1CBE6FF2B
:102F1000E66E01EBE6FF5DEC13F043E9016E015054
:102F200037EF20F0C6EC1FF083E949E8010E0B6E85
:102F3000020E0B6E0050011001E12DD180EB03F069
:102F400081EB04F05BEC20F008E05BEC20F0200863
:102F500004E0032A000E0422F5D75BEC20F02008E1
:102F600001E019D1F6EC20F09CEC21F017EC21F0F7
:102F70006CEC85F044E9000901E10DD1090EA0ECEB
:102F800020F0FAEC21F09CEC21F0CEEC1FF09CEC50
:102F900021F06AEC8FF04AE99DEC1FF04EEC20F036
:102FA0008EEC82F046E99DEC1FF0BBEC21F06CEC5E
:102FB00085F044E9000901E0EED09CEC21F09DECA5
:102FC0001FF0A2EC85F044E917EC21F0ECEC21F0C5
:102FD000FAEC21F06FEC22F06AEC8FF04AE94EEC4B
:102FE00020F0A9EC20F094EC8EF048E9096A0A6A16
:102FF000D8900A5004E6000E095C040E0A580AE252
:10300000D5EC21F0A9EC20F0E9EC20F0092A000E23
:103010000A22EED74EEC20F093EC20F094EC8EF0E8
:1030200048E9096A0A6AD8900A5004E6000E095C69
:10303000040E0A580AE2D5EC21F093EC20F0E9ECFA
:1030400020F0092A000E0A22EED70B01010E506F64
:103050000A0EA0EC20F005EBE9FF06EBEAFFEF50CB
:10306000500843E10B0180511FE1096A0A6A160EFC
:10307000D8900ABE03D0095C000E0A5813E2C5ECD2
:1030800021F0D5BFD66961EC20F0690E0924E96E04
:103090000B0E0A20EA6EE552E750EF6E092A000E89
:1030A0000A22E5D70B017F6B806B590EE66EC90EC5
:1030B000E66E000EA1EC21F07DEC21F0ECEC21F0AD
:1030C000B2EC20F00B01010E806FA0EC20F064EC5C
:1030D00021F0E1EC22F07DEC21F0CEEC1FF07DEC54
:1030E00021F06AEC8FF04AE902D00B01806B0B01F2
:1030F000CFAF4FD0CF9FCFEC20F0370EE66EC90E8A
:10310000E66E000EA5EC22F0E7EC21F00F0EF66E55
:10311000000EF76E000EACEC21F0C1EC1FF0100EAB
:10312000F66E000EF76E000EACEC21F0C1EC1FF055
:1031300077EC20F0C0EC21F03AEC21F000011051C6
:103140001111121108E04FEC21F0C0EC21F0BAECA3
:1031500022F0E7EC21F00B5057EC22F0C1EC1FF00D
:103160000B01CE5108EC22F00B01CF51E66EE66A5E
:1031700087EC21F0C0EC21F0F0EC43F047E9E7ECFC
:1031800021F00B01D05108EC22F005EC21F0B2EC5B
:1031900020F024EC7DF04AE9E7CFD9FF120090EC53
:1031A00022F00B0150511EE1070EE66EE66A2F0E6B
:1031B000E66EC90EE66E000EE66E9CEC21F0B4ECF5
:1031C00084F047E9000901E0CDD0070E0B0100248F
:1031D0005FEC22F0A7DE42E90601060ED06F0E0E6C
:1031E000D16FC0D09DEC1FF09CEC21F03DEC21F0A4
:1031F0000B01CFBF03D00B01410ED06FBBEC21F010
:103200009DEC1FF0A9EC20F0E9EC20F0050EE66E35
:10321000E66A290EE66EC90EE66E000EF5EC22F0A7
:10322000B4EC84F047E9000905E0400EE66E41EC9D
:1032300004F08ED0050E006E070E016EB6EC20F085
:10324000EF50450838E10028E96E000E0120EA6ED3
:10325000EF504D0830E1020E0026000E0122010E53
:10326000E66E060EE66E0EEC20F03DEC21F0F1EC81
:1032700021F0036A046AD890045004E6000E035C4F
:10328000040E045808E2D5EC21F02AEC22F0032ABF
:10329000000E0422F0D7BBEC21F0010EE66E060E04
:1032A000E66E2AEC22F0B6EC20F0EFCF00F6000E2E
:1032B000006E060E016E0B01CFBF03D00B01420E54
:1032C000D06FB6EC20F0EF50430A44E02B0A37E011
:1032D000320A0FE01B0A46E10B01515143E1220E75
:1032E000E66EC90EE66E000EA1EC21F0B2EC20F005
:1032F00039D00EEC20F0DAEC20F0036EF450046EBE
:103300000001CA51F36E043417E20350F35C000E5F
:10331000045412E20B01816B826B896B8A6B836BA5
:10332000846B856B866B876B886B8F6B906BBBEC4C
:1033300020F0A9EC03F042E903EBCAF013D00EEC45
:1033400020F009EC7FF042E9F3CFE6FF4BEC7DF093
:1033500041E908D00EEC20F007D842E90B015151A9
:1033600001E1C9D937EF20F090EC22F080EB03F0B7
:1033700081EB04F05BEC20F008E05BEC20F02C0823
:1033800004E0032A000E0422F5D75BEC20F02C08A1
:1033900002E1F6EC20F09CEC21F009EC7FF042E930
:1033A000F3CF91FBF4CF92FB03EB93FB04EB94FB85
:1033B00037EF20F0C6EC1FF081E945E80B01CFBFE5
:1033C00003D00B01430ED06F310E0B01911901E1B7
:1033D000925101E175D1290E911901E1925101E15A
:1033E00060D1280E911901E1925101E137D1070E08
:1033F000911901E1925101E1D7D0060E911901E135
:10340000925101E1CED0050E911901E1925101E1F5
:10341000BCD0040E911901E1925101E180D0030E5C
:10342000911901E1925159E0020E911901E1925175
:1034300022E0010E911901E1925102E0000E57D1F4
:10344000016A100E015C01E351D10150E66EE66A9B
:10345000170EE66EC90EE66E000E99EC21F0100E06
:10346000A4EC21F056EC21F0EF50A4EC21F06FEC2D
:1034700012F0012AE6D782EC21F0B3EC1FF006E04F
:103480003EEC22F003E09DEC22F0F7D73EEC22F078
:1034900001E001D183EC22F072E2100E015C6FE2D8
:1034A0008AEC21F0DAEC20F0E66E56EC21F0E552E1
:1034B000E750EF6E080E015C09E38AEC21F0080E7C
:1034C000015C180FE66E2DEC8BF043E90F0E015CEA
:1034D00001E006D1D9EC6AF003D1016A200E015C4B
:1034E00001E304D101EBE6FF49EC20F0090E015C99
:1034F00003E194EC22F0EF6A0150E66EE66A0C0EEE
:10350000E66EC90EE66E000E99EC21F0200EA4ECDA
:1035100021F022EC20F06FEC12F0012ADFD782ECD0
:1035200021F0B3EC1FF006E03EEC22F003E09DEC4E
:1035300022F0F7D73EEC22F001E0ADD083EC22F090
:103540001EE2180E015C1BE20150010803E3B3EC1C
:103550001FF015E08AEC21F001EBE6FF2DEC8BF07B
:1035600043E90BEC21F094EC21F0020E015C04E045
:103570000E0E015C01E0B8D0D9EC6AF0B5D0040EB3
:10358000E66E230EE66E010EADD00BEC21F094EC4E
:1035900021F06FEC12F0040EE66E41EC04F041E90C
:1035A000A5D05AEC1FF0A0D02DEC22F0C5EC20F0F5
:1035B0003AEC43F044E90801000ECF6F080ED06FDB
:1035C000000EE66EE66AA6EC00F042E9C5EC20F0DB
:1035D000D60EE66E060EE66EFEEC50F044E9016E85
:1035E000CFC8E9FFD0C8EAFFEF6A0801CF6BD06B04
:1035F000C4EC22F099EC21F0010ED8800154A4EC27
:1036000021F0015071E053EC20F02C0EEF6E000E13
:10361000026E080E036EB3EC1FF01AE0B3EC1FF05D
:103620000A0804E153EC20F00D0E0ED03EEC22F01F
:1036300004E153EC20F03B0E07D0B3EC1FF0E66E34
:1036400053EC20F0E552E750EF6E9DEC22F0E3D70B
:1036500004EBE9FF05EBEAFFEF6A46D082EC21F0CC
:10366000B3EC1FF006E03EEC22F003E09DEC22F00C
:10367000F7D73EEC22F00DE116EC20F061EC49F0BA
:1036800042E91CEC21F0260EE66ECA0EE66E000E34
:103690001ED032EC12F0D80EE66E220EE66E010E4F
:1036A00021D0000EE66EC90EE66E000E32EC20F060
:1036B00042EC21F0FA0EE66EC80EE66E000E07D060
:1036C00042EC21F0F80EE66EC80EE66E000E32EC0B
:1036D00020F0050EE66EF7EC3DF041E932EC12F019
:1036E0000BEC21F094EC21F06FEC12F0010E46E9A6
:1036F000E7CFD9FF12000B01CFBF03D00B01440E5F
:10370000D06F280E0B01D89092BF03D0915D000EB0
:10371000925907E3923507E291513108000E925514
:1037200002E232EC12F000013751381139110FE08A
:103730002DEC22F0CAEC20F0010EE66E39C0FBFF42
:1037400038C0FAFF3751140045E900090CE132DEB8
:10375000000909E1730EE66E230EE66E010E94EC8D
:1037600021F06FEC12F04EEC12F00B01916B926BAA
:1037700093CBE9FF94CBEAFFEF6A1200C6EC1FF08F
:1037800085E90B0150512FE051512DE1800E0B01C5
:10379000CC1529E10B01CFBF03D00B01450ED06F33
:1037A00032EC12F0A8EC22F0E50EE66EC80EE66EE2
:1037B000000E88EC22F08AEC21F0ECEC21F0DC0E1B
:1037C000E66EC80EE66E000E88EC22F09B0E00241A
:1037D000E96E000E0120EA6EEF6A9CEC21F0ECEC41
:1037E00021F032EC22F041E9E7CFD9FF1200CEDB25
:1037F00084E944E8066A076A0B01505101E176D07A
:103800000150021073E0005071E00050E66EE66A6D
:10381000220EE66E72EC20F096EC84F045E9F3504F
:10382000066EF450076E065007102FE0062A000EB1
:1038300007220B015DEC21F0D151005E86EB01F017
:1038400087EB02F0DFEC20F0EF501CE0DFEC20F023
:10385000EF50220817E05DEC21F00050D890D2BF65
:1038600003D0D15D000ED2590DE2DFEC20F0EF5015
:103870002C0804E1DFEC20F02E0EEF6E062A000E7D
:103880000722E0D7DFEC20F0EF6A290EE66EE66A49
:103890003C0EE66ECA0EE66E000E99EC21F0065064
:1038A00007100DE072EC20F0D80EE66EC80EE66E42
:1038B000000EE66EDAEC21F06BEC22F007D0C10EC0
:1038C000E66EC80EE66E000E9CEC20F0B5EC22F021
:1038D0000B01515104E005EC21F0046A056AB2ECD9
:1038E00020F00450051002E105EC21F045E9E7CF96
:1038F000D9FF12004BDB83E94CE800017B51036EDA
:103900007C51046E00017951056E7A51066E0001FA
:10391000BB51076EBC51086EBD51096EBE510A6E97
:10392000BD0E0B6EC80E0C6E000E0D6E4B0E000120
:103930000F5D23E1BBEC21F0B7EC21F00B01D1517D
:10394000036ED251046E65DBB7EC21F00B01D1514F
:10395000056ED251066EFFEC20F0F9DA0B01D15161
:10396000076ED251086ED351096ED4510A6EB90E4A
:103970000B6EC80E0C6E000E0D6E0001E53532E2C6
:10398000A9C0E6FFAAC0E6FFAE0EE66EC80EE66E60
:10399000000ECCDAE8C0E6FFE9C0E6FFAB0EE66E4B
:1039A000C80EE66E000EC2DAE5C0D1FB0B01D26B89
:1039B000D1BFD269E1DAA70EE66EC80EE66E000E40
:1039C000B5DAEAC0E6FFEBC0E6FF9E0EE66EC80E73
:1039D000E66E000EABDA910EE66EC80EE66E000ED5
:1039E000E66EA8DA000171A5B5D0010E0E6E0001D9
:1039F0006851040A18E0070A10E0020A08E0010A08
:103A000019E1850EE66EC80EE66E000E11D07A0E34
:103A1000E66EC80EE66E000E0BD0710EE66EC80E96
:103A2000E66E000E05D0620EE66EC80EE66E000E63
:103A3000E66E80DA000166510F0A20E0020A18E003
:103A4000090A10E0060A08E0030A20E1590EE66EB2
:103A5000C80EE66E000E17D04D0EE66EC80EE66E6E
:103A6000000E11D0410EE66EC80EE66E000E13D0A9
:103A7000370EE66EC80EE66E000E05D0250EE66E19
:103A8000C80EE66E000EF2EC22F008D0160EE66EBE
:103A9000C80EE66E000EF2EC22F00E6A0E5061E0E7
:103AA00060C0E6FF61C0E6FFBEEC22F03FDA000135
:103AB0006251E66EE66A100EE66EC80EE66E000E05
:103AC00035DA0E0EE66EC80EE66E000EF2EC22F04F
:103AD0000001DB350BE2DAC0E6FFDBC0E6FF050ED6
:103AE000E66EC80EE66E000E67EC22F00001E251B1
:103AF000000811E2E251E66EE66ABEEC22F016DA48
:103B0000DEC0E6FFDFC0E6FFFB0EE66EC70EE66E28
:103B1000000E67EC22F00001E0510008000EE155B4
:103B200020E24B0E00010F5D03E1D1EC22F001D049
:103B300088DB22DABEEC22F0D2EC21F0DCC0E6FF1A
:103B4000DDC0E6FFF80EE66EC70EE66E000EEED99B
:103B500068DB05D0EB0EE66EC70EE66E000EE66E75
:103B6000E9D9C1DBE30EE66EC70EE66E000EFDEC92
:103B700021F00550061008E04CDAD10EE66EC70EB3
:103B8000E66E000ED2EC21F00350041008E0F3DBE7
:103B9000C20EE66EC70EE66E000ED2EC21F00750A4
:103BA000081009100A100AE0E6DA29DBBA0EE66E00
:103BB000C70EE66E000EE3DAE5EC22F00001D75105
:103BC000D8110AE04FEC22F0E66AE66AB20EE66E21
:103BD000C70EE66E000ED3DA0001D9510AE0D951C2
:103BE000E66EE66AAA0EE66EC70EE66E000EFDEC05
:103BF00021F000EBF3FF01EBF4FF4DE9E7CFD9FF34
:103C00001200C4D985E95BE800017951056E7A514B
:103C1000066E076A086A096A0A6A0001D7510B6EC4
:103C2000D8510C6E000160510D6E61510E6E000195
:103C300063510F6E106A00019151116E9251126E14
:103C400000016851136E146A156A166A000140512A
:103C50004111421109E1980EE66EC70EE66E000EA4
:103C6000E66EFFEC22F022D10050011001E17DD080
:103C700063DB2FDB1B6EF4501C6E5EDBCAEC86F040
:103C800042E91C3469E21B500008000E1C5464E237
:103C90000B01DCD9EF501F6ED9D9EF6A1C344AE210
:103CA0001B500108000E1C5445E246DB83DA1D6EF2
:103CB000F4501E6E1F50440A38E0070A2AE0020A38
:103CC00023E0170A1CE0010A15E0720A0EE0600A00
:103CD00007E0160A3DE19DEB05F09EEB06F038D0BB
:103CE0009DEB07F09EEB08F033D09DEB09F09EEBC7
:103CF0000AF02ED09DEB15F09EEB16F029D09DEB2F
:103D00000DF09EEB0EF024D09DEB0FF09EEB10F02B
:103D10001FD0640EE66EE66A1DEBE6FF1EEBE6FFC3
:103D2000DDDA0C6EE7500B6E13D09DEB11F09EEBBD
:103D300012F00ED01F50500A08E0020A04E0010AF7
:103D400007E1136A04D0030E01D0040E136E146A47
:103D50000B017CD91FEBEFFFEFDAEDEC4AF042E903
:103D6000F350006EF450016E7FD70E3418E20D5000
:103D70000008000E0E5413E2103411E20F50000838
:103D8000000E10540CE20FEBE6FF10EBE6FF0DEB1C
:103D9000E6FF0EEBE6FFA2DA166EE750156ED8903E
:103DA000165004E6E80E155C030E165806E27F0E68
:103DB000E66EC70EE66E000E63D0D950170FE66EA2
:103DC000DACFE6FF11EBE6FFFFD909EBE6FF0AEBDE
:103DD000E6FFD6DA1ED915EBE6FF16EBE6FF13EB8E
:103DE000E6FF42C0FBFF41C0FAFF00014051140052
:103DF0004EE9F350196EF4501A6E0BD98FD917EBA8
:103E0000E6FF18EBE6FF7A0EE66EC70EE66E000ED2
:103E1000E66E97DB6F0EE66EC70EE66E000EE66E80
:103E2000BAD81A3422E233DA4AEC5FF077D9300E8E
:103E3000E66E020EE66EE66A2ADA4DEC5FF0E552B7
:103E4000E5CFD2FBE7CFD1FB74DBD2AF02D0D36991
:103E5000D46963DB6D0EE66EC70EE66E000EE66E8D
:103E600059DA3EEC44F04CE91CD0FD0E19180BE178
:103E7000FF0E1A1808E15E0EE66EC70EE66E000E23
:103E8000E66EBDDB0ED019EBE6FF1AEBE6FF560E31
:103E9000E66EC70EE66E000EE66E3CDA6DEC43F0A1
:103EA00047E93DDA02EBF3FF03EBF4FF5CE9E7CF10
:103EB000D9FF12006BD881E942E84ADBF350BEDA41
:103EC00019DD42E9D4D0D7DA42E80B01CCB70BD0E8
:103ED00032EC12F03DDB23DA00EBE6FF1BDA45ECB7
:103EE0000FF043E9BFDAC3D051D887E942E832EC9A
:103EF00012F0950EE66E0B0EE66E4E0EE66EC70ED7
:103F0000E66E000E72DBB6D955DAE66AE66ABAD812
:103F100000EBE6FFE7D803EBE6FFB4D8A3DAA7D0BF
:103F20005EDB66DB90D2F3D9A1EF22F0E66E04DA15
:103F30005FDB8BD201DA1EDB88D2000EE66E070E45
:103F4000E66E1200E4D917DA53DBE2EF21F0B3ECAE
:103F50003EF044E9FCC0D1FBFDC0D2FBFEC0D3FB68
:103F6000FFC0D4FB1200E0DAEF50120045DB98EC02
:103F700043F049E98FEF21F0D1CBE6FFD2CBE6FF4A
:103F80001200E66EFDD934DBE7EF21F0D9CFE6FF72
:103F9000E1CFD9FF120033DB8FEF21F0DCEC85F0AD
:103FA00042E936EF22F0E66AE66A19DB7AEC44F081
:103FB0004BE949D2E66EABD9DDEF22F01DDB7AEC9E
:103FC00044F04BE98FEF21F0000EE66E030EE66E33
:103FD000FC0EE66E040EE66E1200D3CBE6FF9FECFD
:103FE00081F0E552E7CFD3FBE552E7CFD2FBE552B4
:103FF000E7CFD1FB3BDA4DEC5FF0E552E5CFD5FBE7
:10400000E7CFD4FB0B01D66B1200F2DA2FDABAEF4E
:1040100022F005EBE6FF06EBE6FF12000B0100289D
:104020005FEF22F099D9E66EA1EF22F07DDA85DA12
:10403000EF6A2DEF22F0E66E00EBE6FF5DEC13F089
:1040400043E9120067D9CBDA46DAFDD11B04D16F00
:10405000000E1C58D26FD1510024E96ED2510120BC
:10406000EA6E1200E66E57EC02F043E9120043E9F3
:10407000E7CFD9FF12004BD97ED96DEC45F049E965
:10408000E2EF21F044D97CD998EC43F049E9E7EF1D
:1040900021F018EC8BF041E98FEF21F0100EE66E65
:1040A000E66AEAEF22F004EBE9FF05EBEAFF042AF7
:1040B000000E0522120003EBE9FF04EBEAFFEF50CC
:1040C0001200D151D425F36ED251D521F46ED351C3
:1040D000D621F86EF4CFF7FFF3CFF6FF0800F550C6
:1040E000E66E120001EBE6FF02EBE6FF12000E0E99
:1040F000E66E18EC8BF041E9B9D97CEF22F0EA6A60
:104100000234FE0BE96EEA36AD0EE926000EEA2215
:10411000EECFD1FBEFCFD2FB0B011200E66AE66ACD
:10412000E66AA1EF22F0000EE66E010EE66EF80ED2
:10413000E66E040EE66E1200E66E3CD9BAEF22F08F
:10414000E66E18EC8BF041E9F350056EF450066E04
:104150001200000EE66E020EE66EFA0EE66E040E19
:10416000E66E120032EC12F032EF22F000EBE9FFC3
:1041700001EBEAFF1200010EE66EE66A1200E66E3F
:10418000DBD8DEEC44F04BE960D1000EE66E060EA3
:10419000E66E120091CBE6FF92CBE6FF12000E0E08
:1041A000F66E000EF76E000EF86E0800F550E66E23
:1041B000E66A120009EC7FF042E9F350120006EBC8
:1041C000E9FF07EBEAFF12000BEBE6FF0CEBE6FF63
:1041D000120001EC8FF048E912009ACBE6FF9BCB6E
:1041E000E6FF9CCBE6FF9DCBE6FF120003EBE9FF69
:1041F00004EBEAFF032A000E0422EF6A1200C0D883
:1042000009EBE6FF0AEBE6FF1200140EE66EF7EC90
:104210003DF041E91200D50EE66E220EE66E010E6B
:104220001200FF0EE66EC70EE66E000E1200520E72
:10423000E66E0B0EE66E12006DD8E3EC02F042E97A
:104240001200E0C0D1FBE1C0D2FB99EF22F06DEC8F
:1042500045F049E98FEF21F0B9C0D1FBBAC0D2FBDC
:1042600099EF22F087D9E2EF21F0E66AE66AE66A82
:10427000BBEF21F030D9E7EF21F090EC83F044E977
:10428000E2EF21F0EAD8E3EC02F042E912003C0E42
:10429000E66EE66A19EBE6FF1AEBE6FF120010C0C5
:1042A000E6FF11C0E6FF12C0E6FF12000150EA6A05
:1042B000BE0FE96E0B0EEA2212000150065CD16FB0
:1042C00002500758D26F1200E80EE66E040EE66E3A
:1042D0001200DCEC85F042E9F350120002EC61F0D0
:1042E000E552E550120000017851E66EE66A1200D0
:1042F000D3CBE6FFD4CBE6FF1200690EE66E0B0EC1
:10430000E66E12009351026E9451036E120027D98B
:10431000E66E120002EBE6FF03EBE6FF1200F3503D
:10432000026EF450036E1200E66E2ED95ED905EFD0
:1043300020F00BD9B5EF22F000EBE6FF01EBE6FF32
:10434000120053D9BAEF22F0E66EE66A90EF1FF042
:10435000E66EE66A93EF1FF0F86E0800F550E66E21
:10436000E66A900EE66EC90EE66E000E1200E66A70
:10437000E66AA7EF1FF003EBE6FF04EBE6FF12008F
:1043800007EBE6FF08EBE6FF12000B01140ED16FFE
:10439000240ED26F010ED36F400EE66EE66AECDD9E
:1043A000EDEF1FF0C3DDE5EF22F00701006BE3DE68
:1043B0009DEF1FF004EBE6FF05EBE6FF1200DCDDEE
:1043C00090EF1FF0F350036EF450046E1200F350A0
:1043D000076EF450086E1200B0DD18EC85F044E969
:1043E0001200100EE66EE66A6FDFEEDD94EC8EF0E2
:1043F00048E91200EFD8E1EF22F098DDE10EE66E19
:10440000C70EE66E000EF2EF22F0B6DD93EF1FF05E
:10441000E66EE66AA4D8C1EF1FF06FEC12F0A6DEDC
:1044200004EBEEFF05EBEDFF12009ECBE6FF9FCB0A
:10443000E6FFA0CBE6FFA1CBE6FF1200016EF45031
:10444000026E72EF20F0B5EF22F0F350006EF450E0
:10445000016E1200B9DDE9EF20F093CBE6FF94CBBB
:10446000E6FF12006FEC12F04EEF12F0F3CFE6FF12
:10447000F4CFE6FF12008ADD82E9120074DD2C0819
:104480001200190EE66ECA0EE66E000E32EF20F034
:104490000F0EE66ECA0EE66E000E32EF20F0020E30
:1044A000E66EE66AD7C0E6FFD8C0E6FF1200E66E09
:1044B000E66A8B0EE66EC90EE66E000E1200D16F34
:1044C000000E0120D26FD1CBE6FFE66E12002EDD8A
:1044D000A8DEF2EF22F04DEC43F047E912002DDDAB
:1044E0005DDD9DEF1FF028DEB5EF22F019DD7BC00A
:1044F000E6FF7CC0E6FF12008E0EE66EC90EE66E89
:10450000000EE66E120092DD55DE016ED8901200AC
:104510006CD83CEC85F045E912002EDD78EF21F0F7
:1045200035DD83E942E8120002EBE9FF03EBEAFF25
:1045300012000B01D36BD46B1200022A000E03226F
:104540001200E8DE55D88FEF21F04FD8F8EF22F0B7
:10455000F00EE66EC80EE66E000EA1EF21F0060E1C
:10456000E66ECA0EE66E000E1200F350046EF450B2
:10457000056E120019EC43F045E91200130EE66EC9
:10458000C80EE66E000E120005DECE0EE66E220E9E
:10459000E66E010E1200EBDEFCC0E6FFFDC0E6FF9A
:1045A0001200E0C0E6FFE1C0E6FFB7EF21F0B9C0BE
:1045B000E6FFBAC0E6FFB7EF21F0ACDE8CDF8FEF8D
:1045C00021F027DDEBDC09EF20F0FEDD0DEBE6FF4F
:1045D0009AEF1FF0D80EE66E040EE66E120097DE1C
:1045E000DAEF21F0E66E9AEF1FF0E66E9DEF1FF016
:1045F0006DEC43F047E912008ADE8AEF21F08ADE93
:04460000BAEF22F0FB
:0C46040015EC2FF081E947E8000102519D
:1046100001E032D3010E031901E02ED3000106514F
:10462000A60A01E122D3030A01E1F6D2010A01E15F
:10463000E9D2070A01E1D1D23D0A01E1A1D2080A7B
:1046400001E128D2030A01E1DCD11A0A01E1B9D162
:104650001C0A01E14CD11A0A01E105D1010A01E16C
:10466000ECD00D0A01E1B5D0010A01E191D0070AB1
:104670006EE0010A62E0030A3FE0010A17E0860AE1
:1046800001E00DD31B0E075D03E10AC0BFF00AD0A5
:104690001A0E075D01E003D30A51F3500B25000108
:1046A000C06FC16B0001010EC76FF9D207C078F06F
:1046B000C6EC2EF00001796F000E0B010121000104
:1046C0007A6FB4EC2FF000017B6F000E0B0101211B
:1046D00000017C6F000179517008170E7A5502E2D3
:1046E000796B7A6B00017B517008170E7C5501E3E2
:1046F000D6D27B6B7C6BD3D2EFEC2EF004E00B01B7
:1047000069EC2FF0FDE189EC2EF004E00B0170EC78
:104710002FF0FDE192EC2EF004E00B018AEC2FF07B
:10472000FDE10B0122EC2FF000CB88F001CB89F0EA
:1047300002CB8AF003CB8BF0B2D207C091F000011C
:10474000926B91BF92690001780EC36FA8D2EFEC13
:104750002EF004E00B0169EC2FF0FDE189EC2EF066
:1047600004E00B0170EC2FF0FDE192EC2EF004E080
:104770000B018AEC2FF0FDE10B0122EC2FF000CBB6
:104780009AFB01CB9BFB02CB9CFB03CB9DFB87D20F
:10479000EFEC2EF004E00B0169EC2FF0FDE189EC69
:1047A0002EF004E00B0170EC2FF0FDE192EC2EF006
:1047B00004E00B018AEC2FF0FDE10B0122EC2FF05D
:1047C00000CB9EFB01CB9FFB02CBA0FB03CBA1FB4D
:1047D00066D207C0C2F00001C2512CE0C6EC2EF038
:1047E0000B01A26F000E0B0101210B01A36F680EDC
:1047F000A21905E1010EA31902E1A26BA36BF00E51
:1048000000010B1504E00B01A46BA56B0FD00BC0CE
:1048100001FB0B01006B00010A510B0100250B018C
:10482000A46F000E0B0101210B01A56F0001780E92
:10483000C56F35D20001C56B32D200016351000152
:104840000C5D03E0020E83EC2EF007C062F00CC09A
:1048500063F0C6EC2EF00001646F000E0B01012125
:104860000001656F1CD24D0E00010F5D03E107C012
:1048700077F033D063EC30F0490EE66E060EE66E4C
:10488000E66AE66A07C0E6FFE66AA9EC30F0E552A0
:10489000E5CF07FBE5CF06FBE5CF05FBE7CF04FB44
:1048A000F40E0B010427010E0523000E0623072337
:1048B00004CBE6FF05CBE6FF06CBE6FF07CBE6FF22
:1048C0002CEC60F0E552E5CF03FBE5CF02FBE5CF32
:1048D00001FBE7CF00FB00CB77F0C6EC2EF0000128
:1048E000606F000E0B0101210001616FD8D10751EB
:1048F000016EC6EC2EF0026E000E0121036E0DC09B
:1049000000FB016B026B036B180E1F0B08E00B0121
:10491000D8900037013702370337E806F9E10CC0B9
:1049200004FB0B01056B066B076B100E1F0B04E0FD
:104930000B0169EC2FF0FDE16EEC30F00BC008FBD1
:10494000096B0A6B0B6B080E1F0B04E00B0170EC7C
:104950002FF0FDE178EC30F00AC00CFB0D6B0E6B14
:104960000F6B22EC2FF00051046E0151056E0251C5
:10497000066E0351076E021C01E1031C01E18FD199
:10498000140E015C0BE1190E021808E1035006E158
:10499000F0EC2FF07DEC03F046E902D001A00BD043
:1049A00004EBE6FF05EBE6FF1DEC30F002EBE6FF63
:1049B00003EBE6FF02D0F0EC2FF07DEC03F046E9CC
:1049C0006ED1B4EC2FF0026E000E0121036E025086
:1049D000031005E00001758F0A016C6960D10001C8
:1049E000E5350CE200017551800B08E00001E52B74
:1049F0000A013C0E6C6F020E83EC2EF00001759FD5
:104A00004ED1000166510001075D0EE000016651C4
:104A1000020803E20F0E665D07E1040E0001075D68
:104A200003E0040E83EC2EF0000166510001075DE7
:104A300005E1000167510001085D09E0020E83EC09
:104A40002EF00001070503E10A01020E766F07C090
:104A500066F008C067F00B01CCA104D00F0E000176
:104A60000A1504D000010B390F0B0F0B016E00016A
:104A70006851015C05E001EB68F0020E83EC2EF05A
:104A800009C069F000010D510A0DF3CF6AF0F4CFAF
:104A90006BF005D10F0E0001665D02E10001078990
:104AA000000107510001715D0FE100010851000193
:104AB000725D0AE1000109510001735D05E1000129
:104AC0000A510001745D03E0020E83EC2EF0800EAB
:104AD000000172150AE1800E0001081506E0100EB3
:104AE000081503E0100E83EC2EF0020E0001741581
:104AF00007E1020E00010A1503E0200E83EC2EF000
:104B000007C071F008C072F009C073F00AC074F0F9
:104B100027EC30F01FE100018C518D118E118F11A7
:104B200019E10001885189118A118B1113E00A01E2
:104B3000020E766F88C08CF089C08DF08AC08EF02E
:104B40008BC08FF000018C07000E8D5B8E5B8F5B3E
:104B5000020E13D027EC30F001E1A1D000018C51FE
:104B60008D118E118F1101E19AD00A01020E766F1C
:104B700000018C6B8D6B8E6B8F6B83EC2EF08FD066
:104B80000A01760502E1030E766FE66A010EE66E13
:104B900000010851640DF3CF02FBF4CF03FB800E3C
:104BA0000B010227000E032302CBE6FF03CBE6FF37
:104BB00092EC5FF0E552E5CF01FBE7CF00FB00018F
:104BC0000951640DF3500B0100250001D76FF4501B
:104BD0000B0101210001D86F62D007C0A5F00001D0
:104BE000A66BA5BFA669000108510001A76FA86BBD
:104BF0000CC0A9F00001AA6BA9BFAA690001780E38
:104C0000C46F4DD0016A070E015C49E2BDEC2FF084
:104C1000015099EC2FF0F7D7016A070E015C07E20B
:104C2000BDEC2FF0070E012499EC2FF0F6D7410EC2
:104C30000001095D03E0420E095D03E10B01320E44
:104C400002D00B01310E976F380E0001095D02E1B1
:104C50000B01CC81330E0001075D03E10B01530E04
:104C600002D00B014E0E986F1AD007C0A1F008C0F9
:104C7000A2F009C0A3F013D0020E021910E1010E38
:104C800003190DE1000106510E0A09E10751000167
:104C9000765D03E0020E83EC2EF007C076F0010E85
:104CA00048E9E7CFD9FF12000001025142E1040EAA
:104CB00003193FE1020E0001065D01E0CCD0010EB8
:104CC0000B01CB1501E1C7D0010ECC1501E0C3D01B
:104CD00027EC30F001E1BFD0000108510001775D01
:104CE00001E1B9D00B01CD51000801E3B4D006C0F9
:104CF0006DFA07C06EFA77C06FFAF00E0001091561
:104D00000A01706F0AC071FA0BC072FA0CC073FA14
:104D10000DC074FA0F0140B7FDD7FDEC2EF00A016B
:104D2000050E756F75510A0801E395D00A0E756F6F
:104D3000010C440E021937E1030E031934E100019E
:104D40000951000808E208C0B5F009C0ADF0000143
:104D5000AE6BADBFAE6900010D51000808E20CC09A
:104D6000B6F00DC0AFF00001B06BAFBFB06900018D
:104D70000751000808E206C0B7F007C0B1F0000113
:104D8000B26BB1BFB26900010B51000808E20AC062
:104D9000B8F00BC0B3F00001B46BB3BFB46900014D
:104DA000780EC66F010C020E021955E1040E0319AC
:104DB00052E100010651FA0A4EE109C010FB0B0155
:104DC000116B126B136B0AC014FB156B166B176B10
:104DD000080E1F0B08E00B01D89014371537163753
:104DE0001737E806F9E10B0114511027155111236B
:104DF00016511223175113230BC018FB196B1A6B92
:104E00001B6B100E1F0B08E00B01D89018371937D9
:104E10001A371B37E806F9E10B0118511027195111
:104E200011231A5112231B51132310CBBBF011CBAA
:104E3000BCF012CBBDF013CBBEF00DC011FB106B5C
:104E400000010C510B0110250001B96F000E0B0180
:104E500011210001BA6F010C0A01755102E1050E22
:104E6000756F000C0A017651010826E20B01CD5145
:104E700003E10A01766B20D0020E0A01765D0AE199
:104E8000010E766F0F0140B7FDD78CEC30F0A3EC2C
:104E90002FF012D0030E765D0FE1766B0F0140B755
:104EA000FDD7BBEC30F0476B486BA3EC2FF07CECEC
:104EB0002DF0020E83EC2EF00A01755101E1000C79
:104EC000020E6D5D18E1010E0B01CB1514E0010E11
:104ED000CC1511E127EC30F00EE00B01CD510008AC
:104EE0000AE2010EE66EBEEC92F041E90F0140B716
:104EF000FDD7FDEC2EF00A017507000C0F0140B73D
:104F0000FDD77DEC2EF00A0E466F010E456F080EA0
:104F1000406F40B7FED712000F0140B7FDD7BBEC82
:104F200030F02C0E476F010E486F496B4A6B090E2B
:104F30004B6F100E4C6F4D6B080E456F406F40B7B6
:104F4000FED712000F0140B7FDD78CEC30F0496B53
:104F50004A6B800E4B6F4C6B080E4D6F456F406F68
:104F600040B7FED712005FEC30F00F0140B7FDD71D
:104F70006AEC30F0190E1AEC2FF040B7FED795EF1F
:104F80002FF05FEC30F00F0140B7FDD76AEC30F046
:104F9000020E1AEC2FF040B7FED795EF2FF05FEC22
:104FA00030F00F0140B7FDD76AEC30F0030E1AEC79
:104FB0002FF040B7FED795EF2FF015EC2FF084E9D6
:104FC00044E85AEC30F07EEC7FF042E9FCC0D1FBC3
:104FD000FDC0D2FBFEC0D3FBFFC0D4FB0B01D151FF
:104FE000046ED251056ED351066ED451076E020E77
:104FF000025C03E127EC30F06EE10F0140B7FDD712
:105000007DEC2EF00B0E466F02EB47FF486B496BB1
:1050100057EC2FF00B01D1510F014A6F57EC2FF0D5
:10502000080E0B0108EC30F0FDE10B01D1510F012E
:105030004B6F57EC2FF0100E0B0108EC30F0FDE138
:105040000B01D1510F014C6F5AEC30F0DCEC85F0C4
:1050500042E9F3CFD5FBF4CFD6FB040EF3CFD1FB5F
:10506000F4CFD2FB000A06E00B01D890D137D2373B
:10507000E804FBE10B01D36BD46B04EBD7FB05EB2E
:10508000D8FB06EBD9FB07EBDAFB180ED890DA3326
:10509000D933D833D733E806F9E10B010F0EDB6FB4
:1050A000DC6BDD6BDE6BDB51D717DC51D817DD51C4
:1050B000D917DE51DA17D751D127D851D223D95178
:1050C000D323DA51D423D1CB4DFF0F01080E456F06
:1050D000406F40B7FED745E9E7CFD9FF120015EC86
:1050E0002FF084E90BDF0F0140B7FDD76AEC30F0F9
:1050F0001B0E476F486B496B02EB4AFF4B6B9AECF8
:1051000030F040B7FED7020414E16AEC30F01A0E1A
:10511000476F486B496B0B0101EBD1FBD26BD1514F
:105120000F014A6FFF0E00144B6F9AEC30F040B73E
:10513000FED795EF2FF05FEC30F00F0140B7FDD7B1
:105140007DEC2EF0090E466F476B00EB48FF030E17
:10515000456F080E406F40B7FED795EF2FF015EC66
:105160002FF081E944E800017151100B02E0010EBB
:1051700001D0000E0001EC6F68C0E6F063C0E7F0FC
:105180000F0EE66E18EC8BF041E9F350016EF4500F
:10519000026E0FEC30F001EBE6FF02EBE6FFAAEC4B
:1051A0002FF015E0F8EC2FF0F3CFE8F0F4CFE9F0B2
:1051B0000FEC30F0000EE66EE66AAAEC2FF00BE082
:1051C000F8EC2FF0F3CFEAF0F4CFEBF008D01F0E9D
:1051D0000001E86FE96B3C0E0001EA6FEB6B000128
:1051E000AA35AA510001E91902E6C6EC2FF02DE21A
:1051F00000017151800B29E17151040B26E07EDE24
:105200000A0EADEC30F0036A046A020ED89004BEB8
:1052100003D0035C000E045813E20D0EE66EB1DEFF
:1052200091EC2FF0030EE66E9EDE91EC2FF0010E56
:10523000E66EB5DE91EC2FF0032A000E0422E5D7CE
:1052400081DE0001E56B0A016C6945E9E7CFD9FF12
:10525000120015EC2FF086E943E8086A02EBF3FF31
:1052600003EBF4FF190EF31801E1F45001E113D13F
:10527000180EF31801E1F45001E105D1170EF318EF
:1052800001E1F45001E1E6D0160EF31801E1F4500B
:1052900001E1D9D0150EF31801E1F45001E1CCD0B1
:1052A000140EF31801E1F45001E1BFD0130EF3180E
:1052B00001E1F45001E1B4D0120EF31801E1F45011
:1052C00001E1A9D0110EF31801E1F45001E17AD007
:1052D000100EF31801E1F45052E00F0EF31801E143
:1052E000F45046E00C0EF31801E1F4502DE00B0EE3
:1052F000F31801E1F4500FE00A0EF31801E1F45045
:1053000002E0000EE5D00B01CD5101E1C7D012EC57
:105310002FF029DEBED00B01CD5101E1BFD0040E2C
:10532000000171150BE0070E0001675D07E0010E3B
:10533000E66E35DE41E90601FC6BB7D01E0EE66E67
:10534000230EE66E010EB6D00B01CD5101E1A6D0C1
:10535000000171A907D0E66A22DE41E906011E0EAE
:10536000FC6FA3D0440EE66E230EE66E010EA2D0B3
:105370000B01CD5101E192D05AEC30F01FD00B015E
:10538000CD5101E18BD080EB06F081EB07F03CECD6
:105390002FF008E03CEC2FF02C0804E0062A000E69
:1053A0000722F5D73CEC2FF02C082FE1CFEC2FF0A3
:1053B00012EC2FF0D8DD41E91DEC30F09DEC30F01F
:1053C000E0DD67D00B01CD5169E080EB06F081EBA9
:1053D00007F03CEC2FF008E03CEC2FF02C0804E048
:1053E000062A000E0722F5D73CEC2FF02C080DE121
:1053F000CFEC2FF01DEC30F09DEC30F0F4CFE6FF59
:1054000012EC2FF06CDE43E950D0D80EE66E220E7F
:10541000E66E010E4FD00B01CD5140E06FDD03D0A1
:105420000B01CD513BE078DD40D00B01CD5115E0B3
:105430005AEC30F0020E1AD00B01CD510EE05AECAE
:1054400030F0E66A14D00B01CD5107E05AEC30F091
:10545000030E0CD00B01CD5106E1EA0EE66E220ED2
:10546000E66E010E0BD05AEC30F0010EE66EA5DDB3
:1054700043E9D50EE66E220EE66E010ED8EC2EF054
:10548000010E086E19D00B01CD5108E012EC2FF07F
:1054900052DE41E90AD00B01CD5106E1EA0EE66E7B
:1054A000220EE66E010E06D05ADED50EE66E220EF4
:1054B000E66E010ED8EC2EF0045009E06FEC12F00D
:1054C000020EADEC30F0E66A33EC16F041E9010E65
:1054D00044E9E7CFD9FF120015EC2FF08FE964E81B
:1054E0007F0E0601C85D33E10D50E66EE66A550E8B
:1054F000E66ECF0EE66E000E7BEC2FF009EBE6FFBA
:105500000AEBE6FFDBDB07EBE6FF08EBE6FFD6DBAB
:1055100005EBE6FF06EBE6FFD1DB03EBE6FF04EB72
:10552000E6FFCCDB0BEBE6FF0CEBE6FFC7DB02EBA9
:10553000D1FB0B01D26BD1BFD26922EC30F0BEDBC4
:105540004E0EE66ECF0EE66E000E2BEC2FF00350E3
:10555000041004E1800E036E3E0E046E063404E275
:1055600005500008000E065403E3640E056E066A3B
:105570000D50040A5CE0070A34E0030A0AE0640EF6
:105580000D240B01D16FD26BD16DD21F000ED2232F
:105590007CD2B3EC2EF0DAAF02D0DB69DC69CFEC61
:1055A0002EF0A50EE66E040EC2EC2EF0800E0B015E
:1055B000D527380ED623010ED723000ED82352EC60
:1055C00030F0BF0E1D6E1E6AA90E216E226ACA0E31
:1055D000236E030E246E256E266A410E276E4D0E35
:1055E0004BD0C1DBDAAF02D0DB69DC69D8DB0A0E55
:1055F000E66E060EC7DB200E0B01D55F300ED65BC4
:10560000050ED75B000ED85B52EC30F0F40E1D6E29
:105610001E6AD70E216E226ABC0E236E3C0E246ECB
:10562000030E256E266A470E276E600E25D09BDB83
:10563000DAAF02D0DB69DC69B2DB580EE66E050E2C
:10564000A1DBD00E0B01D55FFB0ED65B010ED75B45
:10565000000ED85B52EC30F0DA0E1D6E1E6AA70EFB
:10566000216E226A940E236E8C0E246E060E256E19
:10567000266A520E276E5A0E286E083404E207502E
:105680000008000E085420E3640EE66EE66A05EB9F
:10569000E6FF06EBE6FF1FEBE6FF20EBE6FF02EC82
:1056A00061F0E552E5CFD2FBE7CFD1FB320E0B0123
:1056B000D127000ED22322EC30F04AEC5FF0E55205
:1056C000E550086EE750076E0050011008E000EB4F
:1056D000E9FF01EBEAFF07EBEEFF08EBEDFF0C340F
:1056E00004E20B500008000E0C5402E3FE0ED5D06D
:1056F00008340A50081804E60750095C08500A5894
:1057000002E3FD0ECAD0023405E202503C0802E278
:105710003C0E026E0B0100EC30F00926D2510A2239
:1057200000EC30F00726D251082208341E50081829
:1057300004E607501D5C08501E5804E29DEB07F07C
:105740009EEB08F0D8900C5004E6FC0E0B5C080EA3
:105750000C5807E3200ED16F010ED26FD36BD46BC0
:105760000FD0E90ED56F020E97DBDEAF02D0DF69F6
:10577000E069A6DBC70EDFDAD36FDC51D859D46FEE
:10578000D1510F6ED251106E040ED56F0E0E84DB08
:10579000DEAF02D0DF69E06993DBFA0ECCDADC51D0
:1057A000D859D151116ED251126E123402E3116ADE
:1057B000126A0FEBD1FB10EBD2FBD36BD46BD2AFE1
:1057C00002D0D369D46963EC30F002EBDDFBDE6B11
:1057D000DF6BE06BDDAF03D0DE69DF69E06970DBB2
:1057E00011EBD9FB12EBDAFBDB6BDC6BDAAF02D02F
:1057F000DB69DC69D4DA96EC61F0CEEC5FF082EC28
:1058000030F00B01D551D127D651D223D751D32314
:10581000D851D423D151136ED251146E0BEBD9FB56
:105820000CEBDAFBDB6BDC6BDAAF02D0DB69DC693B
:10583000B6DA100EE66E0E0EE66EE66AE66A13EB58
:10584000D5FB14EBD6FBD76BD86BD6AF02D0D7699C
:10585000D86935EC30F096EC61F0B7EC30F00B0124
:10586000D151156ED251166ED351176ED451186E98
:105870009FDBE20EE66EE6681D0E39DBD8900B0169
:10588000D451000A08E6F40ED15D000ED259000E84
:10589000D359000ED45904E2FC0EF36EF468F9D02B
:1058A000196A1A6A1B6A1C6A22340A50221804E612
:1058B0002150095C22500A582EE222340850221846
:1058C00004E62150075C2250085805E207EBD1FBA3
:1058D00008EBD2FB04D021EBD1FB22EBD2FBD15160
:1058E0002B6ED2512C6E09502B5CD56F0A502C5860
:1058F000D66FD76BD86BD6AF02D0D769D869B5DB76
:1059000057DB96EC61F0A7DBD950190FE96EDACFBF
:10591000EAFF0B0156DB08342250081804E6075052
:10592000215C0850225801E39DD00A3422500A1805
:1059300004E60950215C0A50225805E209EBD1FB2C
:105940000AEBD2FB04D021EBD1FB22EBD2FBD151ED
:105950002D6ED2512E6E0C340AE20B50D008070E79
:105960000C5405E2D00ED56F070ED66F04D00BEBAA
:10597000D5FB0CEBD6FBD76BD86BD6AF02D0D76973
:10598000D86973DB480EE66E0B0EE66E110EAFDAC9
:105990000B01D1512F6ED251306E08342E500818A1
:1059A00004E607502D5C08502E585CE22DEBE6FF14
:1059B0002EEBE6FF640EE66EE66A02EC61F00B0188
:1059C000FE0EE350275CD56F41E9E5502858D66FAD
:1059D000D76BD86BD6AF02D0D769D86946DB23EB3B
:1059E000E6FF24EBE6FF25EBE6FF26EBE6FFBFDB59
:1059F0000B01D151316ED251326E323409E2323460
:105A00003050321804E631502F5C3250305805E2E5
:105A1000AFEB31F0B0EB32F016D008DBD2AF02D0F2
:105A2000D369D4691834D451181808E61550D15DDB
:105A30001650D2591750D3591850D45904E295EB47
:105A400031F096EB32F0F2DAD2AF02D0D369D469FA
:105A5000D950190FE96EDACFEAFFB3DA2D2A000E1A
:105A60002E229BD77F0E0601C85D0EE107DBEADA26
:105A70002F0EE66ECF0EE66E000E3DDA2C0EE66EB1
:105A8000CF0EE66E000EE7D9F9DAD1CBF3FFD2CB19
:105A9000F4FF65E9E7CFD9FF12000001E5352BE2FD
:105AA00000017151100B27E0000E0A01E76E6C191E
:105AB00002E76C3502D06C51E75C14E26C070A0E09
:105AC0006C5D06E1040EE66EB3EC27F041E90AD006
:105AD0006C5108E1030EE66EB3EC27F041E90A01D0
:105AE0003C0E6C6F0D0E0001635D05E00D0EE66E61
:105AF000C1EC27F041E9000C000171A949D0C2D9DD
:105B0000640E21DBF3CFDAF0F4CFDBF00001DC69C7
:105B1000DD690001E0510008000EE1550DE2B2D947
:105B2000640EE66EE66AE0C0E6FFE1C0E6FFD1D8AB
:105B3000F3CFDCF0F4CFDDF00001DE69DF690001B6
:105B4000E251000807E29ED9E251FDDAF3CFDEF020
:105B5000F4CFDFF00001E5352BE20001EA07000E8B
:105B6000EB5BA2EC27F00001EA51EB1108E0000129
:105B7000AA35AA510001E91901E608DA19E3BED9EC
:105B800041E90001EC5110E1E66ACFEC27F00BD0BF
:105B9000000E0001E76EE51902E7E53502D0E55198
:105BA000E75C06E2ABD941E90001E5690A016C69ED
:105BB000000C3BD981E942E80B01540E956F520E5F
:105BC000966F976B986B996B900E6F6E6EAEFED75B
:105BD000606A0F01A00E196F1869016B200E006F2B
:105BE000506BE00E1D6F1C69800E096F680E086F08
:105BF000400E0D6F800E0C6F116B106F706AD20E1D
:105C0000716E020E726E200E736E0B01CD51000884
:105C100002E26F6A02D0600E6F6E0001EC6B0A0147
:105C20006D6B756B766B6C690601EE850001D60EA7
:105C3000136F250E146F010E156F0001040E196FFE
:105C4000460E1A6F000E1B6F0001A80E1C6F4C0E43
:105C50001D6F000E1E6F0001580E316F4E0E326F19
:105C6000000E336F00019A0E1F6F5A0E206F000E48
:105C7000216F0001F80E256F5A0E266F000E276F58
:105C80000001640E346F4E0E356F000E366F00014A
:105C9000520E376F520E386F000E396F0001D80E5A
:105CA000406F540E416F000E426F43E9E7CFD9FFBA
:105CB0001200D723D823D9D9B7EF30F0520EE66EB1
:105CC000CF0EE66E000EE66E29EBE6FF2AEBE6FF4E
:105CD00029D279C0E6FF7AC0E6FF00016351E66E83
:105CE000E66A60C0E6FF61C0E6FF02EC61F068C0F2
:105CF000E6FF6CEC2AF04EE91200406B400E426F5A
:105D0000200E416F1200E66EE66AA9EC03F042E94C
:105D10001200E4D90CC008FB096B0A6B0B6B100E68
:105D20001F0B1200E5D90DC00CFB0D6B0E6B0F6B3A
:105D3000180E1F0B1200E66EE66A0BDACEEC5FF06F
:105D4000E552E5CFDCFBE5CFDBFBE5CFDAFBE7CFC8
:105D5000D9FB0B01D951D55DD16FDA51D659D26F2C
:105D6000DB51D7591200A00EE66E860EE66E010ECC
:105D7000E66EE66A03EBD9FB04EBDAFB0B01DB6BA7
:105D8000DC6B1200E66EE5D982EF30F009C001FB52
:105D90000B01006B000108510B0100251200D9CB4B
:105DA000E6FFDACBE6FFDBCBE6FFDCCBE6FF12005B
:105DB000E66E02EBE6FF03EBE6FFCE0EE66E220E8A
:105DC000E66E010EE66ECED96DEC43F047E9F3CFF7
:105DD000E6FFF4CFE6FF19EC43F045E912000AC0F4
:105DE00000FB0B01016B026B036B0BC004FB056B2B
:105DF000066B076B080E1F0B1200406B426B800E88
:105E0000416F6DCA46FF6ECA47FF6FCA48FF70CA2E
:105E100049FF71CA4AFF72CA4BFF73CA4CFF74CA6A
:105E20004DFFADD147D99DEF30F0D9CFE6FFE1CF9F
:105E3000D9FF1200476F486B496B00EB4AFF4B6B71
:105E40009AEF30F00C5100270D5101230E5102231F
:105E50000F5103231200E66E29EBE6FF2AEBE6FF63
:105E600019EC43F045E9F350296EF4502A6E7AD9C3
:105E7000E3EC02F042E9120006EBE9FF07EBEAFF70
:105E8000EF501200000EE66EE66A91C0E6FFD7C042
:105E9000E6FFD8C0E6FF1200D66FD76BD86B13D9D8
:105EA0000BEBDDFB0CEBDEFBDF6BE06B120004EBBE
:105EB000D1FB05EBD2FB06EBD3FB07EBD4FB1200C7
:105EC000DDCBE6FFDECBE6FFDFCBE6FFE0CBE6FF98
:105ED0001200D8900437053706370737E806120056
:105EE000D890083709370A370B37E8061200E66EF4
:105EF000E66AB7EF30F0E66E35D914D106011E0E12
:105F0000FC6FE7C0E6FFC1EC27F041E9E6C0E6FF21
:105F1000B3EF27F0D8900C370D370E370F37E80660
:105F2000120041E9010EADEF30F041E9E7CFD9FFB2
:105F30001200EA6A930FE96E000EEA22E552E7507A
:105F4000EF6E012A1200496B4A6B4B6B4C6B400E93
:105F50004D6F15D103EC91F045E9F350016EF4500B
:105F6000026E0150021012000DC001FB0B01006B0C
:105F700000010C510B01002512000128EA6A060FEE
:105F8000E96E000EEA22EF50E66E12000001A95100
:105F90000001E85D0001AA510001E959120006EB79
:105FA000E9FF07EBEAFF062A000E0722EF6A12005C
:105FB00015EBE6FF16EBE6FF17EBE6FF18EBE6FF47
:105FC0001200D151EE26D251EE22D351EE22D451FD
:105FD000EE2212000B01D1511F6ED251206E120021
:105FE000E66AE66AE66AE66A000EE66EE66A1200AD
:105FF00001EBE6FF02EBE6FF09EC7FF042E912005D
:106000001F501D5CD16F20501E58D26FD15112000D
:10601000D890D433D333D233D133E80612006D0E87
:10602000E66ECF0EE66E000EE66E120031EBD1FB8F
:1060300032EBD2FBD36BD46B120006EBE6FF07EB1F
:10604000E6FF1200D1CBE6FFD2CBE6FF1200800EB6
:10605000000171151200E552E5CFD4FBE5CFD3FB6B
:10606000E5CFD2FBE7CFD1FB1200D5CBE6FFD6CBF5
:10607000E6FFD7CBE6FFD8CBE6FF12003C0EE66E7C
:10608000E66AE66AE66A19EBD5FB1AEBD6FB1BEB70
:10609000D7FB1CEBD8FB1E0E0B01D527000ED62319
:1060A00059EF2EF0500ED527C30ED623000E01DE79
:1060B000EAEF2FF000EBE6FF01EBE6FF1200B5DEA2
:1060C00082E97EEF27F0E80EE66E030EE66EE66AE2
:1060D000E66A120012DE050E466F12000B01045133
:1060E0000027055101230651022307510323120003
:1060F0000B0108510027095101230A5102230B51BA
:1061000003231200E552E5CFD8FBE5CFD7FBE5CF5F
:10611000D6FBE7CFD5FB12002ED8D00E476F070E67
:10612000486F12006DEC43F047E9F350296EF450CC
:106130002A6E12004C6B4D6B22D009EC7FF042E9C5
:10614000F3CFE6FF1200E66EE66AE668E66869EFFE
:106150002EF0E66AE66A96EF61F0E66EF7EC3DF047
:1061600041E91200000EE66E070EE66E1200CEEC5C
:106170005FF02BEF30F0C1DD060E466F1200080E07
:06618000456F406F1200A4
:0A61860019EC3CF083E91BEC3BF040
:1061900079EC3BF0EE6AEE6AEE6AEE6A1BEC3BF0DD
:1061A000EE6AEE6AEE6AEE6A77EC3CF0010EEE6E95
:1061B000230EEE6E450EEE6E670E76EC3BF079EC3C
:1061C0003BF0890EEE6EAB0EEE6ECD0EEE6EEF0E68
:1061D00076EC3BF0080EE926000EEA22FE0EEE6E8B
:1061E000DC0EEE6EBA0EEE6E980E76EC3BF00C0EF8
:1061F000E926000EEA22760EEE6E540EEE6E320E98
:10620000EE6E100EEE6E41E9E7CFD9FF120019ECE9
:106210003CF087E948E80B01030ED56F1EEC3BF01C
:1062200060EC3BF004E00B0166EC3BF0FDE17BEC45
:106230003BF0076ED251086ED351096ED4510A6EED
:1062400000EBD5FB01EBD6FBD76BD86BD6AF02D0FA
:10625000D769D869030E1F0B04E00B0183EC3BF0F8
:10626000FDE11EEC3BF00B01D551EF26EECFD1FB4B
:10627000D651EF22EECFD2FBD751EF22EECFD3FB98
:10628000D851EF22EECFD4FB00EBD9FB01EBDAFBC8
:10629000DB6BDC6BDAAF02D0DB69DC69030E1F0B52
:1062A00008E00B01D890D937DA37DB37DC37E8065E
:1062B000F9E10B01D951D15DDA51D259DB51D359F2
:1062C000DC51D45908E21EEC3BF079EC3BF0EE2AAD
:1062D000EE22EE22EE2200EBD1FB01EBD2FBD36BE0
:1062E000D46BD2AF02D0D369D4691D0E66EC3BF0FB
:1062F000FDE11EEC3BF079EC3BF00B013CEC3CF09B
:10630000400ED56FD66BD76BD86BD950070F57ECB3
:106310003BF0EE50D859D1510D6ED2510E6E0E3465
:1063200001500E1804E60D50005C0E50015845E374
:106330000DEBE6FF0EEBE6FF02EBE6FF03EBE6FFFD
:106340004BEC3BF0E9CFD3FBEACFD4FB0750E92479
:10635000D16F0850EA208AEC3BF0D3EC84F046E998
:106360004BEC3BF04EEC3BF032EC3BF08DEB0BF0AA
:106370008EEB0CF03F0E0B010B24D16F000E0C20A6
:10638000D26F0134D251011804E60050D15D0150A2
:10639000D2590EE202500B24D16F03500C208AEC2C
:1063A0003BF032EC3BF0400E0B26000E0C22E2D705
:1063B000076A086A096A0A6A02D00B6A0C6A0B50FB
:1063C000005CD16F0C5001588AEC3BF002500B245A
:1063D000D36F03500C20D46FD3CBE6FFE66E4BECAB
:1063E0003BF0E9CFD7FBEACFD8FB0750E924D56FC4
:1063F0000850EA20D66FD5CBE6FFE66ED3EC84F0EA
:1064000046E98FEF3BF019EC3CF085E951E8080EC6
:1064100093EC3BF01BEC3BF04EEC3BF0D950050FFE
:10642000E66EDACFE6FF57EC38F048E90B01030ED1
:10643000D56F1BEC3BF060EC3BF004E00B0166EC2D
:106440003BF0FDE17BEC3BF0C0EC3CF0380E0D5C2A
:10645000000E0E58000E0F58000E10580DE2380EA8
:10646000D56FD66BD76BD86BD9500D0F57EC3BF06F
:10647000D36FEE50D85913D0780ED96FDA6BDB6B2F
:10648000DC6BD9500D0FB0EC3DF0D95DD16FEE5003
:10649000DA59D26FEE50DB59D36FEE50DC59D46F1E
:1064A00045EC3CF0115012101310141004E0800E53
:1064B000156EC8EC3CF0156AD950110F40EC3DF058
:1064C000EE06000EEE5AEE5AEE5A1150121013104C
:1064D000141003E0C8EC3CF0EFD7080EE66EE66A55
:1064E000D950050F21EC3BF0100E93EC3BF077EC0C
:1064F0003CF04EEC3BF002EBE6FF03EBE6FF57EC23
:1065000038F048E952E9E7CFD9FF120019EC3CF026
:1065100085E950E802EBE9FF03EBEAFFEE50056E78
:10652000EE50066EEE50076EEF50086E040E2CEC27
:106530003BF0EE50096EEE500A6EEE500B6EEF50CF
:106540000C6E080E2CEC3BF0EE500D6EEE500E6E05
:10655000EE500F6EEF50106E0C0E2CEC3BF0EE5028
:10656000116EEE50126EEE50136EEF50146E400E20
:1065700093EC3BF000EBE6FF01EBE6FFBE0EE66EB0
:106580000A0EE66E8CEC38F048E975EC39F0D9501B
:10659000090FB0EC3DF00B01CFEC3CF099EC39F079
:1065A000D6EC39F08EEC3DF0F0EC39F0780EDD6F82
:1065B000A40EDE6F6A0EDF6FD70E44EC3DF004E0F0
:1065C0000B016BEC39F0FDE17CEC3CF064EC39F054
:1065D000FDE109EC3DF001EC3AF0560EDD6FB70E2F
:1065E000DE6FC70EDF6FE80E49EC3DF004E00B01F3
:1065F0006BEC39F0FDE180EC3CF064EC39F0FDE14E
:10660000EAEC3CF012EC3AF0DB0EDD6F700EDE6F60
:10661000200EDF6F240E67EC3DF004E00B016BEC05
:1066200039F0FDE184EC3CF064EC39F0FDE1F7EC8D
:106630003CF023EC3AF0EE0EDD6FCE0EDE6FBD0EB9
:10664000DF6FC10E4EEC3DF004E00B016BEC39F056
:10665000FDE188EC3CF064EC39F0FDE104EC3DF048
:1066600034EC3AF0AF0EDD6F0F0EDE6F7C0EDF6F95
:10667000F50E44EC3DF004E00B016BEC39F0FDE16C
:106680007CEC3CF064EC39F0FDE109EC3DF045ECCC
:106690003AF02A0EDD6FC60EDE6F870EDF6F470EF3
:1066A00049EC3DF004E00B016BEC39F0FDE180ECCE
:1066B0003CF064EC39F0FDE1EAEC3CF056EC3AF0E9
:1066C000130EDD6F460EDE6F300EDF6FA80E67EC27
:1066D0003DF004E00B016BEC39F0FDE184EC3CF0A3
:1066E00064EC39F0FDE1F7EC3CF067EC3AF0010EB8
:1066F000DD6F950EDE6F460EDF6FFD0E4EEC3DF04A
:1067000004E00B016BEC39F0FDE188EC3CF064EC4B
:1067100039F0FDE104EC3DF078EC3AF0D80EDD6F95
:10672000980EDE6F800EDF6F690E44EC3DF004E0E2
:106730000B016BEC39F0FDE17CEC3CF064EC39F0E2
:10674000FDE109EC3DF089EC3AF0AF0EDD6FF70E9C
:10675000DE6F440EDF6F8B0E49EC3DF004E00B0161
:106760006BEC39F0FDE180EC3CF064EC39F0FDE1DC
:10677000EAEC3CF09AEC3AF0B10EDD6F5B0EDE6FA6
:10678000DF69E0691EEC3CF0B7EC3BF0110E1F0B2B
:1067900004E00B016BEC39F0FDE184EC3CF064ECBF
:1067A00039F0FDE1F7EC3CF0ABEC3AF0BE0EDD6FFA
:1067B000D70EDE6F5C0EDF6F890E4EEC3DF004E00D
:1067C0000B016BEC39F0FDE188EC3CF064EC39F046
:1067D000FDE104EC3DF0BCEC3AF0220EDD6F110E51
:1067E000DE6F900EDF6F6B0E44EC3DF004E00B01AA
:1067F0006BEC39F0FDE17CEC3CF064EC39F0FDE150
:1068000009EC3DF0CDEC3AF0930EDD6F710EDE6FCA
:10681000980EDF6FFD0E49EC3DF004E00B016BECD0
:1068200039F0FDE180EC3CF064EC39F0FDE1EAEC9C
:106830003CF0DEEC3AF08E0EDD6F430EDE6F790E2B
:10684000DF6FA60E67EC3DF004E00B016BEC39F056
:10685000FDE184EC3CF064EC39F0FDE1F7EC3CF058
:10686000EFEC3AF0210EDD6F080EDE6FB40EDF6F35
:10687000490E4EEC3DF004E00B016BEC39F0FDE10C
:1068800088EC3CF064EC39F0FDE10FEC3DF001ECFC
:106890003AF0620ED96F250EDA6F1E0EDB6FF60E20
:1068A00053EC3DF004E00B016BEC39F0FDE18CECB6
:1068B0003CF064EC39F0FDE119EC3DF056EC3AF0B7
:1068C000400ED96FB30EDA6F400EDB6FC00E98EC3E
:1068D0003DF004E00B016BEC39F0FDE190EC3CF095
:1068E00064EC39F0FDE123EC3DF0ABEC3AF0510EF5
:1068F000D96F5A0EDA6F5E0EDB6F260E9CEC3DF000
:1069000004E00B016BEC39F0FDE194EC3CF064EC3D
:1069100039F0FDE12DEC3DF0F0EC39F0AA0ED96F25
:10692000C70EDA6FB60EDB6FE90EA0EC3DF004E0A7
:106930000B016BEC39F0FDE198EC3CF064EC39F0C4
:10694000FDE10FEC3DF045EC3AF05D0ED96F100E15
:10695000DA6F2F0EDB6FD60E53EC3DF004E00B0127
:106960006BEC39F0FDE18CEC3CF064EC39F0FDE1CE
:1069700019EC3DF09AEC3AF0530ED96F140EDA6F21
:10698000440EDB6F020E98EC3DF004E00B016BEC63
:1069900039F0FDE190EC3CF064EC39F0FDE123ECE2
:1069A0003DF0EFEC3AF0810ED96FE60EDA6FA10EF2
:1069B000DB6FD80E9CEC3DF004E00B016BEC39F082
:1069C000FDE194EC3CF064EC39F0FDE12DEC3DF0A0
:1069D00034EC3AF0C80ED96FFB0EDA6FD30EDB6FD2
:1069E000E70EA0EC3DF004E00B016BEC39F0FDE1AB
:1069F00098EC3CF064EC39F0FDE10FEC3DF089ECF3
:106A00003AF0E60ED96FCD0EDA6FE10EDB6F210E94
:106A100053EC3DF004E00B016BEC39F0FDE18CEC44
:106A20003CF064EC39F0FDE119EC3DF0DEEC3AF0BD
:106A3000D60ED96F070EDA6F370EDB6FC30E98ECE8
:106A40003DF004E00B016BEC39F0FDE190EC3CF023
:106A500064EC39F0FDE123EC3DF023EC3AF0870ED5
:106A6000D96F0D0EDA6FD50EDB6FF40E9CEC3DF096
:106A700004E00B016BEC39F0FDE194EC3CF064ECCC
:106A800039F0FDE12DEC3DF078EC3AF0ED0ED96FE8
:106A9000140EDA6F5A0EDB6F450EA0EC3DF004E0E9
:106AA0000B016BEC39F0FDE198EC3CF064EC39F053
:106AB000FDE10FEC3DF0CDEC3AF0050ED96FE90E9B
:106AC000DA6FE30EDB6FA90E53EC3DF004E00B012F
:106AD0006BEC39F0FDE18CEC3CF0F6DBFEE119ECFF
:106AE0003DF012EC3AF0F80ED96FA30EDA6FEF0E0C
:106AF000DB6FFC0E98EC3DF003E00B01ECDBFEE1FC
:106B000090EC3CF0E1DBFEE123EC3DF067EC3AF089
:106B1000D90ED96F020EDA6F6F0EDB6F670E9CEC29
:106B20003DF003E00B01D7DBFEE194EC3CF0CCDB65
:106B3000FEE12DEC3DF0BCEC3AF08A0ED96F4C0E24
:106B4000DA6F2A0EDB6F8D0EA0EC3DF003E00B0137
:106B5000C2DBFEE198EC3CF0B7DBFEE176EC3DF009
:106B600045EC3AF0420ED96F390EDA6FFA0EDB6F50
:106B7000DC6928EC3CF0AFEC3BF0040E1F0B03E0AB
:106B80000B01A9DBFEE19CEC3CF09EDBFEE179EC25
:106B90003DF078EC3AF0810ED96FF60EDA6F710E97
:106BA000DB6F870EA4EC3DF003E00B0194DBFEE10C
:106BB000A0EC3CF089DBFEE17CEC3DF0ABEC3AF084
:106BC000220ED96F610EDA6F9D0EDB6F6D0EA8EC91
:106BD0003DF003E00B017FDBFEE1A4EC3CF074DB55
:106BE000FEE17FEC3DF0DEEC3AF00C0ED96F380E92
:106BF000DA6FE50EDB6FFD0EACEC3DF003E00B0150
:106C00006ADBFEE1A8EC3CF05FDBFEE176EC3DF0F8
:106C1000F8DB440ED96FEA0EDA6FBE0EDB6FA40EFE
:106C20006CEC3DF003E00B0156DBFEE19CEC3CF02C
:106C30004BDBFEE179EC3DF034EC3AF0A90ED96F74
:106C4000CF0EDA6FDE0EDB6F4B0EA4EC3DF003E0EF
:106C50000B0141DBFEE1A0EC3CF036DBFEE17CEC1D
:106C60003DF067EC3AF0600ED96F4B0EDA6FBB0E59
:106C7000DB6FF60EA8EC3DF003E00B012CDBFEE130
:106C8000A4EC3CF021DBFEE17FEC3DF09AEC3AF025
:106C9000700ED96FBC0EDA6FBF0EDB6FBE0EACECA0
:106CA0003DF003E00B0117DBFEE1A8EC3CF00CDB50
:106CB000FEE176EC3DF0CDEC3AF0C60ED96F7E0EDB
:106CC000DA6F9B0EDB6F280E6CEC3DF003E00B01DE
:106CD00002DBFEE19CEC3CF0F7DAFEE179EC3DF002
:106CE0007FDBFA0ED96F270EDA6FA10EDB6FEA0E8B
:106CF000A4EC3DF003E00B01EEDAFEE1A0EC3CF089
:106D0000E3DAFEE17CEC3DF09EDB850ED96F300EC0
:106D1000DA6FEF0EDB6FD40EA8EC3DF003E00B0151
:106D2000DADAFEE1A4EC3CF0CFDAFEE17FEC3DF0F4
:106D3000BDDB050ED96F1D0EDA6F880EDB6F040EFA
:106D4000ACEC3DF003E00B01C6DAFEE1A8EC3CF050
:106D5000BBDAFEE176EC3DF0DCDB390ED96FD00E0C
:106D6000DA6FD40EDB6FD90E6CEC3DF003E00B0153
:106D7000B2DAFEE19CEC3CF0A7DAFEE179EC3DF002
:106D8000BCEC3AF0E50ED96F990EDA6FDB0EDB6FD3
:106D9000E60EA4EC3DF003E00B019DDAFEE1A0EC71
:106DA0003CF092DAFEE17CEC3DF0EFEC3AF0F80ECC
:106DB000D96F7C0EDA6FA20EDB6F1F0EA8EC3DF0D0
:106DC00003E00B0188DAFEE1A4EC3CF07DDAFEE1A1
:106DD0007FEC3DF027DB650ED96F560EDA6FAC0EF7
:106DE000DB6FC40EACEC3DF003E00B0174DAFEE1A6
:106DF000A8EC3CF069DAFEE182EC3DF0F1DA440EF9
:106E0000D56F220ED66F290ED76FF40E58EC3DF0D9
:106E100003E00B0160DAFEE1ACEC3CF055DAFEE198
:106E200085EC3DF054DB970ED56FD6692A0ED76FEF
:106E3000430E5DEC3DF003E00B014DDAFEE1B0ECFA
:106E40003CF042DAFEE188EC3DF0B8DBA70ED56FEE
:106E5000230ED66F940ED76FAB0E71EC3DF003E0AE
:106E60000B0139DAFEE1B4EC3CF02EDAFEE18BECFA
:106E70003DF00BDB390ED56FA00ED66F930ED76F9A
:106E8000FC0E62EC3DF003E00B0125DAFEE1B8EC0C
:106E90003CF01ADAFEE182EC3DF06EDBC30ED56FFA
:106EA000590ED66F5B0ED76F650E58EC3DF003E0C0
:106EB0000B0111DAFEE1ACEC3CF006DAFEE185EC08
:106EC0003DF0C1DA920ED56FCC0ED66F0C0ED76F97
:106ED0008F0E5DEC3DF003E00B01FDD9FEE1B0EC5F
:106EE0003CF0F2D9FEE188EC3DF024DB7D0ED56F5D
:106EF000F40ED66FEF0ED76FD86932EC3CF0B7ECDA
:106F00003BF00F0E1F0B03E00B01E5D9FEE1B4ECE3
:106F10003CF0DAD9FEE18BEC3DF073DAD10ED56F9F
:106F20005D0ED66F840ED76F850E62EC3DF003E0E8
:106F30000B01D1D9FEE1B8EC3CF0C6D9FEE182EC00
:106F40003DF0D6DA4F0ED56F7E0ED66FA80ED76FF6
:106F50006F0E58EC3DF003E00B01BDD9FEE1ACEC47
:106F60003CF0B2D9FEE185EC3DF039DBE00ED56FA7
:106F7000E60ED66F2C0ED76FFE0E5DEC3DF003E0F3
:106F80000B01A9D9FEE1B0EC3CF09ED9FEE188EC02
:106F90003DF08CDA140ED56F430ED66F010ED76F0D
:106FA000A30E71EC3DF003E00B0195D9FEE1B4ECCA
:106FB0003CF08AD9FEE18BEC3DF0EFDAA10ED56F03
:106FC000110ED66F080ED76F4E0E62EC3DF003E047
:106FD0000B0181D9FEE1B8EC3CF076D9FEE182EC00
:106FE0003DF042DA820ED56F7E0ED66F530ED76F0C
:106FF000F70E58EC3DF003E00B016DD9FEE1ACEC6F
:107000003CF062D9FEE185EC3DF0A5DA350ED56F96
:10701000F20ED66F3A0ED76FBD0E5DEC3DF003E079
:107020000B0159D9FEE1B0EC3CF04ED9FEE188EC01
:107030003DF0F8D9BB0ED56FD20ED66FD70ED76FF5
:107040002A0E71EC3DF003E00B0145D9FEE1B4ECF2
:107050003CF03AD9FEE18BEC3DF05BDA910ED56F56
:10706000D30ED66F860ED76FEB0E62EC3DF003E0C9
:107070000B0131D9FEE1B8EC3CF026D9FEE16CDB26
:1070800008D902EBE9FF03EBEAFF57EC3CF0040EF2
:10709000E3DA4EEC3CF0080EDFDA69EC3CF00C0E63
:1070A000DBDA60EC3CF051E9E7CFD9FF1200E7DA18
:1070B00014DB31E2A8DBD7EC3CF0DEEC3CF0EFCFA8
:1070C000D4FB0B01D151E66E06500D24E96E07503A
:1070D0000E2071D9080E0B01F7D8FEE172EC3CF0DE
:1070E000D12B9DDB68D9100E0B01EED8FEE172ECBE
:1070F0003CF0020ED12793DB5ED9180E0B01E4D8C9
:10710000FEE1F0DB030ED1278ADBEA6EE552E750A1
:10711000EF6E7FDACDD703D3B2DADFDA01E38FD0B7
:1071200004500D24E96E05500E20EA6EEFCFD1FB1E
:107130000B01D26BD36BD46B63DAD92B000EDA233D
:10714000DB23DC23D9510424E96EDA510520EA6EF1
:10715000EFCFD5FBD66BD76BD86B080E1F0B03E0B8
:107160000B01D1DAFEE1F8DA0DEBE1FB0EEBE2FB0D
:107170000FEBE3FB10EBE4FB020EE127000EE22332
:10718000E323E423E1510424E96EE2510520EA6E91
:10719000EFCFDDFBDE6BDF6BE06B100E1F0B08E04B
:1071A0000B01D890DD37DE37DF37E037E806F9E14D
:1071B0000B01DD51D113DE51D213DF51D313E05156
:1071C000D4130DEBE9FB0EEBEAFB0FEBEBFB10EB43
:1071D000ECFB030EE927000EEA23EB23EC23E95135
:1071E0000424E96EEA510520EA6EEFCFE5FBE66B79
:1071F000E76BE86B180E1F0B08E00B01D890E53722
:10720000E637E737E837E806F9E10B01E551D11336
:10721000E651D213E751D313E851D413F4DA06241C
:10722000E96E41E9E5500720EA6ED1CBEEFFD2CB03
:10723000EEFFD3CBEEFFD4CBEEFFEBD96ED76FD200
:10724000D551D113D651D213D751D313D851D4130A
:10725000120040EC3DF03CEF3CF0D151056ED251B4
:10726000066ED351076ED451086ED950050F40EC0D
:107270003DF04EEF3CF009DBD950110F40EC3DF0F2
:1072800057EF3CF0D1517CDBD9500D0FF9DB60EFAB
:107290003CF0D151096ED2510A6ED3510B6ED451CC
:1072A0000C6ED950090FECDB69EF3CF0B0EC3DF00F
:1072B000D11BEE50D21BEE50D31BEE50D41B12004C
:1072C000B0EC3DF0CFEF3CF0D890D833D733D63385
:1072D000D533E8061200D890D137D237D337D43718
:1072E000E8061200DC6F28EF3CF00DEBD1FB0EEB53
:1072F000D2FB0FEBD3FB10EBD4FB120005EBD1FB61
:1073000006EBD2FB07EBD3FB08EBD4FB120009EB37
:10731000D1FB0AEBD2FB0BEBD3FB0CEBD4FB120043
:1073200011EBD1FB12EBD2FB13EBD3FB14EBD4FB31
:10733000120009EBD5FB0AEBD6FB0BEBD7FB0CEBF2
:10734000D8FB120005EBD5FB06EBD6FB07EBD7FB12
:1073500008EBD8FB120011EBD5FB12EBD6FB13EBBD
:10736000D7FB14EBD8FB12000DEBD5FB0EEBD6FBD5
:107370000FEBD7FB10EBD8FB1200F2DBD113EE5072
:10738000D213EE50D313EE50D413D9501200E06F45
:107390001EEF3CF0D86F32EF3CF0D551D11BD651E7
:1073A000D21BD751D31BD851D41B1200D51FD61FC7
:1073B000D71FD81F1200EA6EE552E750EF6E23DAAE
:1073C000F6DAEECFD5FBEECFD6FBEECFD7FBEFCF85
:1073D000D8FB1200D11FD21FD31FD41FD9501200C7
:1073E0000A01BE510B01D1270A01BF510B01D22363
:1073F0000A01C0510B01D3230A01C1510B01D4234F
:1074000012000A01C2510B01D1270A01C3510B011D
:10741000D2230A01C4510B01D3230A01C5510B0128
:10742000D42312000A01C6510B01D1270A01C7510A
:107430000B01D2230A01C8510B01D3230A01C95100
:107440000B01D42312000A01CA510B01D1270A01F2
:10745000CB510B01D2230A01CC510B01D3230A01DA
:10746000CD510B01D42312000A01CE510B01D127BB
:107470000A01CF510B01D2230A01D0510B01D323B2
:107480000A01D1510B01D42312000A01D2510B0180
:10749000D1270A01D3510B01D2230A01D4510B0188
:1074A000D3230A01D5510B01D42312000A01D6516E
:1074B0000B01D1270A01D7510B01D2230A01D85160
:1074C0000B01D3230A01D9510B01D42312000A0165
:1074D000DA510B01D1270A01DB510B01D2230A013A
:1074E000DC510B01D3230A01DD510B01D42312001F
:1074F0000A01DE510B01D1270A01DF510B01D22312
:107500000A01E0510B01D3230A01E1510B01D423FD
:1075100012000A01E2510B01D1270A01E3510B01CC
:10752000D2230A01E4510B01D3230A01E5510B01D7
:10753000D42312000A01E6510B01D1270A01E751B9
:107540000B01D2230A01E8510B01D3230A01E951AF
:107550000B01D42312000A01EA510B01D1270A01C1
:10756000EB510B01D2230A01EC510B01D3230A0189
:10757000ED510B01D42312000A01EE510B01D1276A
:107580000A01EF510B01D2230A01F0510B01D32361
:107590000A01F1510B01D42312000A01F2510B012F
:1075A000D1270A01F3510B01D2230A01F4510B0137
:1075B000D3230A01F5510B01D42312000A01F6511D
:1075C0000B01D1270A01F7510B01D2230A01F8510F
:1075D0000B01D3230A01F9510B01D42312000A0134
:1075E000FA510B01D1270A01FB510B01D2230A01E9
:1075F000FC510B01D3230A01FD510B01D4231200CE
:107600000DEBD9FB0EEBDAFB0FEBDBFB10EBDCFB3E
:107610001200D950090F34DAEE2A000EEE22EE22C3
:10762000EE22D9500D0F2CDA040EEE26000EEE22BB
:10763000EE22EE2212005BD9100E9ED1C6D9100E9A
:107640009BD1E66EDACFE6FF00EBE6FF01EBE6FF4B
:1076500007EC31F046E912000224E96E000E032027
:10766000EA6E1200B2D9E9CFD3FBEACFD4FBE9CF5F
:10767000E6FFEACFE6FF86EC32F044E91200D9D803
:1076800089E948E8096A0A6A0B6A0C6A0D6A0E6A97
:107690000F6A106A120099D9180E6ED1E9CFD1FB8A
:1076A000EACFD2FBE9CFE6FFEACFE6FF120058DAD5
:1076B000D55DD16FEE50D659D26FEE50D75912002A
:1076C000D5511F0B7BD9EECFD4FB1200D890D43309
:1076D000D333D233D133E806120000500D5C015091
:1076E0000E5802500F58035010581200EE6E77EFEC
:1076F0003CF0040E41D13F0E0B01D117D26BD36B7E
:10770000D46BD1511200D890D537D637D737D83768
:10771000E8061200D26FD1CBE6FFE66E120049E90F
:10772000E7CFD9FF1200E66EE66AE66AE66A120063
:1077300017DAD517EE50D617EE50D717EE50D817E8
:1077400020EF39F0D951D517DA51D617DB51D717B9
:10775000DC51D81720EF39F00B0120EF39F0050F7D
:1077600078DD7EEF39F0110F74DD90EF39F00D0FF9
:1077700070DD75EF39F0090F6CDD87EF39F0F3D963
:1077800095DDE9DDCDEF39F0F5D990DDEDDDCDEF1B
:1077900039F0F7D98BDDCDDDCDEF39F0F9D986DDC4
:1077A000D1DDCDEF39F075DDBBDD14DE090FE5DD90
:1077B0000D0F56EF39F051DD98DD0CDE050FDDDDE4
:1077C000090F56EF39F057DDA2DD04DE110FD5DDCC
:1077D000050F56EF39F056DD91DDFCDD0D0FCDDDE7
:1077E000110F56EF39F06CDDADDDD6EF39F068DD05
:1077F000B2DDD6EF39F064DDB7DDD6EF39F060DD0C
:1078000098DDD6EF39F0040EE66EE66A09EBE6FF86
:107810000AEBE6FF02EC61F0FE0EE3501200000EF0
:10782000D223D323D423D1510624E96ED251072089
:107830001200D9CFE6FFE1CFD9FF1200DD51D127E9
:10784000DE51D223DF51D323E051D423D95012008B
:10785000D951D127DA51D223DB51D323DC51D423A0
:10786000D9501200D551D127D651D223D751D32385
:10787000D851D423D9501200D151EE26D251EE2244
:10788000D351EE22D451EE221200D151116ED251B9
:10789000126ED351136ED451146E12000950EE269D
:1078A0000A50EE220B50EE220C50EE221200055030
:1078B000EE260650EE220750EE220850EE2212006D
:1078C0001150EE261250EE221350EE221450EE22EA
:1078D00012000D50EE260E50EE220F50EE221050E8
:1078E000EE2212000B01D551E66E75EF39F000EB78
:1078F000E9FF01EBEAFF120025DD190E0B01120072
:107900002ADD140E0B0112002FDD0F0E0B011200E9
:1079100010DD0A0E0B01120015DD1B0E0B0112000B
:107920001ADD170E0B0112001FDD120E0B011200E3
:1079300000DD0C0E0B01120005DD1C0E0B01120008
:107940000ADD150E0B0112000FDD100E0B011200E7
:10795000F0DC090E0B011200F5DC1A0E0B0112000F
:10796000FADC160E0B011200FFDC110E0B011200E7
:10797000E0DC0B0E0B011200E926000EEA221200D9
:107980000D6ED2510E6ED3510F6ED451106E120087
:10799000010EE66EE66AD950150F21EF3BF0D117C4
:1079A000EE50D217EE50D317EE50D4171200042425
:1079B000E96E41E9E5500520EA6E1200EECFD1FBF9
:1079C000EECFD2FBEECFD3FB120004EBE9FF05EBC9
:1079D000EAFF1200C1DED5D80ADF09EBD9FB0AEBBA
:1079E000DAFB0BEBDBFB0CEBDCFBA2EF3BF0B4DEDA
:1079F000CFD801DF05EBD9FB06EBDAFB07EBDBFBAE
:107A000008EBDCFBA2EF3BF0A7DEADD8F8DE8EEF93
:107A10003DF0A2DEAFD8E7DEF3DDA2EF3BF09CDE67
:107A200038DC7EDCD950090FE2DED9500D0F98EF1B
:107A30003BF092DE12DC59DCD950050FDCDED95068
:107A4000090F98EF3BF088DE16DC61DCD950110F8E
:107A5000D6DED950050F98EF3BF07EDE13DC4EDC0E
:107A6000D9500D0FC0DED950110F98EF3BF03ADC22
:107A7000B3EF3BF037DCB7EF3BF034DCBBEF3BF070
:107A8000E96EDACFEAFF120082DC69DE070E1F0B17
:107A900012007DDC68DE0C0E1F0B120078DC6BDE42
:107AA000160E1F0B12001EDC5ADE050E1F0B1200F5
:107AB00071DC55DE060E1F0B12006CDC54DE0A0E64
:107AC0001F0B120067DC57DE150E1F0B12005FDC68
:107AD0004EDE110E1F0B120005DC41DE040E1F0BE3
:107AE000120058DC44DE0F0E1F0B120035DEBFEF14
:107AF0003BF032DEC4EF3BF02FDEC9EF3BF02CDE73
:107B0000CEEF3BF029DED3EF3BF026DEDBEF3BF0A0
:107B100023DEE3EF3BF020DEEBEF3BF011EBD9FB94
:107B200012EBDAFB13EBDBFB14EBDCFBA2EF3BF01D
:107B30009EDF090E1F0B12009DDF0E0E1F0B1200A1
:107B40009CDF140E1F0B120092DF0B0E1F0B120096
:107B500091DF100E1F0B120090DF170E1F0B12008B
:107B60008FDFEE50120049EC39F075EC39F0D95046
:107B7000090F12002DEC39F087EC39F0D950050FC0
:107B800012003BEC39F07EEC39F0D950110F1200A5
:0E7B900042EC39F090EC39F0D9500D0F120094
:027B9E00FF00E6
:107BA00012009DEC46F0FDEC47F0060E015C05E28C
:107BB0009EA2FED79E92012AF8D761EF48F09DEC75
:107BC00046F082E9005003E0ECDF0006FBD7D1EF7E
:107BD00046F09DEC46F0FDEC47F07A0E015C05E2C4
:107BE0009EA2FED79E92012AF8D761EF48F09DEC45
:107BF00046F082E9005003E0ECDF0006FBD7D1EF4E
:107C000046F09DEC46F082E9D1EF46F09DEC46F05F
:107C100082E9D1EF46F081B004D08180050E65EC99
:107C200048F081900F0E65EC48F08180190E65EFE9
:107C300048F002EC49F037EC48F0420EE66ECD0E0B
:107C4000E66E000E06EC47F002E1000E25D037ECA0
:107C500048F03E0EE66ECD0EE66E000E06EC47F0E6
:107C600002E1010E19D037EC48F03A0EE66ECD0E67
:107C7000E66E000E06EC47F002E1030E0DD037EC85
:107C800048F0360EE66ECD0EE66E000E06EC47F0BE
:107C900002E1040E01D0000ED1EF46F002EC49F0F3
:107CA00049E86AEC48F0010E076E086AD950050FE2
:107CB000BFEC47F0F6EC48F00B6E0B5036E02D0EA3
:107CC0000B5C09E1E668E66805EC48F0E550086EF3
:107CD000E750076EEFD73A0E0B5C05E1D950030F62
:107CE000BFEC47F0E7D70A0EE66EE66AC7EC48F04D
:107CF000EECFE6FFEECFE6FF02EC61F0E552E5CF16
:107D0000D4FBE7CFD3FB0B500B01D325D16F000E73
:107D1000D421D26F300ED15F000ED25BC7EC48F099
:107D2000D1CBEEFFD2CBEDFFC5D73C0EE66E9CEC7F
:107D300047F002EC61F00B01FE0EE3500324D36F19
:107D400041E9E5500420D46FD3CBE6FFE66E05ECA5
:107D500048F021EC49F0D1CBF3FFD2CBF4FF4AE954
:107D6000E7CFD9FF1200E6EC48F047EC48F0FDE120
:107D7000EEEC46F0FE0EE66E9B0E30EC49F06FEC3A
:107D800048F0EE500B01D127EE50D223EE50D32312
:107D9000EE50D423FE0EE66E9B0E17EC47F0FF0E5E
:107DA0000B01D5277F0ED623000ED723D823100E24
:107DB0004EEC48F0FDE109EF49F0E6EC48F047EC05
:107DC00048F0FDE1EEEC46F0120EE66E9F0E30EC50
:107DD00049F0120EE66E9F0E17EC47F0060EC4EC4B
:107DE00048F00DEC47F0ABEC47F0DD697F0EDE6F3D
:107DF000DF6BE06BDD51D527DE51D623DF51D72372
:107E0000E051D823100E4EEC48F0FDE109EF49F0A7
:107E10009DEC46F08BE954E806EBD1FB07EBD2FB77
:107E200008EBD3FB09EBD4FBD90E0B01D1270B0ECA
:107E3000D223010ED323000ED423E0EC46F00AEC4B
:107E400048F0CCEC48F0040E3CEC49F0D1510F6EF8
:107E5000D251106ED351116ED451126E040ECEEC6D
:107E600046F00FEBE6FF9FEC47F00AEC48F096EC8B
:107E700061F00DEC47F0030E0B01D927000EDA2359
:107E8000DB23DC23D9CBE6FFDACBE6FFDBCBE6FF57
:107E9000DCCBE6FFB2EC46F0E0EC46F0090EE66E15
:107EA0004B0EE66E160EE66EE66A0BEBD5FB0CEBA0
:107EB000D6FB0DEBD7FB0EEBD8FBD52B000ED62354
:107EC000D723D82360EC47F0A00EE66E0F0EE2EC4D
:107ED00048F096EC61F0AAEC48F0C6EC47F0040ECE
:107EE000CEEC46F013EBE6FF14EBE6FF15EBE6FFF6
:107EF00016EBE6FF36EC49F0B2EC46F01F0ED12748
:107F0000000ED223D323D423E0EC46F055EC48F006
:107F1000CCEC48F0500E3CEC49F0CFEC47F0500E62
:107F2000CEEC46F0D8EC47F055EC48F096EC61F01A
:107F3000B2EC46F0D1511B6ED2511C6ED3511D6E66
:107F4000D4511E6E0B0ECEEC46F0D8EC47F0AAECE6
:107F500048F0E0EC46F017EBD5FB18EBD6FB19EB3D
:107F6000D7FB1AEBD8FB020ED527000ED623D7235A
:107F7000D823CCEC48F00C0ECEEC46F096EC61F039
:107F80000DEC47F00B01D951D55DD16FDA51D659BF
:107F9000D26FDB51D759D36FDC51D859D46FCFECA6
:107FA00047F00FEBD5FB10EBD6FB11EBD7FB12EB39
:107FB000D8FB310ED55F000ED65BD75BD85B60EC8B
:107FC00047F0640ECEEC46F0A6EC48F013EBD9FB7C
:107FD00014EBDAFB15EBDBFB16EBDCFB0B01D951E9
:107FE000D127DA51D223DB51D323DC51D4230BEB3D
:107FF000DDFB0CEBDEFB0DEBDFFB0EEBE0FBDD5105
:10800000D127DE51D223DF51D323E051D423C6EC54
:1080100047F004EBE9FF05EBEAFF13EBEEFF14EB8F
:10802000EDFFA6EC47F017EBEEFF18EBEDFFE9ECE8
:1080300046F01BEBEEFF1CEBEDFF55E9E7CFD9FF58
:1080400012009DEC46F087E90B014B0E005CD56FEA
:108050007D0E0158D66FD76BD86BD6AF02D0D769DB
:10806000D869040ECEEC46F0C00E0424E16F120E67
:108070000520E26F0C0E78EC48F0E56F000E035817
:10808000E66FE5CBE6FFE66E4AEC5FF0E552E5CF42
:10809000E4FBE7CFE3FB0B01E151E325DD6FE251A8
:1080A000E421DE6FDF6BE06BDEAF02D0DF69E069F9
:1080B000DDCBE6FFDECBE6FFDFCBE6FFE0CBE6FF86
:1080C00036EC49F0CEEC5FF00DEC47F0ABEC47F04E
:1080D0000C0EE66EE66A020E025CED6F000E0358AF
:1080E000EE6F0C0EE66EE66A78EC48F0F16F000E6B
:1080F0000358F26FF1CBE6FFE66E4AEC5FF002EC5C
:1081000061F0E552E5CFF0FBE7CFEFFB0B01EF515C
:10811000ED5DEB6FF051EE59EC6FEBCBE6FFE66EE9
:108120006F0EE66E010EE66E02EC61F04AEC5FF057
:10813000E552E5CFE8FBE7CFE7FB0B01E96BEA6B24
:10814000E8AF02D0E969EA69E751D527E851D623BB
:10815000E951D723EA51D823040EE66EE66A640E8D
:10816000E66EE66A240E0424F96F130E0520FA6FFA
:108170000C0E78EC48F0FD6F000E0358FE6FFDCB3F
:10818000E6FFE66E4AEC5FF0E552E5CFFCFBE7CF99
:10819000FBFB0B01F951FB25F76FFA51FC21F86F3E
:1081A000F7CBE6FFE66E4AEC5FF037EC48F002EC06
:1081B00061F04AEC5FF0E552E5CFF4FBE7CFF3FB6B
:1081C0000B01F56BF66BF4AF02D0F569F669F3516C
:1081D000D55DD16FF451D659D26FF551D759D36FC0
:1081E000F651D8590DEC49F0E8CFFFF0D1EF46F049
:1081F00002EC49F04EE8FFEC48F0200803E13BECCC
:1082000048F0F9D795EC48F07EEC7FF0AFEC48F001
:108210002E0EE66E95EC48F058EC85F043E9F350ED
:108220000F6EF450106E0F50101051E0076A086A7C
:10823000096A0A6A010E0B6E0C6A0D6A0E6A0F2A31
:10824000000E10220FEBE9FF10EBEAFFEF501FE0EA
:108250005EEC49F0C8EC46F0A6EC48F00FEBE9FF05
:1082600010EBEAFFEF50D00F0B01D56FD66BD76B39
:10827000D86B57EC47F069EC47F05EEC49F0CCEC7A
:1082800048F0A6EC48F00B01E0EC46F0D8D7FFEC44
:1082900048F02D080BE1E668E668E668E668C8EC99
:1082A00046F0A6EC48F00B0169EC47F0CCEC48F046
:1082B00020EC5EF0C8EC46F020EC5EF072EC60F072
:1082C000BBEC48F020EC5EF0B2EC5CF004D0BBEC10
:1082D00048F020EC5EF096EC46F0DCEC46F04FE91E
:1082E000E7CFD9FF120002EC49F047E86AEC48F00A
:1082F000086A096A0050011041E0FFEC48F03EE0D6
:10830000FFEC48F02009076E780E075C03E16AEC89
:1083100048F031D0300E075C0DE3075039080AE30E
:10832000300E075C87EC47F015E00B015AEC48F083
:10833000FDE110D0610E075C21E3075066081EE3E3
:10834000610E075C0A0F87EC47F004E00B015AEC62
:1083500048F0FDE108EBD5FB09EBD6FB0B01D76B31
:10836000D86BD551D113D651D213D751D313D8517D
:10837000D4132AEC47F03BEC48F0BCD703EBFCF0FD
:1083800004EBFDF005EBFEF006EBFFF07DEF48F0AF
:1083900002EC49F048E895EC48F02ADFAFEC48F0F1
:1083A000E66AE66AC80EE66E420EE66EBBEC48F080
:1083B00072EC60F0C1EC5EF096EC46F00B0169ECFB
:1083C00047F0E66AE66A700EE66E420EE66E640EEE
:1083D000CEEC46F0C8EC46F096EC61F020EC5EF096
:1083E000BBEC48F0B0EC5CF072EC60F0C8EC46F02E
:1083F00020EC5EF0B2EC5CF096EC46F00B012AEC5F
:1084000047F0E66AE66AE66A450EE2EC48F0610E7D
:10841000E66E450EE66EBBEC48F0E7EC61F0E7EC8B
:1084200061F0C1EC5EF096EC46F0DCEC46F074EFE7
:1084300048F09DEC46F085E944E80568066801349B
:108440002BE200500008000E015426E2A6EC47F093
:10845000022A000E0322EF50051A000E061A00062B
:10846000015A076A086A080ED89008BE03D0075C54
:10847000000E0858E4E20550010B08E0D8900632DF
:108480000532010E051AA00E061A03D0D890063246
:1084900005323FEC48F0E7D781EC48F045E9E7CFFB
:1084A000D9FF120002EC49F04BE809680A68170E80
:1084B000E66E18EC8BF041E9F3500C6EF4500D6E43
:1084C000036AF6EC48F00B6E0B5048E0060ED890AD
:1084D0000ABE03D0095C000E0A5840E20B50220A83
:1084E00039E0090A33E0040A18E0150A16E0160A12
:1084F00014E00A34E6E2060E095C000E0A58E1E2D6
:108500007BEC47F0EF500A0DF3500B24D00FE66ED2
:108510007BEC47F043EC48F0D4D7091C01E10A1C7E
:10852000D0E00B01D950030FD16FDACFD2FB092A6B
:10853000000E0A2209EBD3FB0AEBD4FBD151D32561
:10854000E96EDA50D421EA6EEF6ABBD7091C01E16B
:108550000A1CB7E0092A000E0A22B3D712EC48F031
:108560000550E66EE66A0450E66EE66A03500B01BB
:10857000DA6BD00FD96F070EDA23D9CBE6FFDACB4F
:10858000E6FF5FDD46E9FCC0D5FBFDC0D6FBFEC0C3
:10859000D7FBFFC0D8FB8C0E0B01D55F3D0ED65B21
:1085A000250ED75B000ED85B60EC47F0A6EC48F0D8
:1085B000DCEC46F04CE9E7CFD9FF1200BEDB83E9E3
:1085C0000050011015E0FFEC48F012E0FFEC48F01D
:1085D0000D0804E1E9EC46F00A0E06D0FFEC48F085
:1085E0005E0803E1F6DB2F0EEF6E3BEC48F0E8D7B8
:1085F000D8D3A3DB86E903EBE9FF04EBEAFFEFCF77
:10860000D1FB72EC47F00B01D15D0CE172EC47F04D
:1086100009E06FEC48F0EE2A000EEE22EE22032A6B
:108620000422E9D772EC47F002E0000E01D0010EFF
:10863000B8D383DB86E96FEC48F0EFCFF6FFEE2A84
:10864000EFCFF7FF000EEE22EFCFF8FFEE2208008B
:10865000F550E66E03EBE9FF04EBEAFF43EC48F06C
:1086600004E0032A000E0422E6D703EBF3FF04EB39
:10867000F4FF97D362DB85E9F6EC48F0E66EA6ECF2
:1086800047F043EC48F004E0022A000E0322F4D73E
:1086900002EBF3FF03EBF4FF84D326EC49F002E096
:1086A00050EC49F095EC48F053EC49F0E3DF44E935
:1086B00078D343DB89E903500410051007E04EDB53
:1086C0001AEC48F0F350066EF450076E95EC48F043
:1086D00002EBE6FF1AEC48F064D326EC49F002E026
:1086E00050EC49F053EC49F095EC48F029EC80F05F
:1086F00044E905EBE9FF06EBEAFFEF5004E0052A49
:10870000000E0622F6D781EC48F04BD329EC49F055
:1087100001E018DB58EC49F0C3EC80F046E9B9DB26
:10872000EF5003E03FEC48F0FAD7EEEC47F039D3D6
:1087300029EC49F001E006DB58EC49F0B8EC81F097
:1087400046E9A7DBEF5003E03FEC48F0FAD7EEEC48
:1087500047F027D3F2DA89E941E8005002260150B8
:108760000322F4DBEF6A80EB09F0095037E00B01DC
:10877000250ED16FCD0ED26F000ED36F04EBD4FB5C
:108780000F0ED417D56BD66BD76BD151D425F36EA2
:10879000D251D521F46ED351D621F86EF4CFF7FF24
:1087A000F3CFF6FF0800F550E66E0206000E035AFE
:1087B000CDDB43EC48F0D950040FE96EDACFEAFF85
:1087C000040EE76ED890030EEB32020EEB32010E70
:1087D000EB32EF32E706F6E10906C7D761EF48F062
:1087E00026EC49F002E050EC49F0040EE66EA4DB02
:1087F00095EC48F0E66AE66AADDF48E905EBE9FF8B
:1088000006EBEAFFEF5004E0052A000E0622F6D739
:1088100081EC48F0C6D229EC49F001E093DA080E69
:10882000E66EE66A58EC49F095DF48E932DBEF5036
:1088300003E03FEC48F0FAD7D1DBB3D214EC49F0B7
:1088400002E041EC49F0020EE66EE66ABFEC48F049
:1088500000EBE6FFE66AE66AE66A7CDF48E904EBDD
:10886000E9FF05EBEAFFEF5004E0042A000E0522C1
:10887000F6D704EBF3FF05EBF4FF93D25EDA8DE954
:108880004CE807500810091008E082DA0BEBE6FF0D
:10889000FAEC48F00A6EF4500B6E9CDBBBEC48F02F
:1088A000B8EC81F046E996DBDCEC85F042E9F35068
:1088B000186E1850F36E02340AE20150F35C000E99
:1088C000025405E2C4DB00EBEFFF182AF2D782DB8B
:1088D0000AEBE6FF0BEBE6FFCDDE44E9F3500A6E50
:1088E000F4500B6E0AEBF3FF0BEBF4FF4DE9E7CF0F
:1088F000D9FF120022DA8CE949E8010E0C6E0D6AEC
:108900000E6A0F6A80EB14F0145011E05EEC49F02F
:108910002CEC49F096EC61F0E552E5500F6EE55015
:108920000E6EE5500D6EE7500C6E1406EDD72CEC74
:1089300049F09AEC48F0AAEC48F043DB06500710E7
:10894000081002E0D0EC48F0105011101210131073
:1089500005E1053403E387DA2D0EEF6EF0DA13EB51
:10896000E6FF7DDBD3DE49E93EDB7DDA2E0EEF6EDE
:10897000300EE66EDADB2CEC49F0053407E3E668EE
:10898000E668E668E668D6DBE1DB08D002EBD1FBFF
:1089900003EBD2FB04EBD3FB05EBD4FBEDEC48F08F
:1089A000D1EC5FF05CDB6ADF4CE91DDB09EBF3FF28
:1089B0000AEBF4FF4AE9E7CFD9FF1200BED98CE9F0
:1089C00047E806500710081001E0EADB89EB0CF0DD
:1089D0008AEB0DF0106A116A0250031004100510A2
:1089E00009E111340150111804E61050005C1150D7
:1089F00001584AE33CDB0B010050105CD36F01507F
:108A00001158D46FD3CBE6FFE66E4DEC5FF0E55224
:108A100021EC49F00B01D151D2110CE1113401507C
:108A2000111804E61050005C1150015803E21BDAE3
:108A30002C0EEF6E5EEC49F07DDB46EC49F0A7DBD7
:108A4000092A0A22D1CBEFFF5EEC49F073DB2CEC54
:108A500060F0E552E550056EE550046EE550036E9A
:108A6000E750026E102A000E112210EBD1FB11EB21
:108A7000D2FB0B010050D119AFE10150D219ACE18A
:108A8000F2D92E0EEF6EA8D709040E6E000E0A580A
:108A90000F6E0E500C5C0F500D5818E2A9DAEF5013
:108AA000126E0EEBE9FF0FEBEAFFEF50E66EA0DA75
:108AB0000C2A000E0D22E7DA0EEBE9FF0FEBEAFFBE
:108AC0000E06000E0F5A12EBEFFFE3D760DBEF6AE2
:108AD00009EBF3FF0AEBF4FF10D32FD98AE944E83E
:108AE00004500510061001E02DD9033412E3D1D94A
:108AF000C6DA2D0EEF6ED2D90B01D11FD21FD31FB4
:108B0000D41FD151006ED251016ED351026ED45197
:108B1000036EE66AE66A610EE66E450E3FD9E66EC2
:108B200017D920EC5EF072EC60F072EC60F0FED8C9
:108B30000B01D1510A6ED2510B6ED3510C6ED45130
:108B40000D6E060E3FDB240EE66E740EE66E490EC9
:108B5000E66E70DB0DEBE6FFE7EC61F0C1EC5EF07A
:108B6000E66AE66AE66ADCDAC5DE4BE945E9E7CFA4
:108B7000D9FF1200E2D88AE947E804500510061030
:108B800001E0E0D887EB0AF088EB0BF00E6A0F6A81
:108B9000030ED8900FBE03D00E5C000E0F5823E2D8
:108BA0000F3409E20E500008000E0F5404E271D990
:108BB00066DA3A0EEF6E020E0E1807E10F5005E16D
:108BC000180E79DB2FEC60F05AD90A0EB7DA0A0ECC
:108BD000DBDA55D9060EB2DA060ED6DA50D90E2AED
:108BE000000E0F22D5D707040C6E000E08580D6E2C
:108BF0000C500A5C0D500B5812E20AEBE9FF0BEB2C
:108C0000EAFFEF50106EF4D9EF50E66E20DA3BDA4F
:108C1000EFD90C06000E0D5A10EBEFFFE9D739D94A
:108C2000EF6ADCD96AD289D88AE94AE8FBD990D8B8
:108C30002CEC60F07BD88C0E0B01D1273D0ED2239B
:108C4000250ED323000ED423BCD9D9500C0FDDDA66
:108C5000D9500A0FDADAD9500E0FD7DA70D913EBE0
:108C6000E6FF08EC3FF04AE90EEBE6FF0FEBE6FF0C
:108C700012DB33DD47E979D90AEBD1FB0BEBD2FBF1
:108C80000B01D36BD46BD2AF02D0D369D469D7D8E0
:108C90006CD90CEBD1FB0DEBD2FB0B01D36BD46B7E
:108CA000D2AF02D0D369D469CAD84BE9E7CFD9FF94
:108CB0001200BADA01E0E5DA0050040A18E0070A07
:108CC00010E0020A08E0010A1CE11A0EE66ECD0E61
:108CD000E66E000E11D0120EE66ECD0EE66E000EA0
:108CE0000BD00C0EE66ECD0EE66E000E05D0000E1B
:108CF000E66ECD0EE66E000EE66E41DA9ADC45E9D0
:108D00000CD00050E66EE66AFA0EE66ECC0EE66E09
:108D1000000EE66E34DAE1DC47E9F350046EF450FD
:108D2000056E04EBF3FF05EBF4FF3BD0E552E5CF16
:108D3000D4FBE5CFD3FB21EF49F0D9CFE6FFE1CF5C
:108D4000D9FF1200A8DA56DA076EF450086E120046
:108D5000ECD902EBE6FF03EBE6FF120003EBE6FFC4
:108D6000BFEF48F0CEEC5FF023DAD9500B0FE96E7D
:108D7000DACFEAFF0B01D551EE5CD16FD651EE5838
:108D8000D26FD751EE58D36FD851EE58D46F12002E
:108D9000C7D909EBE6FF0AEBE6FF120013DAE66A31
:108DA000120041E9E7CFD9FF12000CEBE6FF0DEB13
:108DB000E6FF0EEBE6FF120030DAD4CBFFF0120034
:108DC000D1510B6ED2510C6ED3510D6ED4510E6E2B
:108DD000120000EBE9FF01EBEAFF12000B01D15199
:108DE000056ED251066ED351076ED451086E00EB5A
:108DF000D1FB01EBD2FBD36BD46BD151096ED251B5
:108E00000A6ED3510B6ED4510C6E1200E66E8DD9E2
:108E1000B4EC84F047E900091200E552E5CFDCFB31
:108E2000E5CFDBFBE5CFDAFBE7CFD9FB1200CAD9F0
:108E300009EBE6FFFFD996EC61F0D8EF48F0CDD909
:108E4000230EE66ECD0EE66E000EE66E69D916DDD7
:108E50004CE91200D151036ED251046ED351056E0C
:108E6000D451066E120093D9092A000E0A2212006C
:108E700006EBE6FFBFD9056EF450066E1200E55210
:108E8000E550036EE550026EE550016EE750006E4E
:108E9000120007EBE9FF08EBEAFF120000EBD1FB41
:108EA00001EBD2FB02EBD3FB03EBD4FB1200D55159
:108EB000D127D651D223D751D323D851D42312004E
:108EC000D5CBE6FFD6CBE6FFD7CBE6FFD8CBE6FF88
:108ED0001200D151076ED251086ED351096ED45190
:108EE0000A6E120000EBF6FF01EBF7FF02EBF8FF52
:108EF0000800F5501200D950030F87D9FE0EE35039
:108F00000924E96E41E9E5500A20EA6E1200086E74
:108F1000096A03EBD1FB04EBD2FB05EBD3FB06EBB9
:108F2000D4FB040E1F0B1200300E0B01D127000ED4
:108F3000D223D323D4231200E66A53EF49F010EB77
:108F4000E6FF11EBE6FF12EBE6FF120002EBE9FF92
:108F500003EBEAFF12000B01D951D527DA51D623D2
:108F6000DB51D723DC51D8231200F350076EF450A5
:108F7000086E300EE66E020EE66EE66A120045D905
:108F8000E552E5500A6EE750096E1200D151136E9A
:108F9000D251146ED351156ED451166E1200D151A8
:108FA000176ED251186ED351196ED4511A6E120029
:108FB00017EBE6FF18EBE6FF19EBE6FF1AEBE6FF0F
:108FC0001200D151106ED251116ED351126ED45184
:108FD000136E1200D9500D0F05EF49F007EBF3FFA8
:108FE00008EBF4FF1200F350096EF4500A6E120001
:108FF0000CEBE9FF0DEBEAFF120081E941E8016AA1
:109000007C0ECA6ECC6ACB6812008AD802EC61F082
:10901000E5521200B10EE66E3A0EE66E020EE66EF4
:10902000E66A1200800EE66E510EE66E010EE66EE6
:10903000E66A120006EBE6FF07EBE6FF19EC43F0E9
:1090400045E91200D7D8046EF450056E12000AEB01
:10905000E9FF0BEBEAFF0A2A000E0B221200E66A78
:10906000E66AE66A09EBE6FF0AEBE6FF1200030E8A
:10907000E66EE66A1200002A000E01221200072A9C
:10908000000E08221200E552E750EF6E1200D89051
:10909000D433D333D233D133E8061200D890D83347
:1090A000D733D633D533E80612008F0EE66E090E9D
:1090B000E2EF48F0D890D137D237D337D437E8062B
:1090C000120042E9E7CFD9FF1200E66EF7EC3DF05F
:1090D00041E91200036A046A056A066A1200D9CFE0
:1090E000E9FFDACFEAFF120049E9E7CFD9FF120022
:1090F000E66EE66A0E0E025C120048E9E7CFD9FF81
:10910000120005EBF3FF06EBF4FF120088E90250B2
:109110000310041012008AE9045005100610120012
:1091200007EBE6FF08EBE6FF120000EBE6FF01EBC2
:10913000E6FF120002EBE6FFAEEF46F0BCD8A6D881
:10914000A8DE072A0822D1CBEFFF120096EC61F0CF
:1091500096EF46F0CEEC5FF0E9DD0B01120042E93C
:10916000FCC0D1FBFDC0D2FBFEC0D3FBFFC0D4FBD3
:109170000B012AEF47F0F2DD06EBE6FF120004EBED
:10918000E6FF05EBE6FF120096D82CEF60F009EB46
:10919000E9FF0AEBEAFF12000BEBE6FFD5EF46F022
:1091A00006EBE6FFF5DD19EC43F045E9F3EF47F098
:1091B000E552E5CFD8FBE5CFD7FBE5CFD6FBE7CF30
:1091C000D5FB1200E66EE66AE66A1200B6DD85E9B6
:1091D00048E864DE100E0B011200D1CBE6FFD2CBC3
:1091E000E6FFD3CBE6FFD4CBE6FF1200F2DD43DF90
:1091F000EF50120019EC43F045E9F3501200E9DD9D
:10920000EF5012009ADD83E91200E66EDACFE6FF36
:1092100012000B014CDED0DD67D7D1CBFCF0D2CBF6
:10922000FDF0D3CBFEF0120088DD87E9015002107B
:10923000031012000AEBE6FF0BEBE6FF0CEBE6FF78
:109240001200E5CFD2FBE7CFD1FB120076DD86EF2F
:1092500048F073DD8BEF48F0A8DD0FEBE6FF12005E
:10926000E66EE66A69DE5CDFA6EF48F0B50EE66EF4
:10927000050EA8DF96EF61F091DD96EC61F0AAEFA4
:1092800048F001EBE6FF56DF22EF48F02FEC60F0EC
:109290004DDD94EF47F073DF06EBE6FF90EF48F00B
:1092A00049DF38EF47F005EBE6FF06EBE6FF12007B
:1092B00037DFA8EF46F072DDA8EF46F00A0ECEEFDA
:0292C00046F076
:0E92C200CBEC52F044E80801CF51D01125E169
:1092D0001CEC54F00BE10B01010E516FF70EE66E22
:1092E000CC0EE66E000E4EEC53F017D0F6EC01F00B
:1092F000ED0EE66ECC0EE66E000E4EEC53F042EC38
:1093000052F0E3EC02F042E9E90EE66ECC0EE66EB6
:10931000000E4EEC53F014EC02F0D880000E000169
:109320008855030E8955CC0E8A55120E8B555AE27C
:10933000200E0B01CC1556E1170EE66E14EC53F01F
:109340003C0EE66EE66AE66AE66ADFEC53F04EEC47
:109350003EF042E9F3CFD5FBF4CFD6FB0B01D76B40
:10936000D86BD6AF02D0D769D869D5CBE6FFD6CBBC
:10937000E6FFD7CBE6FFD8CBE6FF96EC61F0E552EF
:10938000E5CFD4FBE5CFD3FBE5CFD2FBE7CFD1FBD5
:10939000880EE96E000EEA6EEE500B01D127EE50FA
:1093A000D223EE50D323EE50D42327EC53F0D4CB6A
:1093B000E6FFE66AE66AE66A5FEC53F0BAEC45F06F
:1093C00049E935EC53F0E60EE66ECC0EE66E000E83
:1093D000E66EF4EC52F019EC43F045E935EC53F04D
:1093E00052EC52F045E9E7CFD9FF12000801CF5106
:1093F000D01101E012001CEC54F008E10B01516B9C
:10940000E10EE66ECC0EE66E000E05D0DF0EE66EC7
:10941000CC0EE66E000E4EEF53F092EC53F086E960
:109420000B01CCB50CD0DFEC53F020EC54F042EC47
:1094300052F002EBE6FF57EC02F043E9D7DF5BEFB7
:1094400053F0CBEC52F00B01CCA502D0000E0ED0A5
:10945000DFEC52F042EC52F020EC54F05FEC53F0B1
:109460007AEC1CF042E947EC54F0010E5BEF53F04C
:109470000BEC53F042E80B01CCA502D0000E10D04B
:10948000DFEC52F08AEC52F020EC54F042EC52F057
:109490005FEC53F001EC1EF044E947EC54F0010E90
:1094A00086EF52F092EC53F084E90C0E0B01CC15D0
:1094B00012E1DFEC52F001EBE6FF02EBE6FF20ECFD
:1094C00054F000EBE6FF5FEC53F045EC0FF043E99E
:1094D00047EC54F08BDF5BEF53F0CBEC52F042E8FB
:1094E000E66A14EC53F0ADEC52F00DE0DFEC53F013
:1094F000ACEC53F0DFEC53F00FEC86F046E90009DA
:1095000002E1010E0AD00B01CCB306D02EEC53F0D1
:1095100042EC52F082DF45E9000E86EF52F00BEC90
:1095200053F042E8010EE66E5AEC54F035EC53F07D
:109530000050011010E0CEEC52F00DE0F4EC52F0CF
:10954000ACEC53F0F4EC52F00FEC86F046E9000975
:1095500002E1010E0AD00B01CCB306D02EEC53F081
:109560008AEC52F05ADF45E9000E86EF52F0CBEC60
:1095700052F042E80050011012E042EC52F0DCECF4
:1095800085F042E908010050F324CD6F0150F4202A
:10959000CE6F0050CD1907E10150CE1904E1000E45
:1095A000F36EF46A18D080EB03F081EB04F0ADECBD
:1095B00052F0200807E0ADEC52F004E0032A000E60
:1095C0000422F5D7ADEC52F0200803E108EC54F08A
:1095D000EF6A3AEC53F086EF52F0CBEC52F042E8EF
:1095E0000050011012E080EB03F081EB04F0ADECD1
:1095F00052F004E0032A000E0422F9D70801CD51ED
:10960000031807E1CE51041804E1000EF36EF46A6A
:109610001BD0032A000E042283EB00F084EB01F040
:10962000ADEC52F0200807E0ADEC52F004E0032A64
:10963000000E0422F5D7ADEC52F0200803E108EC4F
:1096400054F0EF6A3AEC53F086EF52F03FEC54F0EE
:10965000E66AD3EC53F00B01CCA502D0000E09D082
:10966000F6EC53F0CB0EE66ECC0EE66E000E72EC0E
:1096700053F086EF52F0F9EC53F0E66A2DEC8BF0E4
:1096800043E90B01CCA502D0000E0AD03FEC52F00A
:10969000E00EE66E0D0EE66E010E4EEC53F0010E7E
:1096A0005BEF53F03FEC54F0010EE66ED3EC53F059
:1096B0000B01CCA502D0000E09D0F6EC53F0B90E88
:1096C000E66ECC0EE66E000E72EC53F086EF52F0B2
:1096D0004AEC52F0A8EC52F0EF5008E13FEC52F0A7
:1096E000D00EE66E0D0EE66E010E11D042EC52F079
:1096F000010E8FEC52F00B01CCA502D0000E0AD067
:109700003FEC52F00D0EE66E0E0EE66E010E4EECC4
:1097100053F0010E5BEF53F06CEC53F0CCA502D08C
:10972000000E30D0DFEC52F03FEC52F0F9EC52F08A
:10973000300EE66E0F0EE66E010E83EC52F06DEC0D
:1097400045F049E94DEC52F002EC53F0B70EE66EED
:10975000CC0EE66E000E87EC53F0F9EC52F05E0E84
:10976000E66E0F0EE66E010E87EC53F002EC53F03E
:10977000B00EE66ECC0EE66E000E87EC53F052ECA7
:1097800052F0010E86EF52F0F9EC53F05ADE42E946
:109790005BEF53F04AEC52F047E80B01CCA502D046
:1097A000000E5FD03FEC52F0E5EC52F0096E076A14
:1097B000200E075C55E207EBE6FF5AEC54F0F3503D
:1097C0000A6EF4500B6E0AEBE9FF0BEBEAFFEF5069
:1097D00045E00750E66EE66AA60EE66ECC0EE66E33
:1097E000000E83EC52F06DEC43F047E9F3500C6E41
:1097F000F4500D6E0AEBE6FF0BEBE6FFA40EE66EEF
:10980000CC0EE66E000EE66E0CEBE6FF0DEBE6FF0F
:109810000DEC54F00C6EF4500D6E0B01000E0C5C50
:10982000D16F070E0D58D151086E09500824D16F21
:10983000D26BD23511E2D151A008000ED2550CE204
:10984000D5DD140EE66EF7EC3DF041E93FEC52F049
:10985000E5EC52F00824096E52EC52F0072AA8D722
:10986000010E48E9E7CFD9FF12005EEC54F0020E7A
:10987000076E200E075C11E2005001100EE097EC1D
:1098800053F006E1BFEC52F003E197EC52F002D046
:1098900042EC52F02CEC54F0ECD73FEC52F02F0E8F
:1098A000E66E0E0EE66E010E4EEC53F09FDDD9EC27
:1098B0006AF01CEC54F003E0400E12EC54F0000E81
:1098C000D5EF52F05EEC54F0076A200E075C11E20F
:1098D000005001100EE097EC53F006E1BFEC52F09F
:1098E00003E197EC52F002D042EC52F02CEC54F031
:1098F000ECD71CEC54F004E0E66A41EC04F041E9DA
:10990000000ED5EF52F0CBEC52F00E0E57EC52F0A9
:10991000940EE66ECC0EE66E000EE66E42EC52F051
:109920001AEC53F0B5EC53F0E66E42EC52F01AEC40
:1099300053F03AEC53F05BEF53F06CEC53F0CCA5E2
:1099400002D0000E29D03FEC52F0800EE66ECC0E15
:10995000E66E000E59EC53F0080E57EC52F0720E02
:10996000E66ECC0EE66E000E44EC53F0020E57ECA1
:1099700052F0680EE66ECC0EE66E000E44EC53F02C
:10998000030E57EC52F0560EE66ECC0EE66E000E4D
:1099900044EC53F07FEC53F086EF52F0D6EC53F0EA
:1099A000080E56EC53F011E042EC52F0020E56EC69
:1099B00053F00BE042EC52F0030E56EC53F005E08E
:1099C00042EC52F00E0E8FEC52F0D9EC6AF053ECF0
:1099D00053F0B3DFD1EC52F002E0A1EC52F00750AB
:1099E000D5EF52F06CEC53F0CCA502D0000E0BD0AA
:1099F0003FEC52F04D0EE66ECC0EE66E000E59ECCA
:109A000053F07FEC53F086EF52F05EEC54F097EC9D
:109A100053F003E1A8EC52F0EF6A42EC52F00E0E64
:109A20008FEC52F0D9EC6AF053EC53F0DBDFD1EC61
:109A300052F002E0A1EC52F00750D5EF52F06CEC7E
:109A400053F0CCA502D0000E66D03FEC52F0470E8A
:109A5000E66ECC0EE66E000E59EC53F0050E57EC98
:109A600052F03F0EE66ECC0EE66E000E44EC53F064
:109A7000060E57EC52F0360EE66ECC0EE66E000E79
:109A800044EC53F0070E24EC54F0160E57EC52F051
:109A9000210EE66ECC0EE66E000E44EC53F0CE0EB8
:109AA000E66E000EE66E190EE66ECC0EE66E000E49
:109AB00044EC53F0A1EC90F0000906E1070EE66ECD
:109AC000CC0EE66E000E22D00B01505106E0E40EE3
:109AD000E66ECB0EE66E000E19D0200E0601C85DB4
:109AE00006E1C10EE66ECB0EE66E000E0FD0C85139
:109AF000E66EE66AA20EE66ECB0EE66E000EE4ECB3
:109B000053F0A00EE66ECB0EE66E000E48EC53F05E
:109B100052EC52F0010E86EF52F0D6EC53F0050EE7
:109B200056EC53F02EE097EC53F006E1BFEC52F008
:109B300003E197EC52F002D042EC52F0060E56ECE4
:109B400053F00EE097EC53F006E1BFEC52F003E166
:109B500097EC52F002D042EC52F0070E8FEC52F02C
:109B60004AEC54F00EE097EC53F006E1BFEC52F0F3
:109B700003E197EC52F002D042EC52F0160E8FEC5B
:109B800052F053EC53F05BDFD1EC52F002E0A1EC69
:109B900052F00750D5EF52F06CEC53F0CCA502D048
:109BA000000E30D03FEC52F0960EE66ECB0EE66E15
:109BB000000E4EEC53F00D0EE66ED3EC53F007EBB7
:109BC000E9FF08EBEAFFEF5006E18D0EE66ECB0EE3
:109BD000E66E000E0AD032EC54F0E3EC02F042E9FB
:109BE0008A0EE66ECB0EE66E000E4EEC53F0CE0EF5
:109BF000E66E000EE66E800EE66ECB0EE66E000E92
:109C000072EC53F086EF52F03FEC54F0005001102C
:109C100007E1086AD950080FE66EDACFE6FF02D0F6
:109C200042EC52F00D0E8FEC52F053EC53F0B4DFD7
:109C3000D1EC52F002E0A1EC52F0075086EF52F066
:109C40006CEC53F0CCA502D0000E23D03FEC52F0C8
:109C5000780EE66ECB0EE66E000E59EC53F0040E55
:109C600057EC52F0710EE66ECB0EE66E000E44EC31
:109C700053F0090E24EC54F00A0E57EC52F0640E27
:109C8000E66ECB0EE66E000E44EC53F052EC52F052
:109C9000010E86EF52F0D6EC53F0040E56EC53F062
:109CA0000AE042EC52F0090E56EC53F004E0EADB15
:109CB0000A0E8FEC52F053EC53F0C2DFD1EC52F0AD
:109CC00002E0A1EC52F00750D5EF52F06CEC53F0EB
:109CD000CCA502D0000EB3D0D2DB5E0EE66ECB0E6A
:109CE000E66E000E59EC53F00701F651E66EE66A97
:109CF000530EE66ECB0EE66E000E4AEC53F00701F3
:109D0000F751E66EE66A480EE66ECB0EE66E000E82
:109D10004AEC53F00601C851E66EE66A390EE66E6B
:109D2000CB0EE66E000EE4EC53F00001CC510008BF
:109D30001EE2010EE66EE66ACCC0E6FFE66AE66A5F
:109D4000E66A2D0EE66ECB0EE66E000EE8EC53F0E2
:109D5000010EE66EE66ACDC0E6FFE66AE66AE66AEE
:109D6000270EE66ECB0EE66E000EE8EC53F00B010C
:109D7000CE51E66EE66A1C0EE66ECB0EE66E000E67
:109D80004AEC53F00B01CF5158E0120EE66ECB0EA9
:109D9000E66E000E48EC53F00B01CFA107D00D0E7C
:109DA000E66ECB0EE66E000E48EC53F00B01CFA32F
:109DB00007D0080EE66ECB0EE66E000E48EC53F0B0
:109DC0000B01CFA507D0040EE66ECB0EE66E000E9B
:109DD00048EC53F00B01CFA707D0000EE66ECB0E78
:109DE000E66E000E48EC53F00B01CFA907D0FC0E35
:109DF000E66ECA0EE66E000E48EC53F00B01CFABD8
:109E000007D0F40EE66ECA0EE66E000E48EC53F074
:109E10000B01CFAD07D0EC0EE66ECA0EE66E000E5B
:109E200048EC53F00B01D051E66EE66AE80EE66EA0
:109E3000CA0EE66E000E4AEC53F034DB010E66D318
:109E400029DB43E80B01CCA502D0000E28D017DB9C
:109E5000DE0EE66ECA0EE66E000E4EEC53F0076A9A
:109E6000100E075C1BE2B9DBEF5016E00750E66E00
:109E7000E66ADA0EE66ECA0EE66E000E44DB8DEC84
:109E800053F0ABDBEF50E66EE66AA40EE66ECC0E46
:109E9000E66E000E49DB06DB072AE2D7010E44E935
:109EA000E7CFD9FF12005EEC54F00050011002E140
:109EB000000E2CD0FCEC53F0076EE4DA64EC53F0A7
:109EC000D89023E2100E075C20E2005001101DE044
:109ED000FCEC53F0E66E81DBE552E750EF6E080EC6
:109EE000075C05E3CFDA080E075C180F18DB0F0ECE
:109EF000075C02E1D9EC6AF0C2DA490EE66E0E0E9A
:109F0000E66E010ECBDB010E01D0000E4ED3E7DB77
:109F100003E0B8DA180ED2DAB2DA5F0EE66E0E0E91
:109F2000E66E010ED4D2DBDB03E0ACDA140EC6DA47
:109F3000A6DA720EE66E0E0EE66E010EC8D2CFDB0A
:109F400003E0A0DA160EBADA9ADA890EE66E0E0E81
:109F5000E66E010EBCD2C3DB03E094DA150EAEDA76
:109F60008EDAA20EE66E0E0EE66E010EB0D2B7DBF2
:109F700003E088DA170EA2DA82DAB70EE66E0E0E6A
:109F8000E66E010EA4D23FEC54F00050011002E145
:109F9000000E22D077DACAEC86F042E9F7DA14E054
:109FA00071DA19EC3EF042E9300F076E086AD950B9
:109FB000070FE66EDACFE6FF0A0EFBDA4AEC54F042
:109FC00003E060DA0F0EF5DA5ADAD30EE66E0E0E03
:109FD000E66E010E63DB010E99D281DB05E0000E17
:109FE000E66EE66A0B0E6ADA0601FC6B48DAF00EE2
:109FF000E66E0E0EE66E010E6AD271DB05E0000E13
:10A00000E66EE66A0C0E5ADA06011E0EFC6F37DAAF
:10A01000070EE66E0F0EE66E010E59D260DB05E00C
:10A02000000EE66EE66A190E49DA29DA1D0EE66EB2
:10A030000F0EE66E010E4BD22DDA43E8010E076ECD
:10A04000020E076E1CDA0E0EF66E000EF76E000E94
:10A05000E5DAC20EE66ECA0EE66E000E54DA5DDB7D
:10A060000F0EF66E000EF76E000E89DB100EF66E08
:10A07000000EF76E000E83DB0E0E19DABE0EE66ED2
:10A08000CA0EE66E000E6CDA0001105111111211A9
:10A090000EE010C0E6FF11C0E6FF12C0E6FF08EBBD
:10A0A000E6FF09EBE6FF19EC43F045E9F6DB075064
:10A0B000E66EE66ABB0EE66ECA0EE66E000E34DA97
:10A0C000B60EE66ECA0EE66E000EE66EBE0EE66ECA
:10A0D000CA0EE66E000E6DDB59EC43F048E9DDDB9D
:10A0E00044DB3EDA930EE66E000EE66EAE0EE66ED2
:10A0F000CA0EE66E000E34DAD5D9010E44E9E7CF78
:10A10000D9FF1200BCDB040E8DDB000EFFD1C2D9DB
:10A11000B9D9ADDB38EC4AF044E9CDD2B0DB91C01F
:10A12000E6FF92C0E6FF930EE66ECA0EE66E000EE4
:10A13000EAD96DEC43F047E9B0D9A5C0E6FFA6C067
:10A14000E6FF880EE66ECA0EE66E000EA3DAA7C022
:10A15000E6FFA8C0E6FF7B0EE66ECA0EE66E000EB6
:10A1600099DAA9C0E6FFAAC0E6FF6C0EE66ECA0E39
:10A17000E66E000E8FDAABC0E6FFACC0E6FF5D0E08
:10A18000E66ECA0EE66E000E85DA5B0EE66ECA0E4D
:10A19000E66E000E7DDA0001C35103E00001C451F8
:10A1A00006E14F0EE66ECA0EE66E000E71DA67D952
:10A1B00079D9010EABD1B6DA86E90450330A0AE048
:10A1C000010A05E0030A18E1BFDA08E009D01ADB4A
:10A1D00013E104D017DB10E1B7DA02E1000E0DD075
:10A1E000B7D94DDAEDEC4AF042E9F4CFD2FBB0D961
:10A1F000F3CFEEFFD2CBEDFF010E5DD20CDA46E8D5
:10A2000080EB05F081EB06F0C9D918E0C7D920082A
:10A2100015E0C4D960080EE20ADBEFCFD1FB7B0E5C
:10A220000B01D15D07E2BAD9E00FE66E00DBE55223
:10A23000E750EF6E052A000E0622E6D7AFD92008B8
:10A2400003E1052A000E0622076AA1DAF55001E1B2
:10A25000A0D0740ED76F0F0ED86F010ED96F6BDAC6
:10A26000E5CFDCFBE5CFDBFBE7CFDAFB0B01D7511A
:10A27000DA25D46FD851DB21D56FD951DC21D66FC7
:10A28000D4CBE6FFD5CBE6FFE66EEAEC85F043E9FA
:10A29000FCC0D1FBFDC0D2FBFEC0D3FB0B01D1073C
:10A2A000000ED25BD35BD1CBE6FFD2CBE6FF740EC0
:10A2B000E06F0F0EE16F010EE26F3DDAE5CFE5FBD7
:10A2C000E5CFE4FBE7CFE3FB0B01E051E325DD6FD6
:10A2D000E151E421DE6FE251E521DF6FDD2B000E5D
:10A2E000DE23DF23DDCBE6FFDECBE6FFDFCBE6FFC1
:10A2F000C9D8B4EC84F047E9000949E1086A74D987
:10A30000B7EC4AF042E9F350096EF4500A6ED950A6
:10A31000090FE66EDACFE6FFFDD839DAF5CFE6FFB2
:10A320004ADF45E900094BE000013A513B113C117D
:10A3300006E0DFD9010EE66E82D900093AE1075046
:10A34000030DF3CFE9FFF4CFEAFF000EE9260A0E72
:10A35000EA22EECFD1FBEECFD2FBEFCFD3FBC9D9B0
:10A36000D3CBFBFFD2CBFAFF0B01D151140046E94E
:10A37000086E08500AE000013A513B113C1103E01D
:10A38000B8D9E66A5CD9F6EC49F0085019D0072A2A
:10A390005CD700013D513E113F110DE025D96CDA2B
:10A3A0003FC0FBFF3EC0FAFF3D51140046E90009E3
:10A3B00002E0010E05D060DABEEC1BF044E9000EAD
:10A3C00047E9E7CFD9FF120087D9CCA502D0000E0C
:10A3D00055D055D8450EE66ECA0EE66E000E5ED913
:10A3E000076A086AC3D807EBD7FB08EBD8FBD96B21
:10A3F000D8BFD969D7CBE6FFD8CBE6FFD9CBE6FFEC
:10A4000069D8F5503AE0430EE66ECA0EE66E000ECD
:10A4100045D90B01740ED46F0F0ED56F010ED66F98
:10A4200041DA07EBDAFB08EBDBFBDC6BDBBFDC695B
:10A43000DACBE6FFDBCBE6FFDCCBE6FF36EC61F008
:10A44000E552E5CFD9FBE5CFD8FBE7CFD7FB0B0132
:10A45000D451D725D16FD551D821D26FD651D9211A
:10A46000D36FD12B000ED223D323F1D857EC02F0B7
:10A4700043E9072A000E0822B5D7010E47D0F7D9C5
:10A4800020EF54F000EBE6FF01EBE6FF1200E66E72
:10A4900032EF54F047D987E91200F350076EF450B9
:10A4A000086E12000CD9E3EC02F042E91200E66EED
:10A4B00001DAF3CFE6FFF4CFE6FF12008FD9375170
:10A4C000140045E9120000D9005001101200E6D82E
:10A4D000010EF1D036EC61F0E552E5CFD6FBE5CFC9
:10A4E000D5FBE7CFD4FB0B01D151D425F36ED2516C
:10A4F000D521F46ED351D621F86EF4CFF7FFF3CF08
:10A50000F6FF08001200E66E5FEF53F043E9E7CF75
:10A51000D9FF120002EBE6FF03EBE6FF1200E66E46
:10A520002DEC8BF043E9120044D98DEF53F00B0171
:10A530000028D16F000E0120D26FD1CBE6FFE66E6E
:10A5400012000A0E0601CA6FCB6B410E12EF54F0D7
:10A5500000EBE9FF01EBEAFF12005AD9EF501200BD
:10A5600028D95BD9086EF450096E12000B01740EE5
:10A57000D16F0F0ED26F010ED36F52EF54F000283F
:10A58000E96E000E0120EA6EEF5012000001375113
:10A59000381139111200C6D883E9120048D9EF509A
:10A5A000120046E9076E1CEF54F042E9E7CFD9FFED
:10A5B000120014D900013751140045E91200020EAF
:10A5C000E66EF7EC3DF041E91200A80EE66ECC0E07
:10A5D000E66E000E63D8070E12000750EA6ABE0F3F
:10A5E000E96E0B0EEA22120005EBE6FF06EBE6FF32
:10A5F00012009ACBE6FF9BCBE6FF9CCBE6FF9DCB00
:10A60000E6FF12009ECBE6FF9FCBE6FFA0CBE6FF66
:10A61000A1CBE6FF120086D885E91200F86E08008B
:10A62000F550E66EE66A120045D9F350036EF45019
:10A63000046E1200F2D8006EF450016E12003CC09D
:10A64000FBFF3BC0FAFF3A51140047E91200D1CB9F
:10A65000E6FFD2CBE6FFD3CBE6FF1200BE0EE66EDE
:10A660000D0EE66E010EE66E1200F350056EF4500C
:10A67000066E120000EBF3FF01EBF4FF1200EECFC9
:10A68000E6FFEECFE6FF120002DF4DEC43F00FD104
:10A69000FEDEF8D0FCDE6DEC43F009D1E66E57EC3F
:10A6A00002F043E91200E8D837EF54F038DF4AEF00
:10A6B00054F029DFE7D041E9E7CFD9FF1200000EBF
:10A6C000E66E070EE66E1200EDEC4AF042E9F3503A
:10A6D000006EF450016E1200D2D80B011200DADEC7
:10A6E000C6EF52F010DF4DEC43F047E9DBDE010E20
:10A6F000120009EBE6FF0AEBE6FF3CEF54F0B2D89C
:10A7000083EC4CF042E9C9DECDDE010E1200BFDE63
:10A710006DEC45F049E94DEF52F06DEC43F047E93F
:10A720004DEF54F0D9CFE6FFE1CFD9FF120010DF93
:10A73000EF502D081200B6D807EBE6FFE66AE66A8E
:10A7400036EC61F0E552120003DF99DFE3DE8FECB7
:10A750004AF044E900091200DCEC85F042E9F3CF4D
:10A76000E6FFF4CFE6FF42EF52F0950EE66E0B0ED9
:10A77000E66E880EE66ECC0EE66E000E12004EDF20
:10A78000C00EE66ECA0EE66E000E94EF52F0EEDEDC
:10A7900007EBE6FFE66AE66A6AEF52F0DEEC42F0AB
:10A7A00042E952EF52F086D84DEF52F087D842EF8F
:10A7B00052F0E66E08EBE6FF09EBE6FF120003EB52
:10A7C000E6FF04EBE6FF120062DEF0EC43F06FD030
:10A7D0005EDE7AEC44F04BE94DEF52F0E66EE66A4D
:10A7E000E66A39C0FBFF38C0FAFF120048DE32EFDC
:10A7F00054F050DE37EF54F045DE09EC7FF042E9CB
:10A80000F350120087DE6DEC4AF042E900091200B5
:10A8100003EBE9FF04EBEAFF12004DEC43F047E9DC
:10A82000F3501200E66E41EC04F041E9120005EB32
:10A83000E9FF06EBEAFF12007F0E0601C85D120079
:10A8400061EC49F042E9120032DE290EE66ECC0ED0
:10A85000E66E000E44EF53F00750072A60DE12DE6A
:10A8600064EF53F007EBE6FF08EBE6FF120004EBA2
:10A87000E6FF05EBE6FF120005DE8AEF52F00ADE86
:10A8800042E8120019EC43F045E94DEF52F017DFB2
:10A89000CEEF53F0F7DD63EF52F0F350086EF45053
:10A8A000096E1200100EE66EE66AE66A120047E9CB
:10A8B0004DEF52F018EC8BF041E91200EBDD41E86E
:02A8C000120084
:0EA8C200FAEC5BF083E901340050011802E665
:10A8D0000150005C02E2015001D000505EEF5CF0DC
:10A8E000FAEC5BF085E903340150031804E60250EA
:10A8F000005C0350015805E202EB24FB03EB25FB4F
:10A9000004D000EB24FB01EB25FB24CBF3FF25CB8C
:10A91000F4FF5EEF5CF0FAEC5BF086E943E8460E8C
:10A92000066E0F0E076E0B01CD5144E00250080871
:10A9300041E30F0140B7FDD7406B070E0B01031435
:10A94000286F296B050E28CB26FB29CB27FB000A95
:10A9500006E00B01D89026372737E804FBE126CB29
:10A9600042FF0B0103EB26FB04EB27FB030ED89001
:10A9700027332633E804FBE126CB41FF086A025067
:10A98000085C13E208500024E96E000E0120EA6E14
:10A99000EF50E66E08500624E96E000E0720EA6EBE
:10A9A000E552E750EF6E082AEAD702EB45FF0F01A8
:10A9B000080E406F3DEF5CF093EC5CF043E8016AF9
:10A9C000040E015C0BE22BEC5CF0EE52EF6A02EB42
:10A9D000E9FF03EBEAFFEF6A012AF2D73DEF5CF0F3
:10A9E000FAEC5BF084E943E802500D0D6C0EF324A1
:10A9F000056E0A0EF420066E41EC5CF0EE52EF504C
:10AA000002E0015038E041EC5CF0020E7AEC5CF0C0
:10AA100002C0EEFF03C0EDFF41EC5CF0040E7AECE7
:10AA20005CF005C0EFFF046A00010551045C18E208
:10AA3000045062EC5CF041EC5CF0050E7AEC5CF0EA
:10AA4000E9CF2AFBEACF2BFB04500B01EA6AE92489
:10AA5000E96E2B51EA22E552E750EF6E042AE4D763
:10AA600041EC5CF0EE52010EEF6E005004E041EC60
:10AA70005CF0010EEF6E3DEF5CF093EC5CF049E8AA
:10AA8000056A046A040E045C1DE204500D0D6C0E90
:10AA9000F324066E0A0EF420076E05500FE106EB54
:10AAA000E9FF07EBEAFFEF5007E006EBE9FF07EBF2
:10AAB000EAFFEE52EF5002E1000E01D0010E056EEA
:10AAC000042AE0D7055002E1000E7AD032EC12F0F1
:10AAD000046A040E045C73E204500D0D6C0EF32442
:10AAE000086E0A0EF420096E26EC5CF0EF5065E06B
:10AAF00026EC5CF0EE52EF5060E0C50EE66ECF0E35
:10AB0000E66E000E52EC5CF019EC43F045E946ECC1
:10AB10005CF00450E66EE66A38EC5CF06DEC43F0F5
:10AB200047E946EC5CF0BD0EE66ECF0EE66E000E19
:10AB3000E66E96EC5CF019EC43F045E946EC5CF00F
:10AB400026EC5CF0020E7AEC5CF0EECFE6FFEECF86
:10AB5000E6FF38EC5CF0F0EC43F047E946EC5CF0E3
:10AB6000036A26EC5CF0040E7AEC5CF0EF50035CB8
:10AB70001BE226EC5CF0050E7AEC5CF0E9CF2CFBD6
:10AB8000EACF2DFB03500B01EA6AE924E96E2D514F
:10AB9000EA22EFCFE6FF38EC5CF01EEC44F046E929
:10ABA00046EC5CF0032ADDD76FEC12F026EC5CF08B
:10ABB000EF6A26EC5CF0EE52EF6A042A8AD7010EA7
:10ABC0004AE9E7CFD9FF120093EC5CF043E80001BB
:10ABD0000951016E09C02FFB0B012E6B00010A51B8
:10ABE0000B012E25026E000E2F21036E0D0E0001AB
:10ABF000511901E152513AE0020E511950E15251FE
:10AC00004EE1016A00010551015C1FE2015062EC56
:10AC10005CF00551F36EF46AF3500001565D0B01D0
:10AC20002E6FF450000157590B012F6F0150EA6A43
:10AC30002E25E96E2F51EA22930EE926000EEA2214
:10AC4000E552E750EF6E012ADDD70001545155114E
:10AC500026E101500001EA6A5625E96E5751EA22C1
:10AC6000930EE926000EEA22EF6A19D04B0E00017E
:10AC70000F5D03E101EB77F012D001EBE6FFE66A2E
:10AC8000E66AE66ADDEC3EF044E9FCC02EFBFDC05E
:10AC90002FFBFEC030FBFFC031FBFCC077F0010E84
:10ACA0003DEF5CF0ADEC5CF0005002E0010E01D035
:10ACB000000E0001719FE8B0718F005002E0010E9C
:10ACC00001D0000E00017391E8B07381005002E0E2
:10ACD000000E01D0010E0001719DE8B0718D005091
:10ACE00015E000018C518D118E118F110FE08C6BCE
:10ACF0008D6B8E6B8F6B15EC5CF00001719571990B
:10AD000071970001666B0001676B17D0005015E169
:10AD100000018C518D118E118F110FE188C08CF0C4
:10AD200089C08DF08AC08EF08BC08FF08C07000E2A
:10AD30008D5B8E5B8F5B15EC5CF05EEF5CF0ADECD9
:10AD40005CF00050040A56E0070A0DE0010A0BE02F
:10AD5000030A02E0010A58E1000171990001666BE3
:10AD60000001676B51D0000171890001010E666F0F
:10AD70000001030E676F0A01AC3503E30001626B4B
:10AD800018D0020EE66EE66AABCA34FBACCA35FBDD
:10AD90000B01342B000E352334CBE6FF35CBE6FF19
:10ADA0004AEC5FF0E552E5CF33FBE7CF32FB32CB25
:10ADB00062F0020EE66EE66AADCA32FBAECA33FB43
:10ADC0000B01322B000E332332CBE6FF33CBE6FFF1
:10ADD00092EC5FF0E552E5CF61F0E7CF60F0005014
:10ADE0000A01AA5D11E00001646B656B00016A6BEA
:10ADF0006B6B0AD00001626B000171990001040EB7
:10AE0000666F0001030E676F020E005C08E0030E20
:10AE1000005C05E00001626B0001606B616B00503B
:10AE20000A01AA5D02E015EC5CF000EBAAFA5EEF05
:10AE30005CF093EC5CF048E8300E016E010E026E9F
:10AE4000036A046A056A066A076A086A0701F0511C
:10AE5000030A18E0010A06E0030A39E10CC0F1F721
:10AE6000020E05D008C0F2F70BC0F3F7030EF06F27
:10AE700058EC5CF0080EE66E9B0EE66E070E85EC55
:10AE80005CF025D007C0F4F7F1C7A9F00001AA6B68
:10AE9000A9BFAA69F2C736FB0B01376B36BF37690A
:10AEA00005EC5CF0F3C736FB0B01376B36BF376937
:10AEB00005EC5CF0F4C736FB0B01376B36BF376926
:10AEC00005EC5CF000010A0EC46F0701F06B49E964
:10AED000E7CFD9FF120093EC5CF045E80A010A0EB7
:10AEE000A06FC00E0001021908E1050E031905E16B
:10AEF000E66AE66AE66A74DD43E9BB0E0001021900
:10AF000002E1070E031901E1E4D1C00E021902E1CA
:10AF1000050E031901E1D1D1BF0E021902E1050EA0
:10AF2000031901E183D1BC0E021902E1050E0319D8
:10AF300001E111D1B90E021902E1050E031901E177
:10AF4000FBD05A0E021902E1050E031901E1C6D029
:10AF50004C0E021902E1050E031901E191D04B0ECE
:10AF6000021902E1050E031966E0840E021902E1DE
:10AF7000020E031946E0DB0E021901E0ABD1010E0F
:10AF8000031901E0A7D1000106511CEC5CF0D89038
:10AF900038373937E00E00010715E00BE838E84094
:10AFA0000B0138110A01AB6F39CBACFAAC51040B71
:10AFB00002E0F80EAC13000108511CEC5CF0060E28
:10AFC0003A6FC00E000109153ACBE7FFE75204E0E3
:10AFD000E8427F0BE706FCE10B0138110A01AD6F77
:10AFE00039CBAEFAE8CF6FF039CB70F00001050E27
:10AFF0007003F3CF70F06F03F3CF6FF0F45070274E
:10B0000069D10A010A0EA16F010EE66E4BDE41E91D
:10B0100000010A51016E026A81EB02F0016A0B51D4
:10B0200001125C0EE66EE66A96EC5CF06AEC5CF08F
:10B0300038CB77F04FD10A0E0001075D11E0480EC2
:10B04000075D0EE04B0E075D0BE0710E075D08E03B
:10B05000760E075D05E0780E075D02E0000E01D078
:10B06000010E036E00017551800B01E0010E035CBF
:10B0700001E130D10350759FE8B0758FD6DB2AD13E
:10B08000FF0E00010C5D01E125D10C510001916F13
:10B09000926B380E915F000E925B660EE66EE66E66
:10B0A000E60EE66E3F0EE66E91C038FB92C039FBAD
:10B0B0000B01200E385F000E395B8AEC5CF0FFEC70
:10B0C0005DF072EC60F07EEC5EF0E552E5CF92F060
:10B0D000E7CF91F000010A0EC36FFCD000010751C9
:10B0E000FC0BE842E8420001A56FA66B0001085185
:10B0F000FC0BE842E8420701F56F00010B51FC0B25
:10B10000E842E8420001A76FA86BF5C738FB0B01C6
:10B11000396B38BF39698AEC5CF0A5C0E6FFA6C080
:10B12000E6FF70EC54F044E9F3CFA5F0F4CFA6F0BD
:10B1300000010A0EC46FCED0070E000106150B01E8
:10B14000396F386B000107510B0138110001DA6FBC
:10B1500039CBDBF0BFD0000106516EDB060E3A6F33
:10B16000C00E000107153ACBE7FFE75204E0E842C2
:10B170007F0BE706FCE10B013811046E3951056EB7
:10B18000FF0E041804E1030E051801E1A3D004EB3F
:10B19000A6FA05EBA7FAA8CAE6FFA9CAE6FFA6CA5F
:10B1A0003CFBA7CA3DFB640E3D03F3CF3DFB3C03D4
:10B1B000F3CF3CFBF4503D27020EE66EE66AA8CAC8
:10B1C000E6FFA9CAE6FF92EC5FF0E552E5CF3FFB50
:10B1D000E7CF3EFB0B013C513E253A6F3D513F21ED
:10B1E0003B6F3ACBE6FFE66E75DB38CB78F0190E95
:10B1F000E66E010EE66EA6CA38FBA7CA39FB0B0144
:10B20000540E3903F3CF39FB3803F3CF38FBF45036
:10B2100039278C0E3827000E39237CDB92EC5FF047
:10B22000E552E5CF7AF0E7CF79F054D0B00E0001C7
:10B230000A5D0AE10001020E6C6F0001780E636F77
:10B2400000017185718720D00001010E6C6F050E21
:10B25000E66E08C0E6FF1CEC5FF041E9E750000134
:10B26000636F635102E1000E01D0010E0001719580
:10B27000E8B071850001635102E1000E01D0010EBA
:10B2800000017197E8B0718700010A51400A10E08F
:10B29000200A0CE0D00A08E0800A04E0180A1AE14B
:10B2A000E66A08D0010E05D0030E03D0020E01D0CD
:10B2B000040EE66E44DD41E90DD0400E0001065D4E
:10B2C00009E10851FE0BE842D80F0001A96FAA6BF3
:10B2D00001D0AFDD010E46E9E7CFD9FF12003DDB1B
:10B2E00041E80050020A08E0030A04E0010A0BE109
:10B2F0004E0E03D0560E01D0660E026EF3DA6E0EBD
:10B30000E66E050E02DB0BD30A01A35100080DE225
:10B31000A307A2CAE6FFE3DF41E90E0E0A01A35D1F
:10B3200004E1E66ACCEC90F041E9010C16DB42E85E
:10B330000701EF5103E00A01A05102E1005038D0AB
:10B34000A30EE66ECF0EE66E000EACDA19EC43F0FB
:10B3500045E9F9DAABCAE6FFACCAE6FF50DAADCA96
:10B36000E6FFAECAE6FF4BDA00017751E66EE66A09
:10B3700046DAA6CAE6FFA7CAE6FF41DA91C0E6FFB1
:10B3800033DAF1C7E6FF30DAF2C7E6FF2DDAF3C7AA
:10B39000E6FF2ADAF4C7E6FF27DA005002E132ECD2
:10B3A00012F06FEC12F04EEC12F00701EF6B010E91
:10B3B00043E9E7CFD9FF1200B6DA41E8200E0601D3
:10B3C000C85D06E10B01505103E00B01515102E051
:10B3D000010E0CD03DEC55F0016E01EBE6FFA6DF4F
:10B3E00041E9016E015002E04EEC12F098D29BDA76
:10B3F00044E8900EE66ECF0EE66E000EE66E58DA6A
:10B4000019EC43F045E954DA150EE66E2DEC8BF09D
:10B4100043E945E9E7CFD9FF120085DA44E80A019C
:10B42000190EA86F010EA96F150EE66E18EC8BF0C1
:10B4300041E92CDA015002100BE078DA09EC7FF0D8
:10B4400042E9F350036EF450046E0350041002E11D
:10B45000CEDF04D003EBA8FA04EBA9FA45E9E7CF65
:10B46000D9FF12007ADA41E80B01CD5102E1000E5A
:10B4700020D0010EE66ECCEC90F041E9026A32DA9F
:10B480008C0EE66E060E41DA0A0EE66EDFEC3DF03B
:10B4900041E900EBE6FF23DF41E900EBA2FA0A01F4
:10B4A000180EA36F005004E1580EA46F020EA56F92
:10B4B000020E35D20001882B000E89238A238B23AC
:10B4C0000A01A051000801E2A007A151000801E211
:10B4D000A107000E0001E76EC41902E7C43502D0CF
:10B4E000C451E75C01E2C407000E0001E76EC31916
:10B4F00002E7C33502D0C351E75C01E2C3070A018A
:10B50000A4510008000EA55503E2A407000EA55B98
:10B51000A15101E1F3D90A01A05103E1EFD90001E2
:10B52000759F0A01010EA41906E1A55104E1010E5F
:10B53000E66E98DF41E91200F6D948E8020E016E86
:10B54000210E026E040E036E046A056A066A076A1B
:10B55000086A0A01A051050802E3010E07D0A451B0
:10B560000008000EA55501E260D9010E49E9E7CFB8
:10B57000D9FF1200D8D943E8016A040E015C05E244
:10B580006AD9010EEF6E012AF8D70701010EEF6F9D
:10B5900074D130D986E943E8180E021828E1035027
:10B5A00026E1D6D909EC7FF042E9F350076EF4505A
:10B5B000086E0750081009E11A0E026E036A8E0E1B
:10B5C000E66ECF0EE66E000E0DD0010E07180FE1ED
:10B5D00008500DE11A0E026E036A8C0EE66ECF0E55
:10B5E000E66E000EE66EB4D9C3EC85F045E902EBD9
:10B5F000F3FF03EBF4FF1A0EF31801E1F45009E036
:10B600000B0EF31801E1F45002E0000E4BD0020ED5
:10B6100011D08E0EE66ECF0EE66E000E3CD902E122
:10B62000E66A09D08C0EE66ECF0EE66E000E33D9B8
:10B6300005E1010EE66E16DF41E901D0010E066E4E
:10B640000650020A10E0030A08E0010A26E1EA0EA9
:10B65000E66E220EE66E010E0BD0D80EE66E220EBE
:10B66000E66E010E05D0D50EE66E220EE66E010ED8
:10B67000E66E02EBE6FF03EBE6FFCE0EE66E220E71
:10B68000E66E010E0FD96DEC43F047E9F3CFE6FF0C
:10B69000F4CFE6FF19EC43F045E9045002E06FEC0B
:10B6A00012F0010EEAD03FD942E80B014E0E956F21
:10B6B0004C0E966F976B986B996B0001C7690001F0
:10B6C000886B896B8A6B8B6B0A01A36BA6DE00010A
:10B6D000020EEF6FE8CF78F0E66ACCEC90F041E92B
:10B6E000DCEC54F0900E6F6E6EAEFED7606A0F0108
:10B6F000196B1869016BF30E006F506B1D6B1C6B9F
:10B70000010E706ED20E716E020E726E200E736E8E
:10B710000B01CD51000802E26F6A02D0600E6F6E1D
:10B720000A010A0EA06F0001A60E106F240E116F01
:10B73000010E126F0001B00E136F240E146F010E74
:10B74000156F0001C80E196FAB0E1A6F000E1B6F3C
:10B750000001D60E1C6FAE0E1D6F000E1E6F000195
:10B76000B80E346FB30E356F000E366F0001080E41
:10B77000316FB30E326F000E336F0001B40E1F6FC6
:10B78000B40E206F000E216F0001380E226FB50E2F
:10B79000236F000E246F0001740E256FB50E266F07
:10B7A000000E276F0001920E376FB50E386F000E36
:10B7B000396F0B01CD51000809E2BC0EE66E240E74
:10B7C000E66E010EE66E04EC68F043E9020EE66EEA
:10B7D00011EC68F041E90601EE81EE83EE85010E81
:10B7E00043E9E7CFD9FF1200A6D81EEC44F046E9A2
:10B7F000A3EF5CF0D9CFE6FFE1CFD9FF12009BD8D1
:10B80000F0EC43F047E9A3EF5CF036CBE6FF37CB33
:10B81000E6FFA9C0E6FFAAC0E6FF70EC54F044E9D9
:10B82000F3CFA9F0F4CFAAF01200020EE66EE66A9A
:10B83000A9EC03F042E912000B01386F396BD89084
:10B8400038373937D89038373937120008EBE9FFE5
:10B8500009EBEAFF120001500D0D6C0EF324026E8D
:10B860000A0EF420036E02EBE9FF03EBEAFF12007D
:10B87000E66AE66AE66A96EF5CF044E9E7CFD9FF4C
:10B88000120005EBE9FF06EBEAFF1200F350016E30
:10B89000F450026E1200E66E5BD88CEC85F045E940
:10B8A00000091200E66E000EE66E070EE66E12004C
:10B8B000D950010FE66EDACFE6FF120041E9E7CF7B
:10B8C000D9FF1200EA6A060FE96E000EEA22EF5075
:10B8D000E66E120092EC5FF0E552E5CF39FBE7CF60
:10B8E00038FB1200D950020FE66EDACFE6FF010EE8
:10B8F000E66E1200E926000EEA221200E66A52EC19
:10B9000056F041E90001776B1200E66E8BEC54F0C3
:10B9100045E9120038CBE6FF39CBE6FF120042E9D9
:10B92000E7CFD9FF120066DF81E9120001EBE6FFE5
:10B9300002EBE6FF1200E66AE66AE66A02EBE6FF61
:10B9400003EBE6FF1200F350026EF450036E120098
:10B9500000EBE6FF01EBE6FF12004CDF82E912008C
:10B96000D88801D0D8984AE8D9CFE6FFDACFE6FFE9
:10B97000E1CFD9FFE2CFDAFF94E9D8B8037E086AB5
:10B98000B2EC5DF0CAEC5DF008B696EF5DF008A28F
:10B990000AD008AA03D008BE96EF5DF008A4A2EF73
:10B9A0005DF09FEF5DF008AA05D008ACA2EF5DF056
:10B9B0009FEF5DF008A00AD008A808D008BE04D008
:10B9C00008A402D0ABEF5DF0AFEF5DF0096A0E6A3C
:10B9D0000350075C106E10E384EB0AF085EB0BF06C
:10B9E00086EB0CF087EB0FF080EB04F081EB05F0B9
:10B9F00082EB06F0083A09D080EB0AF081EB0BF0FD
:10BA000082EB0CF083EB0FF0106C089E08BC088EE4
:10BA10008FEB0DF008B081EF5DF01A0E106081EF32
:10BA20005DF00D6A076A08A408D0046C051E061EA6
:10BA3000071EE86A05220622072208AC08D00A6C15
:10BA40000B1E0C1E0D1EE86A0B220C220D22116A21
:10BA5000105207E007340632053204321132102E3C
:10BA6000F9D704500A2605500B2206500C22075025
:10BA70000D2291EB09F0089E0DAE0BD0096C0A1E49
:10BA80000B1E0C1E0D1EE86A0A220B220C220D2230
:10BA9000088E0DA006D0D8800C320B320A32093243
:10BAA0000F2A8FEB0DF055EF5DF00C500B100A10C4
:10BAB000091055E00EBE4DD00CBE0CD00D500E102E
:10BAC00048E0D89009360A360B360C360D06D8A059
:10BAD0000E06F2D70E5031E10D282FE009AE11D03D
:10BAE0007F0E091402E10AA00CD00A2AE86A0B2290
:10BAF0000C2207E3D8800C320B320A320D2A0D28B3
:10BB00001CE00D5026E08AEB00F08BEB01F00C34CA
:10BB1000026E0D30036E0232039E08BE038EE552A4
:10BB2000E5CFDAFFE7CFD9FF4EE912007F0E036EB3
:10BB3000FF0E026E016E006EF2D77F0E08BEFF0E82
:10BB4000036E02D07F0E036E800E026E016A006AE1
:10BB5000E6D708AE04D0800E036E026AF7D7036AF8
:10BB6000026AF4D70636073602E30884087E06E147
:10BB70000880076A066A056A046A1200072803E05B
:10BB8000D88006321200D890063202E108821200F4
:10BB9000088612000236033602E3088C087E06E1AE
:10BBA0000888036A026A016A006A1200032803E037
:10BBB000D88002321200D8900232EAE1088A1200DC
:10BBC000D89801D0D88851E8D9CFE6FFDACFE6FF80
:10BBD000E1CFD9FFE2CFDAFF94E9089E04E700AE97
:10BBE00002D0006C088E80EB0CF00B6A0A6A096ABE
:10BBF000860E0D6E0E6A55EF5DF0D89801D0D8888C
:10BC000050E8D9CFE6FFDACFE6FFE1CFD9FFE2CFA8
:10BC1000DAFF94E9089E07E701AE05D0006C011E2B
:10BC2000E86A0122088E81EB0CF080EB0BF00A6AC7
:10BC3000096A8E0E0D6E0E6A55EF5DF0D89801D030
:10BC4000D8884EE8D9CFE6FFDACFE6FFE1CFD9FFBB
:10BC5000E2CFDAFF94E9089E0BE703AE09D0006C4F
:10BC6000011E021E031EE86A012202220322088E20
:10BC700083EB0CF082EB0BF081EB0AF080EB09F028
:10BC80009E0E0D6E0E6A55EF5DF045E8D9CFE6FFCA
:10BC9000DACFE6FFE1CFD9FFE2CFDAFF8BE9086A1E
:10BCA000CAEC5DF008B659EF5EF008AA0AD008BCED
:10BCB00003D07F0E006E1BD0800E006E18D0006A7D
:10BCC00016D008B8FCD7870E0360F1D77E0E036448
:10BCD000F6D7860E035C04E0D8900232032AF9D727
:10BCE00008AC03D0026C02AEEAD782EB00F0E5525A
:10BCF000E5CFDAFFE7CFD9FF48E9120045E8D9CF11
:10BD0000E6FFDACFE6FFE1CFD9FFE2CFDAFF8BE93A
:10BD1000086ACAEC5DF008B692EF5EF008AA0ED091
:10BD200008BC05D07F0E016EFF0E006E23D0800E82
:10BD3000016E006A1FD0016A006A1CD008B8FBD7E8
:10BD40008F0E0360EDD77E0E0364F5D78E0E035C75
:10BD500005E0D89002320132032AF8D708AC06D0A9
:10BD6000016C021EE86A022202AEE5D781EB00F008
:10BD700082EB01F0E552E5CFDAFFE7CFD9FF47E9E3
:10BD8000120045E8D9CFE6FFDACFE6FFE1CFD9FFD1
:10BD9000E2CFDAFF8BE9086ACAEC5DF008B6D5EFAE
:10BDA0005EF008AA0FD008BC07D07F0E036EFF0E0E
:10BDB000026E016E006E2DD0800E036E01D0036AFC
:10BDC000000EF6D708B8FBD7076A9F0E0360EBD7C3
:10BDD0007E0E0364F4D79E0E035C07E0D890023217
:10BDE000013200320732032AF6D708AC0AD0076CBA
:10BDF000001E011E021EE86A00220122022202AE7B
:10BE0000DED782EB03F081EB02F080EB01F087EBF1
:10BE100000F0E552E5CFDAFFE7CFD9FF45E91200A0
:10BE200042E8D9CFE6FFDACFE6FFE1CFD9FFE2CF94
:10BE3000DAFF86E9036A1200F3DF038003D0F0DF44
:10BE400001D00382026A080EE76ED89001360236EE
:10BE50000050025C02E3026E012AE72EF7D703B21C
:10BE6000120003B081EB00F003A082EB00F0E5527A
:10BE7000E5CFDAFFE7CFD9FF43E9120043E8D9CF96
:10BE8000E6FFDACFE6FFE1CFD9FFE2CFDAFF89E9BB
:10BE9000066A1200F3DF068001D0F0DF01AE57EF33
:10BEA0005FF0006C011EE86A012206B0067E03AE58
:10BEB0005FEF5FF0026C031EE86A0322067E97ECD8
:10BEC0005FF003BE81EF5FF006AE08D0026C031E88
:10BED000E86A0322046C051EE86A052206B006D053
:10BEE00084EB00F085EB01F006A004D082EB00F0BB
:10BEF00083EB01F0E552E5CFDAFFE7CFD9FF45E963
:10BF0000000C06BE66EF5FF0E9DFFF0C43E8D9CF17
:10BF1000E6FFDACFE6FFE1CFD9FFE2CFDAFF89E92A
:10BF2000066A1200F3DF068003D0F0DF01D006823C
:10BF3000056A046A100EE76ED8900236033604369E
:10BF400005360050045C0150055805E30050045EBE
:10BF50000150055A022AE72EF0D706B2120006B0A9
:10BF600006D084EB00F085EB01F006A004D082EB54
:10BF700000F083EB01F0E552E5CFDAFFE7CFD9FF20
:10BF800045E9120045E8D9CFE6FFDACFE6FFE1CF79
:10BF9000D9FFE2CFDAFF8FE90C6A1200F3DF0C80E1
:10BFA00001D0F0DFE86A03AEDFEF5FF0006C011E46
:10BFB000021E031E0122022203220CB00C7E07AED9
:10BFC000EAEF5FF0046C051E061E071E052206221E
:10BFD00007220C7E31EC60F007BE1BEF60F00CAE68
:10BFE0000FD0046C051E061E071EE86A05220622F5
:10BFF0000722086C091E0A1E0B1E09220A220B22A8
:10C000000CB00AD088EB00F089EB01F08AEB02F06B
:10C010008BEB03F00CA008D084EB00F085EB01F073
:10C0200086EB02F087EB03F0E552E5CFDAFFE7CFCE
:10C03000D9FF49E9000C0CBEF1EF5FF0E1DFFF0C26
:10C0400045E8D9CFE6FFDACFE6FFE1CFD9FFE2CF6F
:10C05000DAFF8FE90C6A1200F3DF0C8003D0F0DF07
:10C0600001D00C820B6A0A6A096A086A200EE76E20
:10C07000D8900436053606360736083609360A36AD
:10C080000B360050085C0150095802500A58035002
:10C090000B5809E30050085E0150095A02500A5A31
:10C0A00003500B5A042AE72EE4D70CB212000CB04E
:10C0B0000AD088EB00F089EB01F08AEB02F08BEB01
:10C0C00003F00CA008D084EB00F085EB01F086EBC8
:10C0D00002F087EB03F0E552E5CFDAFFE7CFD9FFB7
:10C0E00049E912004AE8D9CFE6FFDACFE6FFE1CF0F
:10C0F000D9FFE2CFDAFF94E9086AB2EC5DF0CAEC4E
:10C100005DF008B696EF5DF008A205D008BA96EF8C
:10C110005DF09DEF5DF008BAA9EF5DF008A005D0D5
:10C1200008B896EF5DF0A9EF5DF008B89DEF5DF0FF
:10C130000E6A7F0E07240D6EE86A0E2203500D5E14
:10C14000E86A0E5A1A0E0F6E076A096A0A6A0B6AC3
:10C150000C6A0050045E0150055A0250065A000E47
:10C16000075A09E700500426015005220250062212
:10C17000000E072201D0098AD8900436053606360B
:10C180000736D89009360A360B360C360F2EE1D713
:10C19000065005100410D8A4098A55EF5DF042E856
:10C1A000D9CFE6FFDACFE6FFE1CFD9FFE2CFDAFF62
:10C1B00086E9036A1200F3DF038001D0F0DF00AEEE
:10C1C00003D0006C03B0037E01AE02D0016C037E8D
:10C1D00021EC5FF001BEFEEF60F003AE02D0016C17
:10C1E000026C03B081EB00F003A082EB00F0E5529B
:10C1F000E5CFDAFFE7CFD9FF43E9000C03BEEFD765
:10C20000F0DFFF0C44E8D9CFE6FFDACFE6FFE1CF5D
:10C21000D9FFE2CFDAFF8AE980EB04F081EB05F089
:10C2200082EB06F002500402F450016EF350006EEF
:10C230000350076E0502F450036EF350026E075070
:10C240000402F3500126F4500222E86A0322065049
:10C250000502F3500126F4500222E86A0322E55257
:10C26000E5CFDAFFE7CFD9FF46E9000C46E8D9CFA2
:10C27000E6FFDACFE6FFE1CFD9FFE2CFDAFF8EE9C2
:10C2800080EB06F081EB07F082EB08F085EB0BF01A
:10C2900084EB0AF083EB09F003500602F450016EC0
:10C2A000F350006E04500702F450036EF350026E18
:10C2B00004500602F3500126F4500222E86A0322D9
:10C2C00009500702F3500126F4500222E86A0322C3
:10C2D00005500602F3500226F450032205500702CF
:10C2E000046AE86A0422F3500326F4500422095039
:10C2F0000802F3500226F4500322056AE86A042279
:10C3000005220A500802F3500326F4500422E86A7A
:10C3100005220B500802F3500426F4500522E55282
:10C32000E5CFDAFFE7CFD9FF49E9000C44E8D9CFE0
:10C33000E6FFDACFE6FFE1CFD9FFE2CFDAFF8EE901
:10C3400080EB08F081EB09F082EB0AF083EB0BF055
:10C3500004500802F350006EF450016E04500902BC
:10C36000F3500126000EF420026E04500A02F3502E
:10C370000226000EF420036E04500B02F350032635
:10C3800005500802F3500126F4500222000E032249
:10C3900005500902F3500226F450032205500A0208
:10C3A000F350032606500802F3500226F4500322ED
:10C3B00006500902F350032607500802F3500326E3
:10C3C000E552E5CFDAFFE7CFD9FF48E9000C4AE8AC
:10C3D000D9CFE6FFDACFE6FFE1CFD9FFE2CFDAFF30
:10C3E00094E9086AB2EC5DF0CAEC5DF008B696EF2D
:10C3F0005DF008A205D008B896EF5DF09DEF5DF006
:10C4000008AA05D008B096EF5DF09DEF5DF008B08A
:10C4100002D008A802D0A9EF5DF00E6A03500724ED
:10C420000D6EE86A0E227E0E0D5EE86A0E5A096AEB
:10C430000A6A0B6A0C6A02500602F4500C6EF35042
:10C440000B6E01500602F3500A26F4500B22000E28
:10C450000C2202500502F3500A26F4500B22000E63
:10C460000C2200500602F3500926F4500A22000E56
:10C470000B220C2201500502F3500926F4500A2227
:10C48000000E0B220C2202500402F3500926F45035
:10C490000A22000E0B220C2200500502F45009263D
:10C4A000000E0A220B220C2201500402F45009262D
:0CC4B000000E0A220B220C2255EF5DF05A
:04C4BC0056656869F0
:10C4C000636C652069732073746F70706564207489
:10C4D00075726E6564206F6E0056656869636C6581
:10C4E00020616C61726D20697320736F756E646971
:10C4F0006E6721005472756E6B20686173206265EF
:10C50000656E206F70656E6564202876616C657459
:10C51000206D6F6465292E00562900562C20726507
:10C52000663D003132562042415454455259204F05
:10C530004B202800414C45525421212120313256B4
:10C540002042415454455259204352495449434191
:10C550004C2028002520534F432900414C4552547C
:10C5600021212120435249544943414C20534F43F8
:10C57000204C4556454C20415050524F4143484570
:10C580004420280053544154002B435553443A004F
:10C590004E4F524D414C20504F57455220444F571B
:10C5A0004E002B4346554E3A0052445900455252D4
:10C5B0004F520053454E44204641494C00434F4E94
:10C5C0004E454354204641494C00434C4F5345444B
:10C5D0000044415441204143434550540053454E8B
:10C5E00044204F4B002B4353513A00535441544580
:10C5F0003A2054435020434C4F5345440053544138
:10C6000054453A2054435020434F4E4E45435449DD
:10C610004E470053544154453A20434F4E4E4543F4
:10C6200054204F4B0053544154453A2000434F4E41
:10C630004E454354204F4B0036342C002C00322CF6
:10C64000002B43434C4B002B434C4950002B504490
:10C65000503A204445414354002B435245473A2029
:10C660003000222C2236383637220D0041542B431D
:10C67000495053544152543D22544350222C2200DD
:10C6800041542B43444E534346473D220041540DF1
:10C690000041542B43494653520D0041542B43490A
:10C6A00050484541443D310D0041542B43494943D5
:10C6B000520D00222C220041542B435354543D224E
:10C6C00000220D0041542B434744434F4E543D310B
:10C6D0002C224950222C22002B43524547002B4349
:10C6E0004F50533A002B434D45204552524F520074
:10C6F000534554555000223B2B434F50533F0D00A0
:10C7000041542B434F50533D312C312C2200415486
:10C710002B434C504F52543D22544350222C22362E
:10C72000383637220D0041542B434950434C4F5368
:10C73000450D0041542B434950534855540D0000BA
:10C740002D002200495000534D53000D0A004D505A
:10C750002D30205045006572726F723A200074616E
:10C76000726765742072656163686564003A0020D1
:10C77000696465616C206D690D0020746F20006E26
:10C780006F20706F776572206C6576656C207370B2
:10C790006563696669656400435450206E6F742058
:10C7A000617661696C61626C65000D20534F483A97
:10C7B00020000D204341433A20000D204F444F3AC2
:10C7C00020000D204573742E2052616E67653A205B
:10C7D000000D20496465616C2052616E67653A20E6
:10C7E0000025000D20534F433A20004E6F74206304
:10C7F00068617267696E67003A2000253A20002060
:10C800006D696E73000D2046756C6C3A2000410016
:10C81000562F000D20004368617267652053746FC6
:10C8200070706564004368617267696E672C2048A8
:10C83000656174696E6700507265706172696E67D8
:10C840000043686172676520446F6E6500546F70C5
:10C8500070696E67206F6666004368617267696E13
:10C860006700506572666F726D616E6365202D2082
:10C870000052616E6765202D200053746F726167EE
:10C8800065202D20005374616E64617264202D2038
:10C89000006D696E732072656D61696E2900637940
:10C8A000636C65732C200043202800432F00436FE6
:10C8B0006F6C646F776E3A2000206B6D00206D699D
:10C8C000002C312C496E76616C69642055535344B9
:10C8D00020726573756C74002C302C00202D204D57
:10C8E00053473A2000534D532046524F4D3A2000B3
:10C8F0004D502D30205041000D00222C31350D00BF
:10C9000041542B435553443D312C22004D502D3082
:10C910002063332C302C004D502D302063312C30CF
:10C920002C004D502D302061004D502D3020004DF9
:10C93000502D53203020004D502D3020482A2D4FAF
:10C94000564D2D446562756743726173682C302CB7
:10C95000323539323030302C004D502D3020455496
:10C96000004D502D3020670043312D362C4334309C
:10C970002D34312C433439004D502D302056004D8C
:10C98000502D3020440056325039002F56002F00D1
:10C990002E004D502D30204600302C302C004D50B4
:10C9A0002D302057004D502D30204C002C706572DA
:10C9B000666F726D616E6365002C72616E676500F3
:10C9C0002C73746F72616765002C7374616E64619F
:10C9D0007264002C73746F70706564002C686561FC
:10C9E00074696E67002C70726570617265002C64EA
:10C9F0006F6E65002C746F706F6666002C636861E3
:10CA00007267696E67002C004D502D302053002056
:10CA1000004D502D43203020000D0A004D502D3088
:10CA200020454D001B001A000A232E0A0041542BFA
:10CA300043495053454E440D002320004D502D30A6
:10CA40002063002000436F6D6D616E64733A000DCA
:10CA50000A2020287374616C6529004300430D0A85
:10CA60002020436861726765723A2000430D0A20F6
:10CA700020426174746572793A2000430D0A2020C7
:10CA80004D6F746F723A2000430D0A202050454DBF
:10CA90003A200054656D7065726174757265733A01
:10CAA0000D0A2020416D6269656E743A20000D0AFE
:10CAB0002056494E3A0056325039002F56002F006A
:10CAC0002E004F564D53204669726D776172652076
:10CAD00076657273696F6E3A20000D0A2000466514
:10CAE0006174757265733A00202D20002053544BF9
:10CAF000554E46002053544B46554C002052490099
:10CB000020544F002050440020504F520020424FEC
:10CB100052000A202E2E6C6173743A000A20437270
:10CB200061736865733A00207265663D000A2031C2
:10CB30003256204C696E653A000A204E4554205307
:10CB4000746174653A3078000A2047524E204C6573
:10CB5000643A000A20524544204C65643A00444936
:10CB600041473A000D0A20506172616E6F69643A64
:10CB7000000D0A2049503A005365727665723A00FA
:10CB800043757272656E743A20000D0A00286E6F4C
:10CB90006E65290D0A0047534D4C4F434B3A200018
:10CBA00029000D0A2047534D2F475052533A204E2B
:10CBB0006F7420636F6E6E656374656420283078CF
:10CBC000000D0A2047534D3A204F4B0D0A20536564
:10CBD000727665723A204E6F7420636F6E6E656375
:10CBE000746564000D0A20475052533A204F4B0D94
:10CBF0000A205365727665723A20436F6E6E6563E4
:10CC0000746564204F4B000D0A20475052533A2060
:10CC100044495341424C4544000D0A2047534D3A84
:10CC2000000D0A20444E533A000D0A2050617373E0
:10CC3000776F72643A000D0A20557365723A000DE1
:10CC40000A2041504E3A00475052533A0056656808
:10CC500069636C653A000D0A204E6F7469666963FA
:10CC60006174696F6E733A000D0A20556E697473B2
:10CC70003A000D0A2056656869636C6549443A00BC
:10CC80004D6F64756C653A000D0A204361725479EA
:10CC900070653A000D0A2056656869636C655479C1
:10CCA00070653A003A000A00506172616D733A0093
:10CCB000266D6C6F6E3D002B004D6F64756C6520AA
:10CCC00070617373776F72643A200052656769739D
:10CCD0007465726564206E756D6265723A20001A23
:10CCE000000A232E0A000D2000220D0A0041542BB9
:10CCF000434D47533D22002320006D6F64652000A3
:10CD0000706572666F726D616E63650072616E67E9
:10CD1000650073746F72616765007374616E64613E
:10CD20007264002D003031323334353637383941B2
:10CD30004243444546005045520052414E00535430
:10CD40004F0053544100232053746F70706564206A
:10CD500043414E2073696D0A00232053746172743D
:10CD6000696E672043414E2073696D0A0041542B60
:10CD70004353510D0041542B4350494E3F0D004148
:10CD8000542B434F50533F0D0023202053696D20F7
:10CD900054783A20002320204348415247453A2006
:10CDA00020200020657374206D696C6573290A006A
:10CDB00020696465616C2C20002520280023202038
:10CDC000534F433A20202020202000290A00202809
:10CDD0000023202056494E3A202020202020000AFF
:10CDE0000A002320205369676E616C3A20202000DE
:10CDF0002320204C4F4747494E473A2020002056D9
:10CE00000A00232020313256204C696E653A2000FA
:10CE1000202F200023202043524153483A20202035
:10CE200020002320205357495443483A2020200013
:10CE300056325039002F56002F002E00232046690D
:10CE4000726D776172653A20000A23204449414798
:10CE50000A0A000A23204C656176696E67204469DE
:10CE600061676E6F7374696373204D6F64650A0048
:10CE7000232027532720434F4D4D414E44533A0022
:10CE80002320274D2720434F4D4D414E44533A0A0E
:10CE90002320002320434F4D4D414E44533A204818
:10CEA000454C50203F20444941472052455345546A
:10CEB000206F72204D2F53202E2E2E0A000A000ABA
:10CEC00023204E4F5449465920414C41524D204158
:10CED0004C4552540A000A23204E4F5449465920CB
:10CEE0005452554E4B20414C4552540A000A2320BF
:10CEF0004E4F544946592043484152474520414CE2
:10CF00004552540A001B5B324A1B5B30313B3031C7
:10CF1000480D23204F564D5320444941474E4F530F
:10CF200054494353204D4F44450A0A000D0A000D51
:10CF30000A23205452206D696E75746573746F6393
:10CF4000686172676520726573756C743D00290DA8
:10CF50000A002C20000D0A23205452206D696E75A2
:10CF6000746573746F63686172676528003A002C9A
:10CF7000002C302C0063004D502D302000585800FC
:10CF80004D49004E4C0056410054520030003100D3
:10CF900047454E5F315F4E45575F4341525F4749BA
:10CFA0004453004D502D3020484E4C2D434F4D2DB5
:10CFB0004849532C322C38363430302C002C38363B
:10CFC0003430302C004D502D3020484E4C2D434FE6
:10CFD0004D2D43414E2C002C2A2D4C6F672D43685C
:10CFE000617267652C002C333135333630303000B8
:10CFF0002C2A2D4C6F672D44726976652C002C000D
:07D000004D502D30206800A7
:08D008001AEC6DF084E900EB65
:10D0100044F001EB45F002EB46F041E9E7CFD9FFE0
:10D0200012001AEC6DF082E9D8900EE2030E005C5B
:10D030000BE200014351005C07E000EB43F04A6B58
:10D040004B6B476B486B496B41E9E7CFD9FF120047
:10D05000000147514811491102E154EC6DF0C3EC55
:10D060006CF013EC6DF00B01D151D21101E1ECD059
:10D07000C3EC6CF0070EF9EC6CF0F6CFD3FBF7CFF6
:10D08000D4FBF8CFD5FBFEEC6CF0E5CFD8FBE5CFB9
:10D09000D7FBE7CFD6FB0B01D351D625F36ED45186
:10D0A000D721F46ED551D821F86EF4CFF7FFF3CF26
:10D0B000F6FF13EC6DF0D1510008000ED25501E3DC
:10D0C000C0D0C3EC6CF0070EF9EC6CF0F6CFDBFBD4
:10D0D000F7CFDCFBF8CFDDFBFEEC6CF0E5CFE0FB3F
:10D0E000E5CFDFFBE7CFDEFB0B01DB51DE25F36E87
:10D0F000DC51DF21F46EDD51E021F86EF4CFF7FF53
:10D10000F3CFF6FF0900F5CFE6FF0900F5CFE6FF04
:10D110004AC0E6FF4BC0E6FF95EC5FF0E552E5CF75
:10D12000DAFBE7CFD9FB0B01D951DA1101E089D045
:10D130000F0140B7FDD776EC6DF0F5CF50F0C3ECA2
:10D140006CF0050EF9EC6CF00900F5CF51F00A0017
:10D15000F5CF52F06EEC6DF013EC6DF00B01D15188
:10D16000D21133E06EEC6DF00900F5CF4CF00A00FF
:10D17000F5CF4DF06EEC6DF00900F5CF4EF00A00E2
:10D18000F5CF4FF00F01406BC3EC6CF05BEC6DF032
:10D19000070E0B011FEC6DF006E00B01D890D137A4
:10D1A000D237E804FBE1D1CB42FFEDDB5BEC6DF065
:10D1B0000B013CEC6DF006E00B01D890D233D1337B
:10D1C000E804FBE1D1CB41FF0FD00001E80E4C6F2A
:10D1D000070E4D6FEF0E4E6F070E4F6F0F01406B36
:10D1E000E00E426FFB0E416F76EC6DF0F550220AB7
:10D1F00017E02B0A09E0280A07E0200A08E0030AE2
:10D2000006E0120A1CE103D00001546B556B0F01BC
:10D21000020E466F50C047FF51C048FF496B0DD00A
:10D220000F01030E466F220E476F0B01D26B52C0E7
:10D2300048FF000151510F01496F44EC6DF062EF5E
:10D240006DF062EC6DF00BD754EC6DF000014A2BE1
:10D25000000E4B234A5110080E0E4B5504E2100EDF
:10D260004A5F0E0E4B5B1200E5DB81E941E80001ED
:10D270005051220A01E1ABD02B0A18E0280A16E02F
:10D28000200A05E0030A03E0120A01E0B8D0400ECC
:10D290005025075D01E0B3D008514CEC6DF001E082
:10D2A000AED069EC6DF001E0AAD0A7D006390F0B23
:10D2B00001084FE1400E5025085D4BE10951ECDBC0
:10D2C00048E169EC6DF045E10F0140B7FDD7406BD7
:10D2D000C0DB070EB4DB06E00B01D890D137D237A4
:10D2E000E804FBE1D1CB42FFB4DBC6DB06E00B0177
:10D2F000D890D233D133E804FBE1D1CB41FF0F0109
:10D30000300E466F476B320E486F496BBDDBF00E37
:10D31000000106150B01D26FD16B000107510B0103
:10D32000D1250001546F000E0B01D2210001556F71
:10D33000030E545F000E555B030E566F576B586B10
:10D34000596B056F0BC006F00CC007F00DC008F05C
:10D3500054D0000106390F0B020851E15451000866
:10D36000000E55554CE2016A070E015C13E20128DC
:10D37000EA6A060FE96E000EEA22EF50E66E0150EF
:10D38000EA6A060FE96E000EEA22E552E750EF6EF8
:10D39000012AEAD7000154510708000E55550BE247
:10D3A000070E545F000E555B070E5627000E5723DD
:10D3B000070E056F08D054C005F05451562755513B
:10D3C0005723546B556B582B000E592316D0620E01
:10D3D000075D15E108C0D4FB0B01D36B00010951B7
:10D3E0000B01D325D16F000ED421D26F0001515112
:10D3F0000B01D11904E16DDB02E1010E01D0000E39
:10D4000042E9E7CFD9FF1200DACFE4FFE2CFDAFF3B
:10D41000E9CFE4FFEACFE4FFD9CFE4FFDACFE4FFBE
:10D42000FCC0E4FFFDC0E4FFFEC0E4FFFFC0E4FF7A
:10D43000F6CFE4FFF7CFE4FFF8CFE4FFF5CFE4FF4A
:10D44000F3CFE4FFF4CFE4FFFACFE4FFFBCFE4FF38
:10D45000E6526050800B45E0000119511A111B1172
:10D4600040E06250D5DA06E00701D890E933E833AE
:10D47000E804FBE16150A7DA010E6014046F0F0E9F
:10D480006514056F66CF06F067CF07F068CF08F028
:10D4900069CF09F06ACF0AF06BCF0BF06CCF0CF0BC
:10D4A0006DCF0DF0609EA49044514511461113E0DC
:10D4B0004C51025D4D51035914E302514E5D03512D
:10D4C0004F590FE3D1DE00090CE01BC0FBFF1AC06F
:10D4D000FAFF000104D01BC0FBFF1AC0FAFF19516C
:10D4E00014000F015051800B38E000011C511D1138
:10D4F0001E1133E03C0E536F0F01525189DA06E0E2
:10D500000701D890E933E833E804FBE10F015151FA
:10D510005ADA070E0F0150150001046F0F0E0F01AC
:10D5200055150001056F56CF06F057CF07F058CFBD
:10D5300008F059CF09F05ACF0AF05BCF0BF05CCF5F
:10D540000CF05DCF0DF00F01509FA4921EC0FBFFA9
:10D550001DC0FAFF00011C511400A450010B01E092
:10D5600078D7A450020B01E074D7E552E5CFFBFF5A
:10D57000E5CFFAFFE5CFF4FFE5CFF3FFE5CFF5FF09
:10D58000E5CFF8FFE5CFF7FFE5CFF6FFE5CFFFF0FA
:10D59000E5CFFEF0E5CFFDF0E5CFFCF0E5CFDAFF1B
:10D5A000E5CFD9FFE5CFEAFFE5CFE9FFE5CFDAFF29
:10D5B000110040DA81E942E80001006B016B0E6B5B
:10D5C000136B146B156B436B446B456B466B476B6E
:10D5D000486B496B4A6B4B6B4C6B4D6B4E6B4F6B97
:10D5E000506B516B526B536B5A6B5B6B5C6B106B7C
:10D5F000116B126B166B176B186B196B1A6B1B6B1D
:10D600001C6B1D6B1E6B1F6B206B216B226B236BC6
:10D61000246B256B266B276B286B296B2A6B2B6B76
:10D620002C6B2D6B2E6B2F6B306B316B326B336B26
:10D63000346B356B366B376B386B396B3A6B3B6BD6
:10D640003C6B3D6B3E6B3F6B406B416B426B06012D
:10D65000EE91020E08DA01EBE9FF02EBEAFFEFCFF1
:10D660000FF00E0E00DA0150021007E10B01956B6E
:10D67000966B976B986B996B36D034DA890EE66EA1
:10D68000CF0EE66E000E95D903E1D9EC2DF02BD02C
:10D6900029DA860EE66ECF0EE66E000E8AD903E119
:10D6A00010EC71F020D01EDA830EE66ECF0EE66E1F
:10D6B000000E7FD903E153EC5BF015D013DA800E36
:10D6C000E66ECF0EE66E000E74D903E149EC7AF0F7
:10D6D0000AD008DA7D0EE66ECF0EE66E000E69D92E
:10D6E00002E172EC92F0080E0601EE15000806E267
:10D6F0000001010E886F896B8A6B8B6BD08EA382C1
:10D70000A380030EA56E43E9E7CFD9FF120092D99B
:10D7100081E942E80001002B000E0123535100086B
:10D7200007E244514511461103E092DC0001530722
:10D73000000E0001E76EC31902E7C33502D0C351E2
:10D74000E75C01E2C307000E0001E76EC41902E7BF
:10D75000C43502D0C451E75C01E2C407000E0001E9
:10D76000E76EC51902E7C53502D0C551E75C01E295
:10D77000C507000E0001E76EC61902E7C63502D0E4
:10D78000C651E75C01E2C60774AE03D0609EA49068
:10D79000749E74AC04D00F01509FA492749C00013D
:10D7A0007351010B04E000017751000803E200010E
:10D7B0000F0E906F00011F512011211106E021C0B2
:10D7C000FBFF20C0FAFF1F5114000A0EE66EE66A46
:10D7D000E1D80BE1000122512311241106E024C0FD
:10D7E000FBFF23C0FAFF22511400000171A925D0CC
:10D7F0000001E0510008000EE15508E2E05100018F
:10D80000795D0001E15100017A5908E20001E2511D
:10D81000000813E2E2510001785D0FE3000EE66EAE
:10D82000E66A0C0EE66EE66AE66A39C0FBFF38C0AF
:10D83000FAFF00013751140045E93C0EE66EE66A36
:10D84000A9D853E10B01C751016E026A010E000114
:10D850000E1513E100017851F36E02340EE201500F
:10D86000F35C000E025409E2040EE66EE66AA9ECCF
:10D8700003F042E900010E811AD0010E00010E15DD
:10D8800016E0000178510B01D16FD26B020E01241A
:10D89000D36F000E0220D46FD235D251D41904E6D2
:10D8A000D151D35DD251D45902E200010E91000151
:10D8B0007351010B0FE0000177510CE1000190075B
:10D8C00009E1400EE66EE66AA9EC03F042E90001C8
:10D8D0003C0E906F000125512611271106E027C04C
:10D8E000FBFF26C0FAFF255114002C0EE66E010E38
:10D8F000E66E50D80BE10001285129112A1106E0EB
:10D900002AC0FBFF29C0FAFF28511400580EE66E0A
:10D91000020EE66E3FD810E100012B512C112D11A3
:10D9200006E02DC0FBFF2CC0FAFF2B511400580E4F
:10D930000001005F020E015B00012E512F1130111A
:10D9400006E030C0FBFF2FC0FAFF2E51140043E960
:10D95000E7CFD9FF1200000131513211331106E037
:10D9600033C0FBFF32C0FAFF315114001200000136
:10D9700034513511361106E036C0FBFF35C0FAFFD1
:10D9800034511400120047C0F6FF48C0F7FF49C0E9
:10D99000F8FF120000C0E6FF01C0E6FF95EC5FF063
:10D9A000E552E5CFD2FBE7CFD1FB0B01D151D2112C
:10D9B0001200E66E01EBE6FF02EBE6FFB4EC84F04A
:10D9C00047E9000912000701ED6FEE6BD890ED37C3
:10D9D000EE37D890ED37EE37D890ED37EE37E85187
:10D9E000ED250001026F0701E951EE210001036FEF
:10D9F0001200F626000EF722F822120073D8E66A0B
:10DA000043C0E6FFE66AE66A36EC61F0E5521200D2
:10DA10000701EA6FEB6B050EEC6FEC51EAC7E8F714
:10DA2000EBC7E9F712000900F5CFD1FB0800F5CFED
:10DA3000D2FB1200D9CFE6FFE1CFD9FF1200D317F6
:10DA4000000ED417050ED3CBD1FBD4CBD2FB000AEA
:10DA5000120002C0D3FB03C0D4FB0B01080ED35F3E
:10DA6000000ED45B1200E66E18EC8BF041E9F35027
:10DA7000016EF450026E1200030ED56FD551D3CB58
:10DA8000D1FBD4CBD2FB12004A6B4B6B4C6B4D6B72
:10DA9000080E456F406F12000B01D16FD26B000171
:10DAA00051510B01D119120044C047F045C048F054
:10DAB00046C049F012000900F5CFD3FB0800F5CFAE
:10DAC000D4FB120000010D0E4727000E4823492306
:10DAD0001200000152510B01D219120054DF020E44
:10DAE000F9EF6CF0020EE66EE66A12004CDF040EEF
:06DAF00080DF08001200B7
:0ADAF60017EC72F043E8036A0A011E
:10DB00007651000807E2760703E10001739102D025
:10DB1000000173810001882B000E89238A238B2347
:10DB20000001625158E000016051611154E00001B0
:10DB30007589000171B718D00C0E71130001686B64
:10DB40000001696B0001010E666F0001030E676F33
:10DB50000001100E636F0001646B656B00016A6B5E
:10DB60006B6BFFEC71F05ED071850A01712B3C0E7E
:10DB7000715D58E3716B0001642B000E652360C07A
:10DB8000E6FF61C0E6FF00016251E66EE66A02EC64
:10DB900061F03CEC72F00A0172270B01D2510A01CC
:10DBA0007323000E74237523600E725DEA0E7359A1
:10DBB000000E7459000E755935E30A0E00016A27EC
:10DBC000000E6B23600E0A01725FEA0E735B000E9B
:10DBD000745B755B27D00001625124E10001605144
:10DBE000611120E1000171A71BD0F30E711771853F
:10DBF0000001686B0001696B5F0E0001785D06E251
:10DC00000001150E666F00010E0E05D00001040E16
:10DC1000666F0001030E676F040E63EC72F0EFDBBA
:10DC2000000175990A017B5116E0010EE66EF7ECD2
:10DC30003DF041E932EC12F07C0EE66E0A0EE66E23
:10DC4000000EE66E070EE66EA2EC85F044E96FEC7E
:10DC500012F00A017B6B705107E10001625104E18F
:10DC600000016051611171E00B01CD516EE0016A5C
:10DC7000026A0B0176DBDABFDB6955DB69EC72F017
:10DC8000D151D21160E06DDBDABFDB694CDB020EF3
:10DC9000F626000EF722F8220800F550E66EE66A36
:10DCA00000C0E6FF01C0E6FF95EC5FF0E5DBD211B6
:10DCB00046E1035002E0E9EC3DF00F0140B7FDD72B
:10DCC000406B8EDBDCBFDD695ADB070ED317000E1D
:10DCD000D417E2DB06E00B01D890D137D237E80445
:10DCE000FBE1D1CB42FF7CDBDCBFDD6948DB030E0F
:10DCF000DE6FDE51D3CBD1FBD4CBD2FB06E00B01E0
:10DD0000D890D233D133E804FBE1D1CB41FF0F01EE
:10DD1000030E466F220E476F0B0123DBDABFDB6970
:10DD200002DB7EDBD2CBD1FBD26BD1CB48FF19DB40
:10DD3000DABFDB69F8DA74DBD1517FDB036E012ACD
:10DD4000000E022296D70A01706B000E44E9E7CF5D
:10DD5000D9FF12006CDB48E8076A086A0A013C0E2A
:10DD6000766F08C01DFB0B011C6B000109510B01F4
:10DD70001C25016E000E1D21026E00010A51036E6A
:10DD80000A01795101184BE17A51021848E17751A3
:10DD90000001021944E10A017851000103193FE131
:10DDA0000A017B513CE1770EE66ECF0EE66E000E67
:10DDB000E66E7C0EE66E0A0EE66E19EC43F045E95F
:10DDC000F350056EF450066E2E0EE66EE66A750E82
:10DDD000E66ECF0EE66E000EF6DA02C0E6FF03C076
:10DDE000E6FF710EE66ECF0EE66E000EECDA01EB8A
:10DDF000E6FF02EBE6FF61DBE6DA046A080E045C8C
:10DE000007E2045005DBE66A58DBDDDA042AF6D7C0
:10DE10000A01010E7B6F776B786B796B7A6B620E00
:10DE20000001075D02E0010E33D1EC0E0001021982
:10DE300001E0A2D0070E031901E09ED034DB340EBE
:10DE4000F31802E1830EF4186CE0430EF31802E1BC
:10DE50001C0EF4185AE04F0EF31802E1430EF418AA
:10DE600048E01E0EF31802E1800EF4183EE01F0E8B
:10DE7000F31802E1800EF41823E0680EF31802E1B3
:10DE8000430EF41815E0690EF31801E000D1430EBB
:10DE9000F41801E0FCD0050EE66EE66A0350E66E6B
:10DEA000E66A92EC5FF0E55203DB1CCB62F0EFD048
:10DEB00003500001606F616BD89060376137E7D025
:10DEC00000013C0EC36F03500B011D6BE8307F0B4C
:10DED0001C6F280E1C5F000E1D5B1CCB91F0000117
:10DEE000926B91AFD4D09269D2D000013C0EC46F36
:10DEF000CED000013C0EC46F03500001A96FAA6B85
:10DF0000280EA95F000EAA5BC2D000013C0EC46FB0
:10DF100003500001A56FA66B280EA55F000EA65B3F
:10DF2000B6D000013C0EC46F630EE66EE66A035085
:10DF3000270DF3CFE6FFF4CFE6FF4AEC5FF0E552A2
:10DF4000B7DA1CCB78F0640EE66EE66ABCCAE6FF70
:10DF5000BDCAE6FF00017851E66EE66A02EC61F0A8
:10DF600092EC5FF0E552E5CF7AF0E7CF79F079C037
:10DF70007BF07AC07CF08BD0E80E021945E1070EE9
:10DF8000031942E190DA0D0EF31801E080D0F4504D
:10DF900001E07DD04B0E00010F5D03E103EB77F054
:10DFA00076D0490EE66E060E9BDAE80EE66E030E9C
:10DFB00097DA03EBE6FFE66AE66AE66A96EC61F05A
:10DFC000E552E5CF23FBE5CF22FBE5CF21FBE7CFF1
:10DFD00020FBF40E0B012027010E2123000E22232B
:10DFE000232320CBE6FF21CBE6FF22CBE6FF23CB8A
:10DFF000E6FF2CEC60F0E552E5CF1FFBE5CF1EFB02
:10E0000057DA1CCB77F043D0E90E021940E1070E36
:10E0100003193DE148DA870EF31839E1240EF418AC
:10E0200036E1640EE66EE66A0AC022FB0AC023FBF4
:10E030000B01226B00010B510B012225206F000EFA
:10E040002321216F20CBE6FFE66E92EC5FF0E66ABB
:10E05000E66ADDEC3EF044E9FCC01CFBFDC01DFBA4
:10E06000FEC01EFBFFC01FFB0B011C51076E1D51A4
:10E07000086E0A010750BC5D0850BD5908E2040E45
:10E080000001665D04E107EBBCFA08EBBDFA010E86
:10E0900049E9E7CFD9FF1200CAD941E80A01010EC8
:10E0A000706F3C0E766F020E0001045D4BE0030EB4
:10E0B000045D0DE1016A080E015C06E20150A8D979
:10E0C000090E0124C5D9F7D70001A46B3BD0040E7B
:10E0D000045D0CE10001310E936F016A080E015CD2
:10E0E00031E2015095D90128B3D9F8D7050E045D66
:10E0F00029E10001065117E10001718D719F0001B6
:10E100008C518D118E118F111DE188C08CF089C04A
:10E110008DF08AC08EF08BC08FF08C07000E8D5B67
:10E120008E5B8F5B0DD00001719D718F00018C5152
:10E130008D118E118F1106E08C6B8D6B8E6B8F6B3A
:10E14000020EC1D9010E42E9E7CFD9FF1200D9CFA3
:10E15000E6FFE1CFD9FF86E902EBF3FF03EBF4FF23
:10E160002E0EF31858E1F45056E1A7D9E66E00EBF5
:10E17000E6FF01EBE6FF76D90CE086D9F3CF77FA1C
:10E18000F4CF78FA9AD9E66E000EE66EE66A6AD99E
:10E1900002E1000E41D078D9F3CF79FAF4CF7AFAC0
:10E1A0000A017B6BE9EC3DF00F0140B7FDD7406BF6
:10E1B000070E0A0177150B01D36FD46B6DD906E0FA
:10E1C0000B01D890D137D237E804FBE1D1CB42FF25
:10E1D0000B01030ED36FD35177CAD1FB78CAD2FBA0
:10E1E00006E00B01D890D233D133E804FBE1D1CB68
:10E1F00041FF080E0A017727000E78230F01030E56
:10E20000466F220E476F0B01D26B7ACA48FF0A0194
:10E21000795113D901D0000E41E9E7CFD9FF12009F
:10E2200006D942E80B01560E956F410E966F976B1B
:10E23000986B996B0A01DC0E6C6FDA0E6D6FD40E61
:10E240006E6F340E6F6F706B716B726B736B746B80
:10E25000756B766B776B786B796B7A6B7B6B000188
:10E26000C7690001886B896B8A6B8B6B230E38D969
:10E27000E66ADDEC3EF044E9FCC0BCFAFDC0BDFA44
:10E28000900E6F6E6EAEFED7606A0F01196B186943
:10E29000016BFD0E006F506BE00E1D6F1C69C00E10
:10E2A000096F400E086F200E0D6F9C0E0C6F800ED4
:10E2B000116FA20E106FA00E156F260E146F010EB7
:10E2C000706ED20E716E020E726E200E736E0B01A6
:10E2D000CD51000802E26F6A02D0600E6F6E00013D
:10E2E000540E196FDD0E1A6F000E1B6F0001980E91
:10E2F0001C6FE00E1D6F000E1E6F0001F60E1F6FEB
:10E30000DA0E206F000E216F00014E0E376FE10E06
:10E31000386F000E396F0601EE81EE83010E43E97E
:10E32000E7CFD9FF1200D9CBE6FFDACBE6FFDBCB94
:10E33000E6FF36EC61F0E552E5CFD8FBE5CFD7FB41
:10E34000E7CFD6FB0B01D351D625F36ED451D7219D
:10E35000F46ED551D821F86EF4CFF7FFF3CFF6FF66
:10E3600012001C0ED36F250ED46F010ED56F050E53
:10E37000B7D801EBD9FB02EBDAFBDB6B1200DBCB8E
:10E38000E6FFDCCBE6FFDDCBE6FF36EC61F0E552E5
:10E39000E5CFDAFBE5CFD9FBE7CFD8FB0B01D551B1
:10E3A000D825F36ED651D921F46ED751DA21F86E03
:10E3B000F4CFF7FFF3CFF6FF0900F5CFD3FB08004A
:10E3C000F5CFD4FB1200E66E05EBE6FF06EBE6FFA9
:10E3D0006DEC43F047E9F350056EF450066E120001
:10E3E0000B011C0ED56F250ED66F010ED76F050ED3
:10E3F00077D801EBDBFB02EBDCFBDD6B12000A01E3
:10E40000716B726B736B746B756B020E63EF72F0F2
:10E41000EA6A060FE96E000EEA22EF50E66E12007D
:10E42000030EF626000EF722F82269EF72F0D9CF1C
:10E43000E6FFE1CFD9FF81E912000F01496F4A6B76
:10E440004B6B4C6B4D6B080E456F406F010E12000D
:10E45000EA6A930FE96E000EEA22E552E750EF6E8A
:10E46000012A120003EC91F045E9F350006EF450DC
:10E47000016E005001101200E552E5CFD2FBE7CF4C
:10E48000D1FB0B01D151120000EBE6FF01EBE6FFDF
:10E4900009EC7FF042E91200050ED3CBD1FBD4CBBF
:10E4A000D2FB000A120001EBF3FF02EBF4FF1200B3
:10E4B000E5CF1DFBE7CF1CFB12006F0EE66ECF0E03
:10E4C000E66E000E1200E66EE66AA9EC03F042E981
:10E4D00012000900F5CFD1FB0800F5CFD2FB1200E6
:08E4E000E66EE66AE66A12002E
:08E4E800E668E6DB0601CE6BDD
:10E4F000CF6B0601CD6B050EE66ECF0EE66E000EFD
:10E50000BCDBCDCBCCF50501CD69CE691200FCECAE
:10E5100076F081E943E80501CE3501E3B4D00B0183
:10E520005E0ED16F1B0ED26F010ED36F020EE66E20
:10E53000E66AE66A660ED76F1B0ED86F010ED96FBA
:10E54000CDC5DAFBCEC5DBFB090EDB03F3CFDBFB6E
:10E55000DA03F3CFDAFBF450DB27DC6BDBBFDC69DB
:10E56000D751DA25F36ED851DB21F46ED951DC2175
:10E57000F86EF4CFF7FFF3CFF6FF0800F5CFE6FF14
:10E58000E66AE66AC3EC76F00900F550016E0A000F
:10E59000F550026E0F01406B070E0B010114D36F93
:10E5A000D46B050ED3CBD1FBD4CBD2FB000A06E053
:10E5B0000B01D890D137D237E804FBE1D1CB42FF31
:10E5C0000B0101EBD1FB02EBD2FB030ED890D2334F
:10E5D000D133E804FBE1D1CB41FF010E036E0B0107
:10E5E00037DBD5BFD66912EC77F0F5CF46FF30DBCD
:10E5F000D5BFD66912EC77F0F5CF47FF29DBD5BF41
:10E60000D66912EC77F0F5CF48FF22DBD5BFD6698B
:10E6100012EC77F0F5CF49FF1BDBD5BFD66912ECC2
:10E6200077F0F5CF4AFF14DBD5BFD66912EC77F04F
:10E63000F5CF4BFF0DDBD5BFD669F4DBF5CF4CFF33
:10E6400092DBF3CFD7FBB1DBD5BFD669EBDBF5CFE0
:10E650004DFF0F01080E456F4087110EE66EE66A0A
:10E66000CDC5D1FBCEC5D2FB0B01D12B000ED223E1
:10E67000D1CBE6FFD2CBE6FF4DEC5FF0E552E5CF24
:10E68000CEF5E7CFCDF5040E4BDB040E2DDB09E014
:10E69000ED0EE66ECE0EE66E000EEFDA0601FA958E
:10E6A000FB95100E3DDB100E1FDB09E0D60EE66E6B
:10E6B000CE0EE66E000EE1DA0601FA99FB99200E05
:10E6C0002FDB200E11DB09E0BF0EE66ECE0EE66EEC
:10E6D000000ED3DA0601FA9BFB9B44E9E7CFD9FF92
:10E6E00012009CDB000EE66EE66AA6EC00F042E942
:10E6F0001CDBD60EE66E060EE66EFEEC50F044E92C
:10E70000C4D28CDB12DBB4EC19F042E90B0191515D
:10E71000921102E07BEC1BF0B8D280DB010EBCDA78
:10E72000930EE66ECE0EE66E000EA7DA800EE66E53
:10E73000CE0EE66E000EA1DAE66AFDEC16F041E9B7
:10E74000700EE66ECE0EE66E000E97DA02EBE6FF76
:10E7500003EBE6FF02EBE6FF03EBE6FFC2DF44E973
:10E7600094D290DAE66AA8DA530EE66ECE0EE66E22
:10E77000000E83DA0A0E90DA050EE66E41EC04F024
:10E7800041E983D27FDA45E8010E076E020E076E7B
:10E79000490EE66ECE0EE66E000E6FDA0E0EF66EC7
:10E7A000000EF76E000EA7DA3C0EE66ECE0EE66E99
:10E7B000000E61DA0F0EF66E000EF76E000E00DB33
:10E7C000100EF66E000EF76E000EFADA0E0EE66E02
:10E7D00018EC8BF041E9F3CFE6FFF4CFE6FFF8DA6F
:10E7E00077DA00011051111112110EE010C0E6FF8E
:10E7F00011C0E6FF12C0E6FF08EBE6FF09EBE6FFFB
:10E8000019EC43F045E9AADA0750E66EE66A350EE0
:10E81000E66ECE0EE66E000E2CDA300EE66ECE0EF2
:10E82000E66E000EE66ED4DABADA59EC43F048E947
:10E8300095DAF1DAA1EC90F0E66EE66A220EE66E69
:10E84000CE0EE66E000E17DAE6DA0B01CE51E66E5A
:10E85000E66A140EE66ECE0EE66E000E0CDA0B01C2
:10E86000CF5173DA0B01D05170DAD5DAE66AE66A75
:10E87000200EE66E410EE66ED2EC90F04ADAFFC052
:10E88000D4FBFCC0E6FFFDC0E6FFFEC0E6FFFFC014
:10E89000E6FFE7EC61F07EEC5EF0E552E550066ED7
:10E8A000E750056E010EE66EE66A05EBE6FF06EB45
:10E8B000E6FFE66AE66A020EE66ECE0EE66E000E31
:10E8C0008DDA7AEC44F04BE949DAFE0EE66ECD0EB5
:10E8D000E66E000EB0D90001F051E66EE66AF00E69
:10E8E000E66ECD0EE66E000EC6D995DA0001CB516C
:10E8F000E66EE66AE20EE66ECD0EE66E000EBBD95F
:10E90000DF0EE66ECD0EE66E000E95D9930EE66E26
:10E91000000EE66ED10EE66ECD0EE66E000E5EDAED
:10E920004DEC43F047E91ADA950EE66E0B0EE66EF3
:10E93000CE0EE66ECD0EE66E000ECAD9CB0EE66E9A
:10E94000CD0EE66E000E77D900017851E66EE66ACC
:10E95000BD0EE66ECD0EE66E000E8DD979C0E6FFD7
:10E960007AC0E6FFB90EE66ECD0EE66E000E81D9D6
:10E970007BC0E6FF7CC0E6FFB00EE66ECD0EE66E15
:10E98000000E77D9A30EE66ECD0EE66E000E53D9BB
:10E9900000016651E66EE66A950EE66ECD0EE66EF5
:10E9A000000E69D900016751D0D935DA0501CE359D
:10E9B00010E2CDC5E6FFCEC5E6FF890EE66ECD0EB0
:10E9C000E66E000E58D9110EE66EE66A01DA51D9EC
:10E9D00022DAB5D909DA7F0EE66ECD0EE66E000EAC
:10E9E00003DA750EE66ECD0EE66E000EFDD96D0EE5
:10E9F000E66ECD0EE66E000E40D946E9E7CFD9FFB0
:10EA0000120040D992D909EC7FF042E9F3CFCBF064
:10EA10003CD138D9CDCBCCF50B01010ECD6FD9EC63
:10EA20006AF00501CD6BCE6B590EE66ECD0EE66E2B
:10EA3000000EDED127D9CCC5CDFBD9EC6AF005019B
:10EA4000CD69CE69460EE66ECD0EE66E000ED0D1D3
:10EA500019D91BD117D919D115D917D1CDD984E915
:10EA600044E83CD901E1E3D039D9230801E1DFD002
:10EA700081EB04F082EB05F00CD918E00AD92008EC
:10EA800015E007D960080EE2BCD9EFCFD1FB7B0EB1
:10EA90000B01D15D07E2FDD8E00FE66EB2D9E55279
:10EAA000E750EF6E042A000E0522E6D7F2D82008C0
:10EAB00003E1042A000E0522066A076A0B01FF0E15
:10EAC000D16F1B0ED26F010ED36F34D906EBD7FB7B
:10EAD00007EBD8FBD96BD8BFD969D7CBE6FFD8CB2A
:10EAE000E6FFD9CBE6FF4FD90800F55001E18FD002
:10EAF000FF0ED76F1B0ED86F010ED96F1BD906EB17
:10EB0000DDFB07EBDEFBDF6BDEBFDF69DDCBE6FFA6
:10EB1000DECBE6FFDFCBE6FF36EC61F0E552E5CF7A
:10EB2000DCFBE5CFDBFBE7CFDAFB0B01D751DA25C6
:10EB3000D46FD851DB21D56FD951DC21D66FD4CB1E
:10EB4000E6FFD5CBE6FFE66EEAEC85F043E9E1D8D7
:10EB5000FCC0E6FFFDC0E6FF0B01FF0EE36F1B0EDE
:10EB6000E46F010EE56FE6D806EBE9FB07EBEAFB85
:10EB7000EB6BEABFEB69E9CBE6FFEACBE6FFEBCB59
:10EB8000E6FF36EC61F0E552E5CFE8FBE5CFE7FBC9
:10EB9000E7CFE6FB0B01E351E625E06FE451E72107
:10EBA000E16FE551E821E26FE0CBE6FFE1CBE6FF64
:10EBB000E66E2CD9B4EC84F047E9000924E106EBB9
:10EBC000E9FF07EBEAFF030EEA02F3CFEAFFE902EF
:10EBD000F3CFE9FFF450EA26CF0EE926050EEA222C
:10EBE000EECFD1FBEECFD2FBEFCFD3FB04EBE6FFB2
:10EBF00005EBE6FF0BD9D3CBFBFFD2CBFAFF0B0122
:10EC0000D151140013D0062A000E072257D766D818
:10EC1000530805E176D803E144D863DD07D05ED818
:10EC20004D0805E16ED803E13CD86BDD44E945E9C8
:10EC3000E7CFD9FF1200B3D819EC43F045E98ED8DD
:10EC4000000EE66E070EE66EE3EC02F042E91200FB
:10EC50008AD8D5EF76F0D151D425F36ED251D52193
:10EC6000F46ED351D621F86EF4CFF7FFF3CFF6FF51
:10EC7000120095D8DAD0B2D8D8D0E66E57EC02F0B0
:10EC800043E91200B9D885E9120041E9E7CFD9FF7D
:10EC90001200B7D8EF501200E66EF7EC3DF041E9F4
:10ECA0001200020E0124D16F000E0220D26FD1CBD0
:10ECB000E6FFE66E06EF77F0010EE66ED9EC8BF01C
:10ECC00042E9E66AE66AD9EC8BF042E900EF8CF0A3
:10ECD00066D84DEC43F047E9AEEF76F001EBE9FF83
:10ECE00002EBEAFFEF5012000601FB150B01D26F99
:10ECF000D151D2111200F86E0800F550E66EE66AA6
:10ED000012000128E96E000E0220EA6EEF50200882
:10ED10001200FCC0D1FBFDC0D2FBFEC0D3FB120031
:10ED20000601FA150B01D16F120000EBE6FF01EBB3
:10ED3000E6FF12001B0EE66EE66AE66A1200BD0EE2
:10ED4000E66ECE0EE66E000E1200E66EE66A100E5D
:10ED5000E66ECE0EE66E000E39EF76F0F350086EDA
:10ED6000F450096E1200660ED16F1B0ED26F010EA9
:10ED7000D36FCDC5D7FBCEC5D8FB090ED803F3CFD3
:10ED8000D8FBD703120036EC61F0E552E5CFD6FB95
:10ED9000E5CFD5FBE7CFD4FB0B012BEF76F0E66E8A
:10EDA00008EBE6FF09EBE6FF1200F450D82703500A
:10EDB000032AF324D46F000ED821D56FD66B12002E
:10EDC0009ADF3A0EE66ECE0EE66E000E39EF76F062
:10EDD000380EE66ECE0EE66E000E1200E66E000EE7
:10EDE000E66E070EE66E120048DF050E4CEF76F079
:10EDF00044DF020E51DF49D7D9CFE6FFE1CFD9FF7B
:10EE0000120004EBE9FF05EBEAFF120001EBE6FF5D
:10EE100002EBE6FF120093DF1BEF76F033DF8FDFAC
:10EE20003DEF76F018DF080012006DEC43F047E983
:04EE3000AEEF76F0DB
:0CEE3400010E0001E76EC41902E7C435AE
:10EE400002D0C451E75C02E3000E01D0010E0001C4
:10EE50007393E8B073830A017251000808E27207E5
:10EE600006E1736B0001606B616B0001626B0A016C
:10EE70007151000814E271070CE100017391000167
:10EE8000719F00017599AADB0AE18EDB020EACDBF3
:10EE900006D0000173810001718F000175890001A6
:10EEA000882B000E89238A238B230A01FF0E7519F4
:10EEB0000AE1765108E1745100080DE274070BE194
:10EEC000010E736F08D0050E745D01E2742B050E00
:10EED000745D01E1736B4B0E00010F5D11E19DDB71
:10EEE000D2350BE2D151C808000ED25506E295DBAF
:10EEF000FF0ED15F000ED25B25D077CA77F024D009
:10EF00008CDBD23519E2D151C808000ED25514E27B
:10EF100077CAD5FBD66BD76BD86BFF0ED55F000ECB
:10EF2000D65BD75BD85BD5CBE6FFD6CBE6FFD7CB9E
:10EF3000E6FFD8CBE6FF05D077CAE6FFE66AE66AC9
:10EF4000E66A40DBD1CB77F00A0EE66EE66AE66A47
:10EF5000E66A78CAE6FF79CAE6FF7ACAE6FF7BCAA4
:10EF6000E6FF96EC61F0DDEC3EF044E9FCC0BBF05E
:10EF7000FDC0BCF0FEC0BDF0FFC0BEF00A01735181
:10EF800028E0000178510A0804E300017B6B7C6BE8
:10EF900047D0140E785D05E20A01140E946F080E36
:10EFA000956F0A0E0A01945DE66EE66A0A0E00018C
:10EFB000785DE66EE66A0A019551E66EE66A02EC55
:10EFC00061F092EC5FF0E552E5CF7CF0E7CF7BF0AB
:10EFD00027D0FF0E751901E1765114E04B0E0001A8
:10EFE0000F5D0CE175CAE6FF76CAE6FFE66AE66ADF
:10EFF000E9DAFCC07BF0FDC07CF004D075CA7BF080
:10F0000076CA7CF0140E0001785D0AE30001050E5B
:10F010007B5D000E7C5904E378C094FA7BC095FABE
:10F02000000178510A0804E30001796B7A6B1BD068
:10F03000640EE66EE66A680EE66EE66A78510B01CB
:10F04000D16FD26B0A0ED15F000ED25BD1CBE6FF3F
:10F05000D2CBE6FF02EC61F092EC5FF0E552E5CF37
:10F060007AF0E7CF79F00A01735109E100016251AA
:10F0700069E0000160516408000E615563E200011F
:10F080007589000171B71FD0718971877185000181
:10F09000686B0001010E666F0001030E676F0A01C5
:10F0A000735103E000017D0E02D00001100E636F6A
:10F0B0000001646B656B00016A6B6B6BC2DA8EDA00
:10F0C00068E172DA66D071850A016C2B3C0E6C5DCA
:10F0D00062E36C6B0001642B000E65230A0173511F
:10F0E0005AE160C0E6FF61C0E6FF00016251E66ED2
:10F0F000E66A02EC61F0E552E5CFD2FBE7CFD1FB47
:10F100000B01D1510A016D270B01D2510A016E2367
:10F11000000E6F237023600E6D5DEA0E6E59000EB7
:10F120006F59000E705937E30A0E00016A27000E6E
:10F130006B23600E0A016D5FEA0E6E5B000E6F5B63
:10F14000705B000C0001625126E10001640E605DFD
:10F15000000E615920E20A0173511DE1000171A7FF
:10F160001AD0719971977195000175995F0E000120
:10F17000785D06E20001150E666F00010E0E05D0E7
:10F180000001040E666F0001030E676F040E2CDA97
:10F1900058DA020E29DA000C46DA44E8036A046AF7
:10F1A000016A026A180ED89002BE03D0015C000EFC
:10F1B000025811E27C0E0124E96E0A0E0220EA6E6A
:10F1C000EF50F46AE8BEF4680326F4500422012AE2
:10F1D000000E0222E7D7180EE66EE66A03EBE6FFA2
:10F1E00004EBE6FF4AEC5FF0E552E5CFAAF0E7CF8B
:10F1F000A9F0000E45E9E7CFD9FF12000A013C0E45
:10F20000716F890E0001021902E1030E03192DE04E
:10F21000740E021902E1030E031913E0460E0219DF
:10F2200036E1030E031933E100010D510A01756F38
:10F23000766B73512CE0FF0E751929E1765127E1A9
:10F2400024D0020EE66EE66A000107510B01426F00
:10F25000436B0A0E425F000E435B42CBE6FF43CB9B
:10F26000E6FFE7D940CB78F0010C0001075100011F
:10F27000606F616B0A0EE66EE66A00010C51E66E85
:10F28000E66AD7D940CB62F00A011E0E726F010CFC
:10F29000CAD943E80A013C0E716FE10E0001021960
:10F2A00002E1060E031901E1B6D0120E021902E1C5
:10F2B000040E03196DE09A0E021902E1020E031901
:10F2C00044E0980E021902E1020E031934E0860EA2
:10F2D000021902E1020E031923E0850E021901E072
:10F2E000D3D0020E031901E0CFD00C0E00010C5D4B
:10F2F00007E10001718D72D901E0C6D055D90DD05A
:10F300000E0E0C5D01E0C0D00001719D67D901E1D6
:10F31000BBD08C6B8D6B8E6B8F6B020E65D9B4D0AE
:10F32000280E0001095D0001A56FA66B800B01E1AD
:10F33000A8D0A669A6D0000109510001A76FA86B4B
:10F34000280EA75F000EA85B9CD00001065109E1C2
:10F35000016A070E015C01E397D056D901504AD9E2
:10F36000F8D706050AE1016A070E015C01E38CD0BB
:10F370004BD9070E01243ED9F7D7020E065D01E0F6
:10F3800083D007C0A1F008C0A2F009C0A3F07CD0D0
:10F3900007C077FA08C044FB0B01456B466B476B0F
:10F3A000100E1F0B08E00B01D89044374537463745
:10F3B0004737E806F9E109C048FB0B01496B4A6B86
:10F3C0004B6B080E1F0B08E00B01D89048374937EC
:10F3D0004A374B37E806F9E10B01485144274951B8
:10F3E00045234A5146234B5147230AC04CFB4D6BE2
:10F3F0004E6B4F6B4C5144274D5145234E51462384
:10F400004F51472344CB78FA45CB79FA46CB7AFA69
:10F4100047CB7BFA39D000010651026E036A010E18
:10F42000025C000E035830E302500C08000E035437
:10F430002BE30B01D8900234446F0334456F020E66
:10F44000445D026E000E4559036E320E0001085DE8
:10F45000E66E7C0E0224E96E0A0E0320EA6EE55287
:10F46000E750EF6E320E095DE66E0228E96E000E7F
:10F470000320EA6E7C0EE9260A0EEA22E552E750E6
:10F48000EF6E00013C0EC46F010E44E9E7CFD9FFD7
:10F490001200C9D843E80B014D0E956F490E966FC7
:10F4A000976B986B996B0001C7690001C46B0001F1
:10F4B000886B896B8A6B8B6B00018C6B8D6B8E6B91
:10F4C0008F6B00010F0EEF6F0A01716B726B736B24
:10F4D000050E746F756B766B776B786B796B7A6BE7
:10F4E0007B6B036A180E035C09E20350EA6A7C0F27
:10F4F000E96E0A0EEA22EF6A032AF4D7900E6F6EC5
:10F500006EAEFED7606A0F01196BE00E186F016BCB
:10F51000680E006F200E056F710E046F506B800E29
:10F520001D6F1C69096F500E086F400E0D6F820E23
:10F530000C6F200E116FDC0E106F156B530E146FD5
:10F54000010E706ED20E716E020E726E200E736E10
:10F550000B01CD51000802E26F6A02D0600E6F6E9F
:10F560000001FC0E196FF10E1A6F000E1B6F0001E7
:10F57000900E1C6FF20E1D6F000E1E6F0001340EF8
:10F580001F6FEE0E206F000E216F0001980E226F8C
:10F59000F10E236F000E246F0601EE81EE83010E43
:10F5A00044E9E7CFD9FF120088C08CF089C08DF004
:10F5B0008AC08EF08BC08FF08C07000E8D5B8E5B47
:10F5C0008F5B1200DDEC3EF044E9FCC0D1FBFDC0D6
:10F5D000D2FBFEC0D3FBFFC0D4FB120000018C5154
:10F5E0008D118E118F111200E66EE66AA9EC03F000
:10F5F00042E91200EA6A930FE96E000EEA22E55230
:10F60000E750EF6E012A12000128EA6A060FE96E40
:10F61000000EEA22EF50E66E12000A0177510B014C
:10F62000D16FD26B1200D9CFE6FFE1CFD9FF81E9CC
:10F63000120092EC5FF0E552E5CF41FBE7CF40FBD3
:10F6400012000A016C6B6D6B6E6B6F6B706B12004E
:10F6500028DB81E941E8016A060E015C10E20150F5
:10F66000220DF3CFE9FFF4CFEAFF000EE926050EE5
:10F67000EA22EF5002E1015003D0012AEDD7FF0E3C
:10F6800042E9E7CFD9FF12000CDB82E944E80B0125
:10F69000CFBF03D00B01500ED06F00EBF0F0000194
:10F6A000F051200A2BE0300A54E10B01CFBF03D008
:10F6B0000B01510ED06FCCDF0001F96FE83404E28A
:10F6C000020E0B01CB1504E10001010EF06F47D0D3
:10F6D000FEDAD1BFD2699FDAF4DA720E83DA3BDB4D
:10F6E000BBC0EEFFBCC0EEFFBDC0EEFFBEC0EEFF74
:10F6F0001BDB150EC1DA160EAADA2BD00B01CFBF19
:10F7000003D00B01520ED06FA3DF0001F96FE83474
:10F7100004E2040E0B01CB1509E10001020EF06FAB
:10F720000B01CFBF1CD00B01530E18D0D0DAD1BFC4
:10F73000D26971DAC6DA680E55DA2BDBF5DACCDA83
:10F7400062C0EFFFF1DA0D0E97DA0E0E80DAE5C037
:10F75000FBF00B01CFBF03D00B01500ED06F45E97A
:10F76000E7CFD9FF12009DDA81E942E80B01CFBF54
:10F7700003D00B01540ED06F0001F051300A01E1AB
:10F78000DBD0100A63E0300A16E0110A0BE0030A2E
:10F7900009E0020A01E0DBD0000171BF12D071B9AB
:10F7A0005BD052D000017151100B4EE07151800BB3
:10F7B00001E0CDD049D0F93504E2020E0B01CB15A2
:10F7C00002E1010EC1D0000171BFC1D00B01CFBF5A
:10F7D00003D00B01550ED06F7ADAD1BFD269DFDAD0
:10F7E0007FDA440E22DAEE5000018B590B0147DA22
:10F7F000C0D95CDAB7DABDD90D0EA3DABAD9ABDA63
:10F80000EE500001BB5D0B01D16FEE500001BC5901
:10F810000B01D26FEE500001BD590B01D36FEE50BA
:10F820000001BE590B01D46FA4D995DAD1CBEEFFFC
:10F83000D2CBEEFFD3CBEEFFD4CBEEFF9AD9180E8E
:10F840009ADA97D9190E03DA300E7ED0F93504E230
:10F85000040E0B01CB1502E1020E76D038DAD1BFCF
:10F86000D2699DDA86D922DAEECFD1FBEFCFD2FB77
:10F87000000160510B01D15D000161510B01D259B2
:10F8800002E277D986DA75D927DAEF500001D880FD
:10F89000625504E26ED920DA62C0EFFF00017151B7
:10F8A000100B09E07151800B06E10001E53541E3E1
:10F8B0000001FB353EE20B01CFBF03D00B01560E1A
:10F8C000D06F0EDA430EB1D9D36FEE5000018B59D1
:10F8D0000B01D46FD4D90001FB3502E2050E02D032
:10F8E00000016851E66E45D9E552E750EF6E040E0F
:10F8F0000001665D03E159DAEF6A0AD0030E0001E8
:10F90000675D03E152DA010E02D04FDA020EEF6EAC
:10F9100030D9100E30DA2DD9110E99D92AD9130EFB
:10F9200069DAD7C0EEFFD8C0EDFF300EE66EACDE70
:10F9300041E9E5C0FBF00BD0000171AF02D0100E21
:10F9400003D071A904D0200EE66E9EDE41E943E9A2
:10F95000E7CFD9FF12000001FA511200A2D981E9C4
:10F9600045E80B01CFBF03D00B01570ED06F036AE0
:10F97000060E035C63E20350220D000EF324046EB6
:10F98000050EF420056E1CDAEF50440825E1020E46
:10F990000B01CB1521E0F0D8F00EE66ECF0EE66E2F
:10F9A000000EA3D924DA0D0E25DADCD8EDD9010E2C
:10F9B0007FD9D1D9D7D8DEEC44F04BE9FCD9B4D902
:10F9C000150EBCD9160E1FDA180EB8D9190EF0D9BB
:10F9D00003DA72D9640E2BD0F3D9EF5043082CE12F
:10F9E000040E0B01CB1528E0C7D8D70EE66ECF0E5C
:10F9F000E66E000E7AD902DAB1D86ED9E8D96ED99E
:10FA0000E6D90D0E9BD90E0EFED9100E97D9A3D9AB
:10FA1000F5D9E2D9D0D9020E4BD9130EC9D9E66A6D
:10FA2000E66A85D97AEC44F04BE946D9630EEF6E6D
:10FA30000001010EFA6F04D0032A9AD70001FA6B75
:10FA400046E9E7CFD9FF12002CD981E943E80B0141
:10FA5000CFBF03D00B01580ED06F0001FA6B016AC3
:10FA6000060E015C14E2015012D9440A0CE0070AA8
:10FA70000AE0270A05E0070A08E16FD9430E02D021
:10FA80006CD9440EEF6E0001FA2B012AE9D744E944
:10FA9000E7CFD9FF120005D982E942E80B01CFBFB9
:10FAA00003D00B01590ED06FD89018E2060E005CFF
:10FAB00015E20050ECD8640804E04FD9EF50630819
:10FAC0000DE1220EE66EE66AE66A02EBE6FF03EB64
:10FAD000E6FFFEEC84F045E940D9EF6A43E9E7CF61
:10FAE000D9FF120012001200CC0EE66EE66AE66A3A
:10FAF000000EE66E050EE66EFEEC84F045E9E66A61
:10FB0000C3DD41E912000001F72B000EF823F45188
:10FB1000000810E2F5C0D1FBF6C0D2FBF507000EDD
:10FB2000F65B0B01D151D21105E1F4C0E6FFACDD6B
:10FB300041E901D018DE3C0EE66EE66A8ED801E19E
:10FB4000D1DF100EE66E0E0EE66E87D806E1CBDF33
:10FB5000100E0001F75F0E0EF85B12003DD92BD995
:10FB600094EF7EF04BD9EECFE6FFEECFE6FF97EFB6
:10FB70007EF005D9070E29D10350E66EE66A000E25
:10FB8000E66ED00EE66E000EE66E000EE66E070E16
:10FB9000E66E6DEC43F047E939D9EE520001885129
:10FBA000EE5C0B01D16F00018951EE580B01D26F51
:10FBB00000018A51EE580B01D36F00018B51EE58B2
:10FBC0000B01D46FD1CBE6FFD2CBE6FFD3CBE6FF60
:10FBD000E66EADD886EC43F049E9EDD8000EE66E4E
:10FBE000E66A1200EF6EECD8EE5288C0EEFF89C0D4
:10FBF000EEFF8AC0EEFF8BC0EEFF96D868C0EFFF25
:10FC000093D8EE52AFD890D8050E9BD894EF7EF0E3
:10FC1000BBD894EF7EF0220ED203F3CFD2FBD103F8
:10FC2000F450D227000EF3241200EF6EA8D8EE5243
:10FC3000EE500001885D0B01D16FEE500001895933
:10FC40000B01D26FEE5000018A590B011200D2D87D
:10FC500079C0EEFF7AC0EDFF1200F7C0E6FFF8C0F2
:10FC6000E6FF95EC5FF0E552E5CFD2FBE7CFD1FBA5
:10FC70000B01D151D21112007ED894EF7EF07FD8C3
:10FC8000050EB8D8D1CBEEFFD2CBEDFF1200220D7E
:10FC9000000EF324026E050EF420036E5ED8EF50C2
:10FCA0001200D9CFE6FFE1CFD9FF1200090E8DD0A7
:10FCB000E66EE66A94EF7EF07ED86FEC12F0E0EF2D
:10FCC0007EF0046E050ED221056EE0EF7EF0F9C0E5
:10FCD000D1FB0B01D26B12000B0E77D00C0E75D03E
:10FCE0000001F969FA2BBFEF7EF07BD86DEC43F091
:10FCF00047E961D8E60EE66ECF0EE66E000E71D8CB
:10FD000019EC43F045E982D8EE522CDF86EC43F043
:10FD100049E97CD8050E77D85AD8EE5268D8050E36
:10FD200069D865D856EF7EF04BD8070E4ED0FE0E40
:10FD3000E66ECF0EE66E000EF1EF7EF05BD8E7EFD9
:10FD40007EF058D89ECBEEFF9FCBEEFFA0CBEEFF10
:10FD5000A1CBEEFF1200110E38D002EBE9FF03EB4E
:10FD6000EAFF12009ACBEEFF9BCBEEFF9CCBEEFF9F
:10FD70009DCBEEFF12003ED878C0EFFF120001EBE2
:10FD8000E9FF02EBEAFF12006DEC45F049E9DBEF19
:10FD90007EF08CDF60C0EEFF61C0EDFF12003BDF44
:10FDA000016E050ED221026E1200E3DE6EEF7EF0D0
:10FDB00021D8FEEF7EF0F350016EF450026E120077
:10FDC00004EBE9FF05EBEAFF1200FAEF7EF0EF50DB
:10FDD000E66EE66AAEEF7DF0AADF6DEC43F047E930
:10FDE0001200E66E01EBE6FF02EBE6FF1200BADE60
:10FDF00008EF7EF0E926000EEA221200EECFE6FFC1
:10FE0000EECFE6FF1200D4DFAEEF7DF0D4DFE0EFFF
:02FE10007EF082
:0EFE1200FF0EE3CFEAFFE552FF0EE3CFE9FF5C
:10FE2000E552E66AE66AD9CFE6FFDACFE6FFFC0ED6
:10FE3000E124D96EFF0EE220DA6EE66AE66AE66A2F
:10FE4000200EEF5C06E0090EEF5C03E0EF6603D0E6
:10FE50003FD0EE50F5D72D0EEF5C03E1FF0EE32A05
:10FE600003D02B0EEF5C01E1EE502F0EEF6424D097
:10FE70003A0EEF6021D0D890F90EE336FA0EE33651
:10FE8000FD0EDECFE3FFFE0EDDCFE3FFD890F90ECF
:10FE9000E336FA0EE336D890F90EE336FA0EE3367F
:10FEA000FD0EE350DE26FE0EE350DD22300EEE5C4A
:10FEB000DE26000EDD22D9D7FF0EE3CFE8FFE852A1
:10FEC00007E0F90EE31EE32AFA0ED8B4E306E31EB8
:10FED000E552E552E552FF0EE3CFDAFFE552FF0EA1
:10FEE000E3CFD9FFE552E1CFE9FFE2CFEAFFED52E0
:10FEF000ED52EECFF3FFEFCFF4FF1200FF0EE3CF92
:10FF0000EAFFE552FF0EE3CFE9FFE552E66AE66A53
:10FF1000E66AE66AD9CFE6FFDACFE6FFFA0EE12419
:10FF2000D96EFF0EE220DA6EE66AE66AE66AE66AF3
:10FF3000E66A200EEF5C06E0090EEF5C03E0EF6678
:10FF400003D06BD0EE50F5D72D0EEF5C03E1FF0E22
:10FF5000E32A03D02B0EEF5C01E1EE502F0EEF648D
:10FF600044D03A0EEF6041D0D890F50EE336F60E4D
:10FF7000E336F70EE336F80EE336FB0EDECFE3FF93
:10FF8000FC0EDECFE3FFFD0EDECFE3FFFE0EDDCF86
:10FF9000E3FFDD52DD52D890F50EE336F60EE33680
:10FFA000F70EE336F80EE336D890F50EE336F60E8C
:10FFB000E336F70EE336F80EE336FB0EE350DE26AB
:10FFC000FC0EE350DE22FD0EE350DE22FE0EE35077
:10FFD000DD22DD52DD52300EEE5CDE26000EDE222A
:10FFE000DE22DD22DD52DD52B9D7FF0EE3CFE8FF7E
:10FFF000E85213E0F50EE31EF60EE31EF70EE31EC5
:020000040001F9
:10000000F80EE31EF50EE32A08E1F60EE32A05E1F9
:10001000F70EE32A02E1F80EE32AE552E552E55233
:10002000E552E552D9CFE9FFDACFEAFFEECFFCF097
:10003000EECFFDF0EECFFEF0EFCFFFF0FF0EE3CFFF
:10004000DAFFE552FF0EE3CFD9FFE552E552E55264
:100050001200D9CFE6FFDACFE6FFFA0EE3CFD9FFE1
:10006000FB0EE3CFDAFFFD0EE35209E72D0EDE6E45
:10007000FC0EE31EE32AFD0ED8B4E306E31EE652AF
:10008000E652E652FD0EE124E76EFF0EE220E46E3A
:10009000E652F70EE3CFE6FFF70EE3CFE6FF99EC6B
:1000A00080F0F90EE124E96EFF0EE220EA6E89ECA1
:1000B00080F00AE186EC80F009E189EC80F008E14B
:1000C00086EC80F007E108D094EC80F08FEC80F0B3
:1000D00094EC80F08FEC80F094EC80F0DE6AF90E06
:1000E000E126FF0EE222FF0EE3CFDAFFE552FF0E1C
:1000F000E3CFD9FFE552FC0EE124E96EFF0EE220CA
:10010000EA6EEECFF3FFEFCFF4FF1200EF380F0BE4
:100110001200EF500F0B02E1EE52D8841200EF38BC
:100120000F0B300FDE6E1200EE500F0B300FDE6E35
:100130001200FC0EE3CFE9FFFD0EE3CFEAFF100E45
:10014000E66EEE6AEE6AEF6AD890FD0EE336FE0EBA
:10015000E336ED36ED36EF36FF0EE30609E0BAEC96
:1001600080F0EE52BAEC80F0EE52BAEC80F0EDD7AF
:10017000E56E1200030EEF24E8B6EF6E300EEF24AA
:10018000E8BEEF6E000CD9CFE6FFDACFE6FFF80E3F
:10019000E3CFD9FFF90EE3CFDAFFFD0EE35215E707
:1001A0002D0EDE6EFA0EE31EFB0EE31EFC0EE31EAA
:1001B000FD0EE31EFA0EE32A08E1FB0EE32A05E139
:1001C000FC0EE32A02E1FD0EE32AE652E652E65275
:1001D000E652E652FB0EE124E76EFF0EE220E46EEB
:1001E000E652F30EE3CFE6FFF30EE3CFE6FFF30EA6
:1001F000E3CFE6FFF30EE3CFE6FF60EC81F0F50E10
:10020000E124E96EFF0EE220EA6E4DEC81F019E187
:1002100050EC81F018E14DEC81F017E150EC81F0E9
:1002200016E14DEC81F015E150EC81F014E14DEC5C
:1002300081F013E150EC81F012E14DEC81F011E11D
:1002400012D056EC81F05BEC81F056EC81F05BEC67
:1002500081F056EC81F05BEC81F056EC81F05BECC8
:1002600081F056EC81F05BEC81F0DE6AF50EE12660
:10027000FF0EE222FF0EE3CFDAFFE552FF0EE3CFDF
:10028000D9FFE552FA0EE124E96EFF0EE220EA6E94
:10029000EECFF3FFEFCFF4FF1200EF380F0B120099
:1002A000EF500F0B02E1EE52D8841200EF380F0B23
:1002B000300FDE6E1200EE500F0B300FDE6E1200AC
:1002C000FA0EE3CFE9FFFB0EE3CFEAFF200EE66E66
:1002D000EE6AEE6AEE6AEE6AEF6AD890FB0EE336DB
:1002E000FC0EE336FD0EE336FE0EE336ED36ED365C
:1002F000ED36ED36EF36FF0EE3060FE08FEC81F0C2
:10030000EE528FEC81F0EE528FEC81F0EE528FECDA
:1003100081F0EE528FEC81F0E1D7E56E1200030E12
:10032000EF24E8B6EF6E300EEF24E8BEEF6E000C5F
:10033000FE0EE3CFFEF4FF0EE3CFFFF41200350E06
:10034000E66E450EE66EFEC4E6FFFFC4E6FF02EC75
:1003500061F0E552E5CFFFF4E7CFFEF40401FE2B98
:10036000E86AFF23FF9FFEC4F3FFFFC4F4FF1200FF
:10037000D9CFE6FFDACFE6FFF80EE3CFD9FFF90ECB
:10038000E3CFDAFFE652E652E652E652E652FB0EC1
:10039000E124E76EFF0EE220E46EE652F30EE3CFB7
:1003A000E6FFF30EE3CFE6FFF30EE3CFE6FFF30E37
:1003B000E3CFE6FF60EC81F0F50EE124E96EFF0E7D
:1003C000E220EA6E2AEC82F019E12DEC82F018E1CD
:1003D0002AEC82F017E12DEC82F016E12AEC82F093
:1003E00015E12DEC82F014E12AEC82F013E12DEC02
:1003F00082F012E12AEC82F011E112D033EC82F0AB
:1004000038EC82F033EC82F038EC82F033EC82F09E
:1004100038EC82F033EC82F038EC82F033EC82F08E
:1004200038EC82F0DE6AF50EE126FF0EE222FF0EC6
:10043000E3CFDAFFE552FF0EE3CFD9FFE552FA0E24
:10044000E124E96EFF0EE220EA6EEECFF3FFEFCF7C
:10045000F4FF1200EF380F0B1200EF500F0B02E108
:10046000EE52D8841200EF380F0B300FDE6E120000
:0A047000EE500F0B300FDE6E12008D
:06047A0021DA87E90B0105
:100480004ADAE840E8403F0BCDD9E66E24DA31DAAB
:1004900042DA030B100D042805DAF00BE8380F0BD5
:1004A000F310C0D9E66E0228E2D923DA01341EE245
:1004B00000500108000E015419E2EDD90428F2D9C8
:1004C0000F0B040DF3CFD7FB060ED86F020E0424DA
:1004D000E9D9C00BD8CBE7FFE75204E0E8427F0B35
:1004E000E706FCE10B01D7119DD901D03D0EE66E68
:1004F00019DAFFD901340CE200500208000E015451
:1005000007E2C9D9020E0424CDD93F0B8BD901D003
:100510003D0EE66E030E0224AAD9E2D1D0D987E9B6
:1005200044E8076A086A096A0A6A0250095C0350CB
:100530000A5829E204500924E96E05500A20EA6E9F
:10054000EF50E66E07EBE9FF08EBEAFFCED9BCD926
:10055000071815E1085013E1030EE66EE66A83D929
:10056000076A086A040ED89008BE03D0075C000E24
:10057000085803E26AD9B9D9F5D7076A086A092A7F
:10058000000E0A22D2D708342EE207500008000ECF
:10059000085429E287EB09F088EB0AF0030ED890A3
:1005A0000ABE03D0095C000E0A580BE2F70E0924BC
:1005B000E96E050E0A20EA6EEF6A092A000E0A2289
:1005C000EDD707EBE6FF08EBE6FF4DD9076A086AAF
:1005D000040ED89008BE03D0075C000E085803E252
:1005E00034D983D9F5D792D9EF6A00EBF3FF01EB49
:1005F000F4FF45E9E7CFD9FF120061D985E944E866
:10060000056A066A076A086A0050075C01500858C4
:1006100028E202500724E96E03500820EA6EEF50EA
:10062000E66E05EBE9FF06EBEAFF052A000E06225F
:100630004BD9051814E1065012E1030EE66EE66A86
:1006400012D9056A066A040ED89006BE03D0055C6E
:10065000000E065802E210D9F6D7056A066A45D997
:10066000D3D7063426E205500008000E065421E2D6
:1006700085EB07F086EB08F0030ED89008BE03D098
:10068000075C000E085804E213D9EF6A2ED9F4D79C
:1006900005EBE6FF06EBE6FFE6D8056A066A040E00
:1006A000D89006BE03D0055C000E065802E2E4D8DE
:1006B000F6D745E9E7CFD9FF120001D985E90BD973
:1006C000EF50040D0228D3D8EF380F0B0B01F310B5
:1006D000E66E1CD90ED926D9EF50E840E8403F0B12
:1006E000D16F0228C4D8EF38F00BD111E66E002884
:1006F000E96E000E0120EA6EFCD8030E0224B7D882
:10070000EFCFD1FB0FD9EF50400DF350C00BD111FB
:10071000E66E020E0024E96E000E0120EA6EE0D0C3
:10072000CED885E948E8010E056E0B6A0C6A0550C3
:100730006FE0096A0A6A076A086A040ED89008BE60
:1007400003D0075C000E085845E2055043E0066AF6
:10075000055030E006502EE1BED8EF5006E0BBD881
:10076000022A000E0322EF5001D0000E056E2B0E60
:10077000055C05E305507A0802E3000E01D0010E86
:10078000000902E0000E0AD00B01550ED16F240EB5
:10079000D26F010ED36F2B0E055C44D8066E065047
:1007A000D7E0240E065C02E1000E02D03D0E065C8E
:1007B000066ECED705500AE0092A000E0A2206501E
:1007C00007E00604E66E74D894D802D071D8EF6AB8
:1007D0008CD8B3D709500A10AAE08FD86EDF44E94D
:1007E000076A086A0B010904D16F000E0A58D26F1C
:1007F000E8340850D21904E6D151075CD2510858A8
:1008000096E223D80B2A000E0C22072A0822EAD7E8
:100810007DD8EF6A0BEBF3FF0CEBF4FF49E9E7CF70
:10082000D9FF1200D46FD56BD66BD151D425F36E9E
:10083000D251D521F46ED351D621F86EF4CFF7FF03
:10084000F3CFF6FF0800F5501200FB0E0724E96E07
:10085000050E0820EA6EEF50E66E58D8002A000E0A
:10086000012279EF84F049D808DE46E91200E96EEA
:10087000000E0320EA6E1200FB0E0524E96E050E41
:100880000620EA6EEFCFE6FF62EC03F041E9052AAD
:10089000000E06221200140ED16F240ED26F010E2C
:1008A000D36F1200E96E000E0520EA6EEF501200C1
:1008B000F70E0724E96E050E0820EA6E1200D9CF64
:1008C000E6FFE1CFD9FF1200F70EE926050EEA2276
:1008D00010D8030E120002EBE9FF03EBEAFF12004F
:1008E00008D841E9E7CFD9FF1200072A000E0822F5
:1008F0001200E552E750EF6E1200FB0EE66E050E99
:10090000E66EF70EE66E050EE66E120000EBE9FFEE
:1009100001EBEAFF1200BFDF04EBE9FF05EBEAFFA2
:0C092000EF501200020E022437EF84F0AA
:04092C00FE0EE3CF09
:10093000E9FFFF0EE3CFEAFFFB0EE35003E1FC0EFD
:10094000E3500FE0FB0EE30602E2FC0EE306FD0EB1
:10095000E350EE5CF1E1ED52E9CFF3FFEACFF4FFB3
:1009600002D0F36AF46A1200FB0EE3CFF6FFFC0E2E
:10097000E3CFF7FFFD0EE3CFF8FFFE0EE3CFE9FF75
:10098000FF0EE3CFEAFFF90EE35003E1FA0EE35066
:1009900009E0F90EE30602E2FA0EE3060900F5505B
:1009A000EE5CF1E01200D9CFE6FFDACFE6FFFA0EF7
:1009B000E3CFD9FFFB0EE3CFDAFFFC0EE3CFE9FF75
:1009C000FD0EE3CFEAFFE9CFF3FFEACFF4FFF80E25
:1009D000E35003E1F90EE35008E0F80EE30602E20B
:1009E000F90EE306DECFEEFFF2D7FF0EE3CFDAFF1C
:1009F000E552FF0EE3CFD9FFE5521200FE0EE3CF22
:100A0000E9FFFF0EE3CFEAFFE9CFF3FFEACFF4FF00
:100A1000FB0EE35003E1FC0EE35009E0FB0EE3069E
:100A200002E2FC0EE306FD0EE350EE6EF1D712007B
:100A3000D9CFE6FFDACFE6FFFA0EE3CFD9FFFB0E00
:100A4000E3CFDAFFFC0EE3CFE9FFFD0EE3CFEAFFD1
:100A5000E9CFF3FFEACFF4FFEE66FED7ED52DFCF2A
:100A6000EEFFDE66FCD7FF0EE3CFDAFFE552FF0EA6
:100A7000E3CFD9FFE5521200FB0EE3CFF6FFFC0EE9
:100A8000E3CFF7FFFD0EE3CFF8FFFE0EE3CFE9FF64
:100A9000FF0EE3CFEAFFE9CFF3FFEACFF4FFEE6604
:100AA000FED7ED520900F5CFEFFFEE66FBD712003F
:100AB000FE0EE3CFE9FFFF0EE3CFEAFFFD0EE350AA
:100AC000EF5C05E0EE66FAD7F36AF46A04D0E9CF8A
:100AD000F3FFEACFF4FF1200D9CFE6FFDACFE6FF4B
:100AE000FA0EE3CFD9FFFB0EE3CFDAFFFC0EE3CF24
:100AF000E9FFFD0EE3CFEAFFDE50EF5C02E1EE66B8
:100B0000FBD7F36EFF0EE3CFDAFFE552FF0EE3CF24
:100B1000D9FFE552F3501200FB0EE3CFF6FFFC0EB7
:100B2000E3CFF7FFFD0EE3CFF8FFFE0EE3CFE9FFC3
:100B3000FF0EE3CFEAFF0900F550EF5C02E1EE663D
:100B4000FAD71200D9CFE6FFDACFE6FFFA0EE3CFED
:100B5000D9FFFB0EE3CFDAFFFC0EE3CFE9FFFD0E7A
:100B6000E3CFEAFFE9CFF3FFEACFF4FFDECFEFFFF9
:100B7000EE66FCD7FF0EE3CFDAFFE552FF0EE3CFC0
:100B8000D9FFE5521200FB0EE3CFF6FFFC0EE3CFD8
:100B9000F7FFFD0EE3CFF8FFFE0EE3CFE9FFFF0EF8
:100BA000E3CFEAFFE9CFF3FFEACFF4FF0900F5CF87
:100BB000EFFFEE66FBD71200FE0EE3CFE9FFFF0E5C
:100BC000E3CFEAFFF36AF46AEE5203E0F34AF42A51
:100BD000FBD71200FF0EE3CFF8FFE552FF0EE3CF85
:100BE000F7FFE552FF0EE3CFF6FFE552E66AE66A4D
:100BF000E66A0900F55209E0FD0EE32A05E1FE0E62
:100C0000E32A02E1FF0EE32AF4D7FD0EE3CFFCF066
:100C1000FE0EE3CFFDF0FF0EE3CFFEF01200D9CFC2
:100C2000E6FFDACFE6FFFA0EE3CFD9FFFB0EE3CF04
:100C3000DAFFFC0EE3CFE9FFFD0EE3CFEAFFF80E8B
:100C4000E35003E1F90EE3500AE0F80EE30602E296
:100C5000F90EE306DE50EF5C02E1EE66F0D7F36ECC
:100C6000FF0EE3CFDAFFE552FF0EE3CFD9FFE552E7
:100C7000F3501200D9CFE6FFDACFE6FFFA0EE3CF4A
:100C8000D9FFFB0EE3CFDAFFFC0EE3CFE9FFFD0E49
:100C9000E3CFEAFFE9CFF3FFEACFF4FFF80EE3502A
:100CA00003E1F90EE3500BE0F80EE30602E2F90E61
:100CB000E306DECFEFFFEE66F1D7DD52EFD7FF0E92
:100CC000E3CFDAFFE552FF0EE3CFD9FFE552120082
:100CD000FE0EE3CFF3FFFF0EE3CFF4FFFB0EE3CFF7
:100CE000F6FFFC0EE3CFF7FFFD0EE3CFF8FFF3CFE7
:100CF000E9FFF4CFEAFF0900F5500CE0F550EF5C96
:100D000002E1EE52F8D7EF5203E0F34AF42AE6D7B5
:100D1000F36AF46A1200FE0EE3CFE9FFFF0EE3CFA1
:100D2000EAFFEF5017E0FB0EE3CFF6FFFC0EE3CF38
:100D3000F7FFFD0EE3CFF8FF0900F55003E0EF5C8D
:100D4000FBE103D0EC5006E0EED7E9CFF3FFEACFAA
:100D5000F4FF1200F36AF46A1200FE0EE3CFE9FF1B
:100D6000FF0EE3CFEAFFF36AF46AEF5012E0FB0EE6
:100D7000E3CFF6FFFC0EE3CFF7FFFD0EE3CFF8FF66
:100D80000900F55006E0EF5CFBE1F34AF42AEC5071
:100D9000EEE11200FE0EE3CFE9FFFF0EE3CFEAFF24
:100DA000E9CFF3FFEACFF4FF610EEF5C05E67B0EBF
:0E0DB000EF5C02E7DF0EEF16EE52F6E11200E6
:020DBE0050657E
:100DC000726D697373696F6E2064656E6965640026
:100DD000496E76616C696420636F6D6D616E64004D
:100DE000596F75722070686F6E652068617320623C
:100DF00065656E20726567697374657265642061EC
:100E00007320746865206F776E65722E004D6F6475
:100E1000756C652070617373776F7264206861739D
:100E2000206265656E206368616E6765642E0050A0
:100E30006172616D657465727320686176652062A8
:100E400065656E207365742E004665617475726504
:100E500020686173206265656E207365742E00489A
:100E60006F6D656C696E6B20616374697661746522
:100E7000640056656869636C65206C6F636B2072F3
:100E800065717565737465640056656869636C6542
:100E900020756E6C6F636B20726571756573746518
:100EA000640056616C6574206D6F646520726571B5
:100EB0007565737465640056616C6574206D6F644C
:100EC000652063616E63656C20726571756573740E
:100ED000656400436861726765206D6F64652063B7
:100EE00068616E676520726571756573746564000D
:100EF00043686172676520737461727420726571F2
:100F00007565737465640043686172676520737406
:100F10006F702072657175657374656400436F6FDF
:100F20006C646F776E2072657175657374656400AB
:100F3000436172206C6F636174696F6E3A0A687402
:100F40007470733A2F2F6D6170732E676F6F676CBB
:100F5000652E636F6D2F6D6170733F713D000A6880
:100F60007474703A2F2F6F736D2E6F72673F6D6CB4
:100F700061743D003352454749535445523F000088
:100F800000000000315245474953544552000000CB
:100F90000000000033504153533F000000000000A8
:100FA00000000000325041535320000000000000B8
:100FB0000000000033475053000000000000000014
:100FC00000000000335354415400000000000000B2
:100FD0000000000033504152414D533F00000000DB
:100FE0000000000032504152414D532000000000EB
:100FF000000000003141502000000000000000000F
:1010000000000000334D4F44554C453F00000000A8
:1010100000000000324D4F44554C452000000000B8
:10102000000000003356454849434C453F0000004E
:10103000000000003256454849434C45200000005E
:101040000000000033475052533F000000000000F2
:101050000000000032475052532000000000000002
:10106000000000003347534D4C4F434B3F000000FE
:10107000000000003247534D4C4F434B000000002E
:1010800000000000335345525645523F0000000017
:101090000000000032534552564552200000000027
:1010A00000000000334449414700000000000000F8
:1010B000000000003346454154555245533F00005F
:1010C00000000000324645415455524520000000C2
:1010D0000000000032484F4D454C494E4B00000087
:1010E00000000000324C4F434B00000000000000A5
:1010F0000000000032554E4C4F434B0000000000F2
:10110000000000003256414C455400000000000031
:101110000000000032554E56414C4554000000007E
:1011200000000000324348415247454D4F4445209E
:101130000000000032434841524745535441525445
:10114000000000003243484152474553544F50007D
:101150001111111132434F4F4C444F574E000000B4
:10116000000000003356455253494F4E0000000026
:1011700000000000335245534554000000000000B9
:101180000000000033435450000000000000000045
:10119000000000003354454D505300000000000093
:1011A000000000003348454C5000000000000000E3
:1011B000000000000000000000000000000000002F
:0411C000000000002B
:0C11C400D9CFE6FFE1CFD9FF81E942E876
:1011D000D01C1F0B016EFCAE02D0200E0126FCAC11
:1011E00002D0400E0126D080D082D088FC9EFC9C8C
:1011F000FE0E936E030E015C2EE10BEC3EF00B0134
:10120000CF6B0B01CE6B74EC7DF0026A080E025CB2
:1012100009E20250EA6ABE0FE96E0B0EEA22EF6A9B
:10122000022AF4D70B01D90E9A6FC60E9B6FDE0E01
:101230009C6F160E9D6F0B01360E9E6F4A0E9F6FB0
:10124000440EA06FFE0EA16F0B01A26BA36B0B01EE
:10125000A46BA56B06D0800E01100B01CF6F0B01A4
:10126000CE2B0B01CFBF03D00B01200ED06F080E89
:10127000026E100E025C1BE2080E025C180FE66E96
:1012800018EC8BF041E9F3CFE6FFF4CFE6FF09EC71
:101290007FF042E9F350E66E0250EA6ABE0FE96E53
:1012A0000B0EEA22E552E750EF6E022AE2D7000168
:1012B000E56998EC90F0870ED56E03EC8CF06EEC3F
:1012C0008AF0D9EC6AF03CEC0FF00B01CFBF03D0F1
:1012D0000B01210ED06F0A0EE66EF7EC3DF041E9EE
:1012E000E668E66AD9EC8BF042E9E66A010EE66E42
:1012F000D9EC8BF042E900EC8CF00A0EE66EF7ECCC
:101300003DF041E90E0EF66E000EF76E000EF86E1F
:101310000800F5CFE6FF010EE66ED9EC8BF042E94E
:1013200000EC8CF0230EE66EF7EC3DF041E9040092
:101330000F0EF66E000EF76E000EF86E0800F5CF79
:10134000E6FF010EE66ED9EC8BF042E900EC8CF082
:10135000230EE66EF7EC3DF041E90400100EF66E48
:10136000000EF76E000EF86E0800F5CFE6FF010ED6
:10137000E66ED9EC8BF042E900EC8CF0230EE66EC1
:10138000F7EC3DF041E90400E66A010EE66ED9ECA7
:101390008BF042E9E66AE66AD9EC8BF042E900ECB0
:1013A0008CF00A0EE66EF7EC3DF041E90400E66AC7
:1013B000010EE66ED9EC8BF042E900EC8CF0E66AA7
:1013C000E66A200EE66E410EE66ED2EC90F0FCC0AE
:1013D000D1FBFDC0D2FBFEC0D3FBFFC0D4FBD1CB01
:1013E000E6FFD2CBE6FFD3CBE6FFD4CBE6FFE7ECBC
:1013F00061F045EC5EF041E9E7500001CC6F00017F
:10140000CD6B026A0B01CFBF03D00B01220ED06F50
:10141000090109010051200B05E1090109010051F1
:10142000100B02E0A3EC00F0090100B709D00B019A
:10143000CFBF03D00B01230ED06FC5EC00F0F4D763
:101440000B01CFBF03D00B01240ED06F0AEC0BF0C1
:10145000B7EC6CF00400D650016E4C0ED75C1BE369
:10146000D76AD66A0B01CFBF03D00B01250ED06F10
:10147000DCEC0EF00B01CFBF03D00B01260ED06FBA
:1014800087EC6BF00B01CFBF03D00B01270ED06FA1
:1014900083EC7DF01ED00250D75C1BE0D750030BCD
:1014A00016E10B01CFBF03D00B01290ED06F3BEC2F
:1014B0000FF00B01CFBF03D00B012A0ED06FABECA6
:1014C0006CF00B01CFBF03D00B012B0ED06FD750A8
:0C14D000026E98D743E9E7CFD9FF120065
:0414DC00120029D9F8
:1014E00082E944E8A66A0050046E056A42D904EB1A
:1014F000E6FF05EBE6FF02EC61F0E552E550056E14
:10150000E750046E0B0105EBD1FBD26BD1CBAAFFE8
:10151000FF0E0414A96E026A036A200ED89003BE5F
:1015200003D0025C000E035809E2A68026D9A8CF9A
:10153000EFFFA92A022A000E0322EFD745E9E7CFE1
:10154000D9FF1200F6D882E945E8026A036A005022
:10155000010803E30701C85167E00050056E066A01
:1015600008D905EBE6FF06EBE6FF02EC61F0E55279
:10157000E550066EE750056E0B0106EBD1FBD26B12
:10158000D1CBAAFF026A036A200ED89003BE03D013
:10159000025C000E035848E20B01000ED76F000EEC
:1015A000D86FF00ED96FE5D8E66A00EBE6FFE66A81
:1015B000E66A36EC61F0E552E5CFDCFBE5CFDBFB1C
:1015C000E7CFDAFB0B01D751DA25D46FD851DB21F5
:1015D000D56FD951DC21D66F02EBDDFB03EBDEFBCF
:1015E000DF6BDEBFDF69D451DD25D16FD551DE2140
:1015F000D26FD651DF21D36FD1CBA9FFA66AA684C3
:10160000BCD8EF50A86EF250046EF29E550EA76E35
:10161000AA0EA76EA68204EBF2FFA6B2FED7A6948E
:10162000022A000E0322B0D746E9E7CFD9FF120005
:1016300080D882E90701C86B200E005C06E200EB4F
:10164000E6FF4DDF41E90701E76B0B01C80ED16FE3
:10165000070ED1CBF3FFF46E7ED06BD884E9200E59
:10166000025C12E20050011009E083D88DD891D8B5
:101670003AEC86F046E90701E76B02D00701C86B38
:1016800002EBE6FF5FDF41E966D053D886E942E826
:1016900004EBE6FFCDDF41E9F350066EF450076E30
:1016A0004DD87CD806EBE6FF07EBE6FF90EC83F025
:1016B00044E943E9E7CFD9FF12003BD886E969D86E
:1016C00063D86CD88EEC82F06ED845D032D886E9DB
:1016D00035D8200E045C0FE204EBE6FF00DF41E9A1
:1016E00000502008000E015404E243D82ED837D809
:1016F000F0D74AD82AD82FD01CD886E9200E045C0F
:1017000011E200502008000E015404E232D80BD838
:1017100026D8F4D72ED8E66A3CD8FEEC84F045E90A
:1017200033D801D818D03AD834D8D3EC84F0D3EFDA
:101730008BF0D9CFE6FFE1CFD9FF120025D8E66ABA
:101740002DD8FEEC84F045E9120023D827D8D3EC3D
:1017500084F046E9120041E9E7CFD9FF1200200EDC
:10176000005E000E015A200E0226000E0322042AFB
:101770001200200EE66EE66A1200C80E0224E96E20
:10178000070E0320EA6E120000EBE6FF01EBE6FF16
:101790001200C80EE66E070EE66E120002EBE6FFC0
:1017A00003EBE6FF120046E904EBE6FFCBDE41E97E
:0217B000120025
:0E17B200D9CFE6FFE1CFD9FF83E90150EA6A03
:1017C000F60FE96E070EEA2200EBEFFFFF0E005C5A
:1017D00013E1040E01240B01D16F010ED15304E07B
:1017E000E846FE0BD107FCE182120150EA6AF80FCD
:1017F000E96E070EEA22EF6A41E9E7CFD9FF12004E
:101800000701FA6B1200CF0E821694160701FB6BCC
:10181000FC6BB50ECD6E9F909D80CE6ACF6A120094
:101820009EA098D0080E0601EE15000821E2B60E23
:101830000701FB27120EFC23FBC7CAF8FCC7CBF835
:101840000801CC6BD890CC51000A06E6710ECA5D37
:10185000B20ECB59000ECC590BE3710E0701FB5FA2
:10186000B20EFC5B0001882B000E89238A238B2398
:101870000701FA3502E3FA2B6CD0FA5127E10B018C
:10188000FF6B020EFF5D1FE274D8E66E6BD8E55267
:10189000E750EF6E6ED805E15ED810E072D8FEE139
:1018A0000DD067D8FF0806E156D802E06AD8FEE1FD
:1018B000821206D050D802E064D8FEE1E81C8216FD
:1018C0000B01FF2BDED707011F0E03D0FA0503E142
:1018D000F60EFA6F3ED0FA070B01FF6B020EFF5DAA
:1018E00038E240D8EFCFCAF8000E0801E76ECA19F7
:1018F00002E7CA3502D0CA51E75C1EE2030EE66E6B
:10190000FAC7E6FFDEEC60F041E9E750000909E1C3
:101910000B0128D8EF061FD802E033D8FEE182126F
:1019200015D0040E0B01FF250801CA6F010ECA5322
:101930000BE027D8FEE108D00B0114D8EF5006E1E8
:101940000AD802E01ED8FEE1E81C82160B01FF2B2C
:10195000C5D79E901200040EFF250801CA6F010E24
:10196000CA531200FF51EA6AF80FE96E070EEA2225
:101970001200FF51EA6AF60FE96E070EEA22EF50F5
:0A1980001200E846FE0BCA07120031
:06198A0009010091008339
:10199000416B426B436B00950087009B0099C46BC1
:1019A000C56BC66B810EAF6EAC84949C948E9F9871
:1019B0009F9AAC8AAB88AB8E9D889D8AF28EF28C02
:1019C0001200C8D882E9090100A102D0000E16D089
:1019D0009D984251EA6A010FE96E090EEA2200EB76
:1019E000EFFF0093412B400E415D01E10081422B4E
:1019F000400E425D01E1426B9D88010E41E9E7CF57
:101A0000D9FF1200400E0901415D04E2400ED8806A
:101A100041551200000C9ED883E9090100A702D0AD
:101A2000000E23D09D9A0095C651EA6A440FE96ED4
:101A3000090EEA22EF50E66E00EBE9FF01EBEAFF48
:101A4000E552E750EF6EC407C45101E10087C62B91
:101A5000C6510B01D16FD26B800ED11904E1D25166
:101A600002E10901C66B9D8A010E41E9E7CFD9FF6A
:101A700012000901C45112006DD881E941E89D505E
:101A8000100B01E0010E0801C86F9E50100B01E021
:101A9000010EC81519E0090100B314D04351EA6AD8
:101AA000010FE96E090EEA22EF50AD6E00B1009110
:101AB0004107415101E10083432B400E435D46E164
:101AC000436B44D09D9842D09D50200B01E0010E05
:101AD000C86F9E50200B01E0010EC81537E0ABB473
:101AE00004D0ABA207D0AB98AB88AE50016E090111
:101AF000008B2CD0090100A504D0AE50016E0089E6
:101B000025D000B523D000990097C551EA6A440F4B
:101B1000E96E090EEA22AECFEFFFC42BC4510801D3
:101B2000C86FC96B800EC81904E1C95102E10901EF
:101B300000850901C52BC5510801C86FC96B800E0E
:101B4000C81904E1C95102E10901C56B42E9E7CFB7
:0E1B5000D9FF1200D9CFE6FFE1CFD9FF120076
:021B5E00000184
:101B600044030004020400830300003F71D1090014
:101B700084030000CCB22E3200A453465A5245389A
:101B80004200A53135423339393900A63939390097
